:020000040802F0
:1000000038E00220850202082F4B020879420208DC
:100010002D4B020887100208F97502080000000045
:10002000000000000000000000000000C501020800
:1000300029110208000000002102020829580208C4
:100040009F0202089F0202089F0202089F02020804
:100050009F0202089F0202089F0202089F020208F4
:100060009F0202089F0202089F0202089F020208E4
:100070009F0202089F0202089F0202089F020208D4
:100080009F0202089F0202089F0202089F020208C4
:100090009F0202089F0202089F0202089F020208B4
:1000A0009F0202089F0202089F0202089F020208A4
:1000B0009F0202089F0202089F0202089F02020894
:1000C0009F0202089F0202089F0202089F02020884
:1000D0009F0202089F0202081D5D02089F0202089B
:1000E000B51202089F0202089F0202089F0202083E
:1000F0009F0202089F0202089F0202089F02020854
:100100009F0202089F0202089F0202089F02020843
:100110009F0202089F020208115902081D59020895
:100120009F0202089F0202089F0202089F02020823
:100130009F0202087D1102089F0202089F02020826
:100140009F0202089F0202089F020208314B020828
:100150009F0202089F0202089F0202089F020208F3
:100160009F0202089F0202089F0202089F020208E3
:100170009F0202089F0202089F020208000000007E
:100180009F0202089F0202089F0202089F020208C3
:100190009F0202089F0202089F0202089F020208B3
:1001A00000000000000000009F020208DFF810D0ED
:1001B00000F042FD00480047ED270308AFF3008040
:1001C00038E002202C4B19680868B0E8F04F80F343
:1001D0000988BFF36F8F4FF0000080F311887047DC
:1001E0000000000008480068006880F308884FF0AD
:1001F000000080F3148862B661B6BFF34F8FBFF37F
:100200006F8F00DF00BF00BF08ED00E0DFF80C00DB
:10021000016841F470010160704700BF88ED00E0A3
:10022000EFF30980BFF36F8F134B1A681EF0100FA6
:1002300008BF20ED108A20E9F04F106009B44FF09C
:10024000500080F31188BFF34F8FBFF36F8F25F0FD
:10025000EBFC4FF0000080F3118809BC19680868B6
:10026000B0E8F04F1EF0100F08BFB0EC108A80F31A
:100270000988BFF36F8F704734010020EFF30580CA
:10028000704700000648804706480047FEE7FEE743
:10029000FEE7FEE7FEE7FEE7FEE7FEE7FEE7FEE736
:1002A000F5580208AD0102082DE9F05F054600206F
:1002B00092469B4688460646814640241BE02846D7
:1002C00041464746224600F051F853465A46C01A66
:1002D000914110D311461846224600F0D3FA2D1A48
:1002E00067EB01084F4622460120002100F0CAFAC0
:1002F00017EB00094E41201EA4F10104DFDC484643
:1003000031462A464346BDE8F09F2DE9F0410024DE
:10031000061B254671F1000605DA01240027D0EB03
:10032000070067EB0101161E73F1000605DA0027CE
:10033000D2EB0702012567EB0303FFF7B5FF864603
:100340000E4617469C46AC4204D00025D0EB050E65
:1003500065EB010624B10020D2EB000760EB030C33
:10036000704631463A466346BDE8F081202A04DBF8
:10037000203A21FA02F00021704721FA02F3D0401E
:10038000C2F1200291400843194670470048704767
:10039000EC97040810B50446FFF7F8FF0068005D0D
:1003A00000F0010010BD00000649074A08685043EC
:1003B00043F2390210440860400870470149086060
:1003C00070470000640C00106D4EC64110B5431A12
:1003D000934209D28318881803E010F8011D03F82E
:1003E000011D521EF9D210BD40EA01039B0703D044
:1003F00009E008C9121F08C0042AFAD203E011F864
:10040000013B00F8013B521EF9D210BDD2B201E00F
:1004100000F8012B491EFBD270470022F6E710B509
:1004200013460A4604461946FFF7F0FF204610BD62
:1004300030B505462A460B4612F8010B13F8014B5E
:1004400008B1A042F8D01CB1002802D06D1CF1E721
:10045000284630BDCAB2401E10F8011F8A4202D0A1
:100460000029F9D100207047421C10F8011B002917
:10047000FBD1801A704710B5002200E0521C835C4B
:100480008C5CA34201D1002BF8D1D8B2E1B2401A62
:1004900010BD30B504460020034600E05B1C9342CB
:1004A00003D2E05CCD5C401BF8D030BD034611F8B0
:1004B000012B00F8012B002AF9D11846704730B5FE
:1004C00005460020034600E05B1C934205D2EC5C2D
:1004D000C85C201A01D1002CF6D130BD10B54843BC
:1004E000044612F0B3F9002805D00021002C02D0F8
:1004F000641E0155FAE710BD2DE9F04791460F46FD
:1005000080460446002614F8015B2DB1FFF73EFF3C
:100510000068405DC007F6D12B2D02D02D2D18D0DC
:10052000641E4A463946204600F0CDF927B13968A5
:10053000A14201D1C7F8008071054FF002040BD52C
:100540004042002803DD07F0B1FC0460A007BDE8CD
:10055000F08746F48066E4E70028F8DA07F0A6FCA6
:1005600004606FF00040F2E770B5064607F09EFCAD
:10057000046805460A2200213046FFF7BDFF2C60C3
:1005800070BD2DE9FE4F804681EA0300C00F0C4686
:10059000009021F0004123F00045B8EB0200A94192
:1005A00005D24046214690461C460B46024623F0A3
:1005B0000040104347D0270DC7F30A00C3F30A5188
:1005C0000290401A019040286BDAC3F3130040F404
:1005D000801B0098924620B10023D2EB030A63EB04
:1005E0000B0B01985946C0F14002504600F04AF901
:1005F00006460D4650465946019A00F052F910EB56
:1006000008006141002487EA115284EAE7731A4323
:1006100040D0009A62B3019A012A4FEA075215DCD2
:10062000001B61EB02014FF0004202EA0752CDE9E4
:100630000042001C41F5801132462B4600F026FA9C
:1006400003B0BDE8F08F40462146F9E7001B61EB9F
:100650000201001C41F5801300185B412018A2F52F
:10066000001747EB030140EAD570B6196D4111E060
:100670006D084FEA360645EAC0754FEA0752001B7F
:1006800061EB0201001C41F5801149084FEA30007E
:100690000019514132462B4603B0BDE8F04F00F03F
:1006A000E6B90098012240000023D0EB020263EB80
:1006B000E073009821464FEAE074B8EB000061EB6C
:1006C0000401E9E783F000435BE781F0004158E76C
:1006D0002DE9FE4F81EA030404F0004421F00041BB
:1006E00000944FF0000B23F0004350EA01045ED069
:1006F00052EA03045BD0C3F30A54C1F30A552C44F5
:10070000A4F2F3340194A0FB0254C1F3130141F4A9
:100710008011C3F3130343F4801301FB024400FB75
:10072000034E840A970A44EA815447EA8357A4FB9C
:10073000076802958D0A05FB07854FEA932C04FB99
:100740000C542705029D4FEA065847EA1637B5EBC9
:1007500008056EEB070C870E920E47EA811742EAF6
:100760008312A7FB0201B6EB0B0164EB00042B0D17
:1007700043EA0C335E1844EB1C50DA465146E7FB63
:100780000201C5F313044FEA0B3343EA14534FEA53
:100790000432019C43EA0603A4F10C040294009C79
:1007A000CDE900B400F072F903B0BDE8F08F00208D
:1007B0000146F9E70EB5C10F80EAE0700844CA07A8
:1007C000002140F233438DE80E000A460B4600F04C
:1007D0005DF903B000BD0EB540F233410291002136
:1007E000CDE900110A460B4600F050F903B000BDF8
:1007F00030B5041E71F1000404DB4FF000444042A8
:1008000064EB0101141E73F1000405DB1C464FF07C
:100810000043524263EB0403994208BF904230BD4B
:1008200001F0004330B421F0004150EA010206D04B
:100830000A0DA2F56072C1F31301002A02DC30BC7C
:1008400000207047440F44EAC104C100E01830BCE6
:1008500000EBC25000F0D4B830B50B460146002082
:100860002022012409E021FA02F59D4205D303FA72
:1008700002F5491B04FA02F52844151EA2F10102F3
:10088000F1DC30BD202A04DB203A00FA02F100201E
:1008900070479140C2F1200320FA03F319439040BE
:1008A0007047202A06DBCB17203A41FA02F043EAD0
:1008B000E07306E041FA02F3D040C2F12002914019
:1008C0000843194670472DE9F05F824600780027FB
:1008D00015468B460AF10104B946302801D09DB176
:1008E00013E014F8010B0127782803D0582801D011
:1008F00045B10AE00DB1102D07D10027102514F8DD
:10090000010B02E0082500E00A250026B0460EE0B3
:1009100005FB080005FB06F1012701EB10461FFA55
:1009200080F8B6F5803F00D3B94614F8010B29468C
:1009300000F094F90028EBDABBF1000F05D00FB1FD
:10094000641E00E05446CBF80040B9F1000F06D019
:1009500007F0ACFA02210160C81EBDE8F09F48EA2A
:100960000640FAE70FB4002300B589B00CA9009146
:100970000B996FF00042CB601E4B06931E4B079302
:100980000423CDE901321D4A089202466B4600203D
:1009900000F006FA09B05DF814FB70B586B00646A3
:1009A0004FF0FF300091CDE90101002015460C46C3
:1009B00004903246694604A8FFF7D4FF0246049823
:1009C000211825B108B1084600E0204628600498A7
:1009D00000280DD0002A02DD0098884208D0081BAC
:1009E0000094CDE901043246694604A8FFF7BAFF36
:1009F00006B070BDD90F0208F70F02089503020870
:100A00000029A8BF7047401C490008BF20F0010022
:100A1000704710B4B0FA80FC00FA0CF050EA010400
:100A200004BF10BC704749B1CCF1200421FA04F492
:100A300011FA0CF118BF012121430843A3EB0C016B
:100A4000CB1D4FEA00614FEA102042BF002010BCCE
:100A5000704700EBC35010440029A4BF10BC70477E
:100A6000401C490008BF20F0010010BC704710B5C1
:100A7000141E73F1000408DA401C41F100019218C1
:100A80005B411A4301D120F0010010BD2DE9F04D6A
:100A900092469B4611B1B1FA81F202E0B0FA80F2BF
:100AA00020329046FFF7EEFE04460F4640EA0A0069
:100AB00041EA0B0153465A46084313D0114653EA04
:100AC000010019D0C8F140025046FFF74FFC05461F
:100AD0000E46504659464246FFF7D4FE084305D01D
:100AE000012004E020463946BDE8F08D0020054392
:100AF00046EAE0762C4337430A986305E40AA0EB04
:100B000008000022FD0A44EA47540A3002D50020BA
:100B10000146E9E7010510196941DDE908450019B9
:100B20006941BDE8F04DA2E72DE9F04D81EA0304EB
:100B300004F0004B21F0004514464FF0000A23F06A
:100B4000004150EA050220D054EA01021DD0C5F34D
:100B50000A570246C5F31303C1F31300C1F30A5643
:100B600040F4801543F48013A7EB0608101BD6460B
:100B700008F2FD3873EB050002D308F1010801E02B
:100B800092185B41B8F1000F03DA00200146BDE87E
:100B9000F08D00204FF48011064684460EE0171BAE
:100BA00073EB050705D3121B63EB050306434CEA01
:100BB000010C49084FEA300092185B4150EA0107E6
:100BC000EDD152EA030012D082EA040083EA050163
:100BD000084305D0101BAB4106D20122002306E0DA
:100BE00000224FF0004302E06FF0010253101AEBB5
:100BF00006004CEB085110EB0A0041EB0B01BDE87D
:100C0000F04DFFF734BFC1F30A52C1F3130140F2B4
:100C1000FF3341F480119A4202DA00200146704706
:100C200040F233439A42A2F2334202DC5242FFF7CF
:100C30009DBBFFF727BE0000064C074D06E0E068AD
:100C400040F0010394E8070098471034AC42F6D313
:100C5000FFF7B0FA2C9D04086C9D04083A2800D2D6
:100C6000303820F02002412A01D3A2F13700884217
:100C700001D34FF0FF3070472DE9FF4F087883B064
:100C80009946FF2805D0491C2D2804D000240020B7
:100C900008E000200BE00124F9E700EB800003EB03
:100CA0004000491C0B78FF2BF7D104B140420023D0
:100CB0000293147819461D462D2C01D02B2C04D1FB
:100CC000521C2D2C13D000240294AA461478FF2C19
:100CD0000FD00A25A3FB057801FB05814FF0000C1E
:100CE00003FB0C11521CE3194AEB0101EEE701244E
:100CF000EAE7814453EA010002D019F5C87F06DA19
:100D000003980021C0E9001107B0BDE8F08F00256D
:100D1000AE4E2F46DFF8B882184600F07DF9CDE9D7
:100D20000001B9F1000002DAC9F1000400E0044654
:100D30000023A74A1AEB030B42EB045A12E0E00728
:100D400007D02A46334638464146FFF7C1FC0746DE
:100D500088462A46334610461946FFF7B9FC054631
:100D60000E466410002CEAD1DDE90001B9F1000F54
:100D70005A46534606DAFFF7D7FE3A464346FFF790
:100D8000D3FE05E0FFF7A4FC3A464346FFF7A0FC7C
:100D9000029A0AB181F00041039AC2E90001B3E767
:100DA0002DE9FF4F1F468DB0D7E901464FF0FF38C0
:100DB0002E2045464FF000090B90B9696D1C0E9826
:100DC0008847396A824688470028F6D1BAF1FF3F42
:100DD0000AD024F4D064002E11DDBAF12B0F08D014
:100DE000BAF12D0F0BD102E0404611B08DE744F46B
:100DF0008064B9696D1C0E9888478246761E6946E4
:100E0000600501D52D2000E02B208DF8000001F1B8
:100E1000010B0DF1200809E0B9696D1C0E98884797
:100E200082460F9844F40074761E0560002E02DDA1
:100E3000BAF1300FF0D00B998A453ED144F08004CE
:100E400006E00F99681CA9F1010944F400740860D8
:100E5000B9696D1C761E0E98884782463028F0D0FE
:100E60002BE00B998A4505D1200603D444F0800479
:100E7000761E18E0504607F0F3F908B30DF11301A0
:100E8000761E44F400748B4508D2AAF130000BF8AA
:100E9000010B200607D5A9F1010003E0200602D4CA
:100EA00009F101008146A00502D50F99681C086070
:100EB000B9696D1C0E9888478246002ED1DC53E03C
:100EC000002E51DDBAF1650F02D0BAF1450F4BD1BA
:100ED000A00549D5B9696D1C24F44074761E0E989E
:100EE00088478246002E0CDD2B2804D0BAF12D0F46
:100EF00007D144F48074B9696D1C0E988847824606
:100F0000761EE00501D52D2100E02B2108F8011BFC
:100F1000CDF82C8021E00DF12901761E44F40074F7
:100F200088450CD2AAF1300010F0FF0088F80000CC
:100F300002D10B99884509D908F1010806E0E005BE
:100F400001D5244801E042F20F708146B9696D1C59
:100F50000E98884782460F980560002E04DD5046A3
:100F600007F07EF90028D6D1F9690E988847FF204E
:100F70008BF8000088F800000020069007904B4690
:100F80006A4608A906A8FFF777FEA00502D46FF00D
:100F900001002AE714F0240F0AD0E00714D1DDE99C
:100FA00006123868031D3B600068C0E900120BE0C0
:100FB000DDE90601FFF734FC0146E00704D138689B
:100FC000021D3A600068016028460EE700001440E8
:100FD0000000F03FF1D8FFFF426842B1016811F80C
:100FE000013B23B1521EC0E900121846704701218F
:100FF000C160881E704742685AB1C368016843B92E
:1010000083688B4205D0491E521CC0E900120020A3
:1010100070474FF0FF3070470EB540F233420292F6
:101020000022CDE900221346FFF730FD03B000BDDA
:1010300070B58C1810F8015B15F0070301D110F89A
:10104000013B2A1106D110F8012B03E010F8016BC7
:1010500001F8016B5B1EF9D12B0705D40023521E4A
:101060000DD401F8013BFAE710F8013BCB1A921CB2
:1010700003E013F8015B01F8015B521EF9D5A142B0
:10108000D8D3002070BDFEE70020704700207047D5
:1010900010B500220449054804F063FF04490348E1
:1010A00004F056FF002010BD042A0020D82A0010AA
:1010B0000422002010B50AF045FA024804F02DFF82
:1010C000002010BDD82A001000207047094A10B532
:1010D000D2F8BC22D2F814220AB1012010BD0A466F
:1010E0000146044804F03DFFBDE81040014804F00B
:1010F000A2BF0000D82A001008B509480C2102231D
:101100000170002141704FF4FA600090044AD02130
:10111000044801F07BFABDE8084000F0CFB80000B9
:101120006C0000205C02002070470000064908B5F2
:1011300009684FF4FA52B1FBF2F14143009100BF4C
:10114000491E0091FBD208BD940A001038B5044630
:10115000006800F58050816941F480118161206848
:1011600000F58050806900900120FFF7DFFF2068C4
:10117000009900F58050816138BD0000014800F001
:101180005ABC0000CC6800202DE9F041044621B192
:101190004FF40060E060C000A060E0690025002816
:1011A00061D02A462368402619683C480140D4E9AA
:1011B00002073843104340F4007008431860206869
:1011C0000768012000F06AFB20680760206846601D
:1011D00020684668012000F061FB206846602068B6
:1011E00085602068C560216888694FF641721040AB
:1011F00040F08000886120688669012000F04EFB85
:10120000206886612068C5612068C569012000F0FA
:1012100045FB2068C561216801F580518869204A35
:101220001040204A02438A61206800F58050856999
:10123000012000F033FB206800F5805085612068B4
:10124000194900F580500160206800F5805005685C
:10125000012000F023FB206800F580500560A069A4
:10126000012803D009E04FF480629BE7206800F575
:101270008050C1690D4A1143C16160690C4A81887F
:1012800011640178C37841EA0361837840781B04D4
:1012900043EA002001435164BDE8F0810F8120FF43
:1012A000233FDEF8040020028020C102400001003C
:1012B000008002404FF4805000F0C0BE10B5D8B19D
:1012C0000E4C0228216805D18869800702D503F0F9
:1012D0005DFB0FE0486910F4F85F0BD0086820F060
:1012E00001000860012013F07AFD2068016841F0D8
:1012F00001010160002010BD012010BD5C02002032
:1013000072B6FEE7002200F001B8000030B50E4BC7
:10131000054601205C7A002C14D1587A1C54587A66
:1013200003EB800045605D7A03F108002A54587A87
:10133000421C5A72303008703A2048702F20887052
:10134000CC70002030BD0000146900202DE9F05F52
:101350008B463849924600EA0107C0F3080400F0C2
:10136000E9F8DFF8D48053213E0C88F80010C7F369
:10137000072588F80160DFF8C49088F80250FFB2B2
:1013800088F8037000220121484600F080FF042104
:10139000404619F0E7FF01221146484600F077FF6A
:1013A0000020401CC0B20528FBD300F0C3F8842104
:1013B00088F80010210C88F80110210A88F8021022
:1013C00088F80340002201214C46484600F05FFFA8
:1013D0000421194819F0C6FF5946504619F0C2FFBA
:1013E00001221146204600F052FF0020401CC0B2EE
:1013F0000528FBD300F09EF8832188F8001088F8B8
:10140000016088F8025088F803700022012120460C
:1014100000F03DFF0421084819F0A4FF0122114605
:10142000204600F034FF0020401CC0B20528FBD34A
:10143000BDE8F09F00FE3F00EC080010000C0240E9
:1014400070B516460D46044600F074F81248E821BF
:101450000170210C4170210A8170C470002101715A
:1014600041718171C1710D4C0A460121204600F085
:101470000EFF0821084819F075FF2946304619F07B
:1014800067FF01221146204600F001FF0020401CAA
:10149000C0B20528FBD370BDEC080010000C024060
:1014A00070B5054600F046F80D499F200D4C0870B8
:1014B00000220121204600F0EAFE0121084819F02F
:1014C00051FF0421284619F043FF0122114620460E
:1014D00000F0DDFE0020401CC0B20528FBD370BD2B
:1014E000EC080010000C024010B510483D21104CD3
:1014F00001702A21417080218170A621C1700022D3
:101500000121204600F0C3FE0421084819F02AFFFB
:1015100001221146204600F0BAFE0020401CC0B255
:101520000528FBD3BDE8104000F004B8EC0800101B
:10153000000C024038B51049D720104C087000222A
:101540000121204600F0A3FE01210B4819F00AFFFB
:101550000121684619F0FCFE9DF800000006F7D551
:1015600001221146204600F092FE0020401CC0B22D
:101570000528FBD338BD0000EC080010000C024029
:1015800070B50D460146002001E0401CC0B20A5C67
:101590002E2AFAD108440446052224A1FEF78FFF23
:1015A000002833D02046042222A1FEF788FF00281D
:1015B0002ED02046052221A1FEF781FF002829D048
:1015C000204603221FA1FEF77AFF002824D02046E0
:1015D00004221DA1FEF773FF00281FD0204605221C
:1015E0001BA1FEF76CFFD8B1204604221AA1FEF71A
:1015F00066FFB8B12046042219A1FEF760FF98B13A
:1016000019A12846BDE87040FEF750BF19A1F8E7C0
:101610001BA1F6E71DA1F4E721A1F2E724A1F0E761
:1016200026A1EEE728A1ECE72AA1EAE72E68746D6F
:101630006C0000002E637373000000002E6A736F4D
:101640006E0000002E6A73002E67696600000000BD
:101650002E6A7065670000002E706E670000000043
:101660002E69636F00000000746578742F706C61E0
:10167000696E0000746578742F68746D6C000000EA
:10168000746578742F637373000000006170706C70
:1016900069636174696F6E2F6A736F6E000000007A
:1016A000746578742F6A617661736372697074000F
:1016B000696D6167652F676966000000696D616724
:1016C000652F6A7065670000696D6167652F706ED0
:1016D00067000000696D6167652F766E642E6D6925
:1016E00063726F736F66742E69636F6E0000000023
:1016F0007CB514490446122008704FF4FA650A4676
:101700000123D0211048009500F080FFFFF7D6FD9F
:10171000002815D0012301AAD0210B48009500F024
:1017200085FEFFF7CBFD00280AD09DF804100806BF
:1017300002D521F0800000E0C8438DF8040020703D
:101740007CBD00006C0000205C020020F8B505465E
:10175000807A504C80064FF00F074FF4FA660FD591
:101760002078022320F00400607027702246D021E8
:101770004948009600F04AFFFFF7A0FD00287DD001
:10178000012020700346434AD0214348009600F0D0
:101790003DFFFFF793FD00287BD007233D4AD02172
:1017A0003D48009600F042FEFFF788FD002870D00B
:1017B0002078012300F00F01C0F3021000EB80003D
:1017C00001EB4000E871607800F00F01C0F30210F7
:1017D00000EB800001EB40002872A07800F00F01C0
:1017E000C0F3011000EB800001EB4000687220792B
:1017F00000F00F01C0F3011000EB800001EB40008E
:10180000A870607900F00F01C0F3001000EB8000B9
:1018100001EB4000E870A07900F00F01000900EB37
:10182000800001EB4001A078800900EBC00202EBD0
:10183000001001EB800000F5FA60A8802770154ABF
:10184000D0211548009600F0E1FEFFF737FD002893
:101850001FD001230F4AD0210F48009600F0E6FD6B
:10186000FFF72CFD002814D02078A97AC20962F372
:101870000001420962F34201020900E009E062F35B
:10188000C301C20862F30411800860F34511A97214
:101890000120F8BD6C0000205C02002070B50446F9
:1018A00000F0FAFC0546601C02D0044800780444AD
:1018B00000F0F2FC401BA042FAD370BD880A001071
:1018C0002DE9F04390F845400025012C0DD04FF054
:1018D000010C80F845C0022480F8444044F2F457DB
:1018E0004FF000495E1E816217E00220BDE8F083E0
:1018F00001EB4514C4F80090C5EBC51808EB480887
:1019000002EB8808C4E90178B54204D204F120084A
:10191000C4F80C8000E0E1606D1C9D42E8D30268D1
:1019200002F58052D16080F844C0002180F8451053
:101930000846DBE72DE9F043914690F84520002466
:10194000012A0AD0012680F84560022280F844204E
:101950004FF4801C5D1EC1621BE00220BDE8F083D5
:1019600001EB4412C2F800C0C4EBC41707EB4708F0
:1019700009EB88079760C7691FB9176847F44007E4
:101980001760AC4203D202F12007D76000E0D160BB
:10199000641C9C42E4D3026802F58052116180F815
:1019A0004460002180F845100846D7E7704730B5FD
:1019B00090F845100023012908D0012280F8452025
:1019C000022180F844100024816A1AE0022030BD10
:1019D0000D685B1CC5F30125022D0AD00D6815F4B6
:1019E000407F09D04163836B5B1C8363012B12D062
:1019F00012E08263016302E0856B6D1C8563C96838
:101A000081620D68002D01DB042BE1D300F8442F27
:101A10004470012030BD01630B68C3F30D431B1FED
:101A2000C363036B9B680364C96840F8281F02778F
:101A30004477002030BD70B50446006800F5805042
:101A400041694FF0000549064FF0010608D52046D0
:101A500000F0DAF92068402100F58050416109E08A
:101A60004069C0070AD0204600F09CFA206800F5C3
:101A70008050466184F8446084F8455020684FF4F3
:101A8000803100F580504161206800F58050406948
:101A900000040CD52046FFF789FF20684FF4004171
:101AA00000F58050416184F8446084F8455070BD71
:101AB0002DE9FC474FF000060400B146009603D024
:101AC00094F8440018B107E00120BDE8FC8784F8D1
:101AD0004560204600F0E2F86648016841F4804124
:101AE0000160006800F4804001906348016821F4BF
:101AF000000101600168226A11430160206800F55D
:101B00008050016841F00101016000F0C5FB05460D
:101B10004FF4FA7709E000BF00F0BEFB401BB8426B
:101B200003D9032004F8440F67E0206800F58050D3
:101B30000068C007F0D12068006920F01C0501F0A2
:101B400045FC4E494E4A0144914202D245F00805F7
:101B500016E04C494C4A0144914202D245F00C0532
:101B60000EE04A494A4A0144914209D3494908448E
:101B70004949884202D245F0040501E045F01005CC
:101B8000206805614FF400420021204600F00CFA65
:101B90000125A8BBFF20FFF781FE606888B300F035
:101BA0007BFB804641F288376A460121204600F0DF
:101BB000E9F800F071FBA0EB0800B84217D80098D4
:101BC0004007F1D54FF480520021204600F0ECF997
:101BD000B0B900F061FB80466A460121204600F062
:101BE000D1F800F059FBA0EB0800B8420AD9012156
:101BF0002046FFF7C9FA04F8445F0320667064E7E3
:101C000024E018E000988006E6D56A4610212046B8
:101C100000F0B8F8D0B90098410703D54FF400613F
:101C2000E16000E0E660800701D5A66019E04FF4AE
:101C30008040A06015E0E068A168C00840EA51005B
:101C400082B20021204600F0AFF930B101212046D8
:101C5000FFF79AFA84F8445036E740F6FF70FFF732
:101C60001DFE49462046FFF78FFA84F844500020B5
:101C70002BE70000443802400438014000D3CEFE78
:101C8000C0E1E40040F1E9FD40787D0100796CFCA1
:101C9000005A6202001F0AFA80F0FA02F0B587B01B
:101CA000044614216846FEF7B8FB31492068884293
:101CB0005BD130480024016841F000710160016887
:101CC00001F000710591016841F0806101600168D7
:101CD00001F080610591016841F0006101600168D7
:101CE00001F000610591016841F0040101600168A3
:101CF00001F004010591016841F0010101600168F2
:101D000001F001010591016841F0020101600068E4
:101D1000022500F0020005903220CDE9000502AA5C
:101D200003260B2782E8D0006946134800F092F999
:101D30008620CDE9000502AA694682E8D0000F4856
:101D400000F088F94FF46050CDE9000502AA694619
:101D500082E8D0000A4800F07DF9002205213D20EC
:101D600000F0B2FD3D2000F0A1FD07B0F0BD000085
:101D7000008002403038024000080240000002406B
:101D8000000402402DE9F047044690F844009146D3
:101D900082281DD0822084F84400226810694FF602
:101DA000FF7500F01C03208A05EAC02018434FF499
:101DB000F86303EA8111014321F0020040F00105BC
:101DC000156100F069FA064601274FF4803810E0EB
:101DD0000220BDE8F08700BF00F05EFA801B40459E
:101DE00005D304F8447F002060700320F1E72068E9
:101DF0000569E807F0D12068406981B2C9F8001090
:101E000084F844700020E4E70148006813F016B934
:101E10001C010020F8B5044690F84500012839D08F
:101E2000012584F84550022084F8440020680026EB
:101E3000016841F0080101602068006800902846B0
:101E4000FFF774F92168009808602068016841F084
:101E5000040101602068006800900120FFF766F926
:101E60002168009808602046FFF770F9206800F5A7
:101E70008050816941F400518161206800F58050F3
:101E8000816941F00201816184F8445084F8456021
:101E90000020F8BD0220F8BDF0B590F845200023E1
:101EA000012A11D0012680F84560022280F84420E2
:101EB000002559B1C76A3A68002A0ADA122100F8E7
:101EC000441F45700120F0BD0220F0BD00F8446FB2
:101ED000F7E740F2F454A1420BD9B1FBF4FCB1FB9B
:101EE000F4F204FB1C1CBCF1000F00D0521C012AB0
:101EF00043D13A6842F040523A60C26AC1F30C01E1
:101F00005160C16A0A6842F000420A60C16AC96849
:101F1000C16234E0C76AD7F800C02CF0405CC7F853
:101F200000C033B9C76AD7F800C04CF0805CC7F86E
:101F300000C0C76A7C60571EBB4214D1C76AD7F87D
:101F400000C04CF0005CC7F800C0C2F10107C7EB4D
:101F5000C71707EB4707D0F82CC001EB8707C7F37B
:101F60000C07CCF80470C76AFF68C762D7F800C0D6
:101F70004CF0004CC7F800C05B1C9342CAD3BFF3BF
:101F80004F8F016801F580514A69520705D5042237
:101F90004A61016801F580514D6000F8446F457059
:101FA0000020F0BD704700002DE9F041044690F894
:101FB000440042281ED0422084F844002368186957
:101FC0004FF6FF7600F01C05208A06EAC020284361
:101FD0004FF4F86505EA8111014390B241F0030521
:101FE00058612068056100F057F9064601274FF453
:101FF000803810E00220BDE8F08100BF00F04CF90D
:10200000801B404505D304F8447F00206070032006
:10201000F1E720680569E807F0D184F84470EAE741
:1020200008B5B0F5805F06D10020009002486946EF
:10203000C06823F09DFF08BD00000020044910B5D2
:102040000A68024202D00860FFF7EAFF10BD0000F4
:10205000143C01402DE9F84FDFF8F4A100220124DF
:102060000AF1040B03254FF00F090BF1040E00BF1A
:102070000B6804FA02F63340B3426FD10F7907F0D0
:102080000307012F01D0022F16D187684FEA4208BB
:1020900005FA08FC27EA0C07D1F80CC00CFA08FC7A
:1020A0004CEA070CC0F808C04768B7430E79C6F37E
:1020B000001696403E4346600E79F643B6070AD0B6
:1020C000C7684FEA420C05FA0CF6B7438E6806FA69
:1020D0000CF63E43C6600E7906F00306022E10D1C0
:1020E000D60800EB8608D8F8206057074FEAD76C6F
:1020F00009FA0CF7BE430F6907FA0CF73743C8F823
:10210000207006684FEA420C05FA0CF7BE430F79BF
:1021100007F0030707FA0CF7374307604E68F6002D
:102120001CD54C4E376847F480473760366822F03C
:10213000030706F480460096474E07EB060CDCF8D2
:10214000086897073F0F09FA07F826EA0806DFF83C
:102150000C81404503D14FF0000841E072E0DFF808
:102160000081404502D14FF0010839E0DFF8F480EA
:10217000404502D14FF0020832E0DFF8EC804045E4
:1021800002D14FF003082BE0DFF8E080404502D198
:102190004FF0040824E0DFF8D880404502D14FF02A
:1021A00005081DE0DFF8CC80404502D14FF006085D
:1021B00016E0DFF8C480404502D14FF007080FE079
:1021C000DFF8B880404502D14FF0080808E0DFF89A
:1021D000B080404502D14FF0090801E04FF00A08F5
:1021E00008FA07F848EA0608CCF80888DAF8006028
:1021F0005746D1F804C09E435FEACC3C00D51E434D
:102200003E60DBF800605F46D1F804C09E435FEAA1
:102210008C3C00D51E433E60DEF800607746D1F866
:1022200004C09E435FEACC2C00D51E433E60084F9D
:102230000C373E68D1F804C09E435FEA8C2C00D571
:102240001E433E60521C102AFFF412AFBDE8F88F07
:10225000003C014044380240003001400000024090
:102260000004024000080240000C0240001002403E
:102270000014024000180240001C024000200240EE
:10228000002402400069084000D0012070470AB1D4
:10229000816170470904FBE70148806870470000CE
:1022A000880A001070B5040025D094F83D00002580
:1022B00020B984F83C50204600F03EFA242084F8EF
:1022C0003D002068016821F001010160206801687B
:1022D00041F4004101602068016821F4004101607F
:1022E00001F07AF84D4A6168914201D84C4900E00A
:1022F0004C49884201D2012070BD4B492368B0FB94
:10230000F1F15E6826F03F060E435E60636893421B
:1023100006D94FF4967359434FF47A73B1FBF3F136
:102320002368491C1E6A26F03F0631431962616822
:10233000914210D84900401EB0FBF1F2521CC2F38A
:102340000B02042A01D2042022E0B0FBF1F0401C71
:10235000C0F30B001CE0A268F2B301EBC10303EB76
:102360000116431EB3FBF6F35B1C43F480431B05CD
:1023700049D092B301EBC10202EB0111401EB0FB48
:10238000F1F0401CC0F30B0040F4804040F40040EA
:102390002168CA694CF6FF739A431043C861D4E9B7
:1023A000071001432068026822F0C0021143016057
:1023B000D4E9030101432068826848F2FF339A435D
:1023C00011438160D4E9050108432168CA6822F0FD
:1023D000FF021043C86001E00EE016E020680168CB
:1023E00041F0010101602564202084F83D0025634F
:1023F00084F83E50002070BD01EB4106431EB3FB44
:10240000F6F35B1CB3E70120C2E701EB4101401E7C
:10241000B0FBF1F0401CC0F30B00B7E7A086010051
:1024200080841E0000093D0040420F002DE9F84F56
:102430001F4690468A460446DDF82890FFF72CFF99
:10244000054694F83D00202875D1192301226C49D6
:102450002046009502F012F80028F5D194F83C00CF
:10246000012868D0012084F83C0020680168C90771
:1024700003D1016841F0010101602068016821F485
:1024800000610160222084F83D00102084F83E00A5
:1024900000262664C4F824806785608D208559480D
:1024A000E0622B464A465146204601F0FDFE0028D8
:1024B00078D1208D544F68B1012814D002282068AB
:1024C000016816D041F4806101602068416980692B
:1024D000009087E02068416981690091016841F4BA
:1024E000007101607EE02068016821F48061016074
:1024F000F0E721F4806101602068016841F4006127
:10250000E2E7032848D801280AD0022814D04B4615
:10251000002239462046009501F0B0FFD8BB27E0E5
:102520002A464946204602F028F8A0BB20680069E8
:10253000616A08704DE061E04B4600223946204652
:10254000009501F09BFF30BB2068016841F40071E9
:10255000016020680069616A0870606A401C6062FE
:10256000218D491E2185618D491E618521682EE0DE
:102570002068016821F48061016020680069616A57
:102580000870606A401C6062208D401E2085608D4E
:10259000401E6085D0E705E02A464946204601F006
:1025A000ECFF10B10120BDE8F88F20680069616A76
:1025B0000870606A401C6062218D491E2185618D12
:1025C000491E618521684A69D24352070AD40969C4
:1025D0000170606A401C6062208D401E2085608D05
:1025E000401E6085208D00288BD1202084F83D007E
:1025F00084F83E6084F83C600020D4E70220D2E7F3
:10260000020010000000FFFF040001002DE9F84F58
:102610001F4690468A460446DDF82890FFF73CFEA8
:10262000054694F83D0020287FD119230122404916
:102630002046009501F022FF002876D194F83C0056
:10264000012872D0012084F83C0020680168C90785
:1026500003D1016841F0010101602068016821F4A3
:1026600000610160212084F83D00102084F83E00C4
:1026700000262664C4F824806785608D20852D4857
:10268000E0622B464A465146204601F083FE90B94F
:10269000206841698069009036E02A464946204614
:1026A00001F09EFF50B1206C042804D1206801681D
:1026B00041F4007101600120BDE8F88F606A216873
:1026C00000780861606A401C6062618D491E618506
:1026D000218D491E89B2218522685369DB435B073E
:1026E0000BD451B100781061606A401C6062608D4B
:1026F000401E6085208D401E20852A464946204682
:1027000001F096FE0028CED1208D0028C5D154F8C6
:102710003D0B016841F400710160202004F81E099E
:10272000E67766770020C7E7FFE70220C4E70000EE
:10273000020010000000FFFF10B586B0044614210F
:102740006846FDF76AFE1A49206888422DD1016863
:1027500041F4004101606420FFF7A0F8206801689F
:1027600021F4004101601348016841F00201016059
:102770000068694600F0020005904FF44070009038
:102780001220019001200290032003900420049065
:102790000948FFF75FFC07481030016841F4001159
:1027A0000160006800F40010059006B010BD000044
:1027B0000054004030380240000402400248816862
:1027C0000278114481607047880A00100B4810B5E8
:1027D000016841F400710160016841F480610160A9
:1027E000016841F480710160032000F08DF8002041
:1027F00000F006F800F03EF8002010BD003C02405A
:1028000010B5014688B00022362000F05DF8362071
:1028100000F04CF813480024016841F010010160F9
:10282000006805A900F010000690684600F0AEFDB3
:1028300000F0D2FD0C494000B0FBF1F10C480B4A0E
:10284000491E026040F2E732C0E90324C0E90114E6
:1028500001F0FDFA10B1012008B010BD044801F0EC
:1028600025FBF9E74038024040420F0000100040CD
:10287000A41300100C4882B0016841F4804101604B
:10288000006800F4804000900748001F016841F094
:10289000805101600068002200F0805000900F21FC
:1028A000901E02B000F010B844380240002809DB46
:1028B00000F01F02012191404009800000F1E0205A
:1028C000C0F8001170470000F0B40E4B1B680C46B6
:1028D000C3F30223C3F10705042D00D90425191DF4
:1028E000072901D2002300E0DB1E012606FA05F1CC
:1028F000491E214099409E40761E16403143F0BC4F
:1029000005F0C4BA0CED00E0064900F007020868C3
:102910004FF6FF03184040EA0220034A10430860C4
:10292000704700000CED00E00000FA0570470068F9
:10293000416200207047F0B50368586A39B19C6A5B
:102940004FF4827600EB144400204D1E0AE040EA6A
:10295000024098620FE006EB8007DF59401C04EB51
:102960001744C0B2A842F6D344EA02404FF4807242
:1029700002EB810158500020F0BDD0F8040403F0B0
:1029800091BDC1EBC10200EB8202D0F80404926C4D
:1029900003F0FEBCC1EBC10200EB8202D0F80404DC
:1029A000D2F8082203F048BDD0F8040403F07CBD3F
:1029B00070B504460B0601F00F00C0EBC00104EB3C
:1029C00081014FF001024FF0000503D581F83D2051
:1029D0003C3103E081F8FD5101F5FE71087094F877
:1029E000BC03012808D084F8BC23206804F016F941
:1029F00084F8BC53002070BD022070BD70B5044641
:102A000001F00F006268904201D9012070BD0B06F1
:102A100001F00F01C1EBC10104EB81014FF0010294
:102A20004FF0000503D581F83D203C3103E081F8EB
:102A3000FD5101F5FE718D70087094F8BC030128FA
:102A400008D084F8BC23206804F0E2FA84F8BC5370
:102A5000002070BD022070BD01F00F01C1EBC1016B
:102A600000EB8100D0F8140270472DE9F0410446D4
:102A70000F0601F00F00C0EBC00104EB81014FF025
:102A800001064FF0000503D581F83D603C3103E0BD
:102A900081F8FD5101F5FE7108708A60CB704A78AB
:102AA00002B1C880022B00D10D7194F8BC0301283B
:102AB00009D084F8BC63206804F00CF8284684F838
:102AC000BC53BDE8F0810220FBE770B50C4601F075
:102AD0000F05C5EBC50100EB8101C1F81032C1F84B
:102AE00008220023C1F8143281F8FD3181F8FC512D
:102AF000036901F5FE71012B00D10A612207027CF6
:102B0000006803D004F0DCFA002070BD04F0C8F9BE
:102B1000FAE770B504460D4601F00F00616888427F
:102B200001D9012070BD29064FF000064FF00102C7
:102B300007D5C0EBC00104EB810181F83D203C3199
:102B400007E0C5EBC50104EB810181F8FD6101F5EA
:102B5000FE718A70087094F8BC03012807D084F8CD
:102B6000BC23206804F080FA280702D007E0022086
:102B700070BD217C04F57172206804F01DFA84F8A0
:102B8000BC63002070BD70B50C4601F00F05C5EBAD
:102B9000C50100EB81010B658A6400234B650123AD
:102BA00081F83D3001F83C5F0369012B00D10A61D7
:102BB0002207027C006803D004F082FA002070BD76
:102BC00004F06EF9FAE700002DE9FC5F05680446A1
:102BD000284604F09EFB00287ED1206804F0C5FB47
:102BE000002879D0206804F0C0FB800704D5216854
:102BF000486900F002004861206804F0B6FBC10695
:102C000004F57170009034D52068816921F01001BD
:102C100081612F6A07F00F00C0EBC00004EB800653
:102C2000C7F3434006F5FE76022802D0062811D0ED
:102C30001AE047F6F070074216D0C7F30A1217469B
:102C40002846F16804F095FBF0683844F060B069FC
:102C5000384408E008222846009904F08AFBB0694D
:102C6000C7F30A110844B0612068816941F010017E
:102C70008161206804F079FB00034FF0010A4FF0F6
:102C8000080B5BD50026206804F04EFB0746DFF8F2
:102C9000689351E0F8074DD0F1B2206804F05DFB75
:102CA0008046C00707D005EB4611C1F808AB314696
:102CB000204601F043FF5FEA087022D505EB46117C
:102CC000C1F808BB2068016C00EB46100191D0F8F8
:102CD000082B494507D900E08BE1110403D54FF4D7
:102CE0000041C0F8081B204600F076FA01984845DC
:102CF00007D92069012804D120680121009A04F035
:102D00005BF95FEAC86004D505EB46111020C1F8F5
:102D1000080B5FEA886004D505EB46112020C1F856
:102D2000080B5FEA884005D505EB46104FF40051CB
:102D3000C0F8081B7F08761C002FABD1206804F078
:102D400014FB40034FF000095CD5206804F0E5FA5D
:102D50000746002654E0F80750D0F1B2206804F08E
:102D6000EAFA8046C00723D006F00F020AFA02F002
:102D7000D5F834288243C5F8342805EB4610C0F84E
:102D800008A9206901280FD1C6EBC60004EB80001A
:102D9000D0E911211144816436B9206D20B9206831
:102DA0000121009A04F008F9F1B22046FFF7E9FD8D
:102DB0005FEA087003D505EB4611C1F808B95FEA70
:102DC000C86004D505EB46111020C1F808095FEA78
:102DD000486004D505EB46114020C1F808095FEAB8
:102DE000887004D505EB46110220C1F808095FEA96
:102DF000086003D53146204601F006FF7F08761CA7
:102E0000002FA8D1206804F0B0FA002811DAD5F814
:102E1000040820F00100C5F8040894F8F403012820
:102E200029D0204600F0BCF92068416901F000413A
:102E30004161206804F099FA00050BD5D5F808081F
:102E4000C00702D0204600F0EFF92068416901F484
:102E500000614161206804F088FAC00468D5D5F8A3
:102E6000040820F00100C5F804081021206804F0CF
:102E700031FA002127E084F8F49300212046FFF77F
:102E800055FDD1E705EB41104FF67F32C0F8082918
:102E9000D0F8003923F40013C0F80039D0F8003915
:102EA00043F00063C0F80039C0F8082BD0F8002BBD
:102EB00022F40012C0F8002BD0F8002B42F0006280
:102EC000C0F8002B491C60688842DBD8D5F81C0884
:102ED00040F00110C5F81C08206B60B1D5F88408DB
:102EE00040F00B00C5F88408D5F8440840F00B000A
:102EF000C5F844080CE0D5F8141842F22B00014341
:102F0000C5F81418D5F8100840F00B00C5F81008E3
:102F1000D5F8000820F4FE60C5F80008217C206880
:102F2000009A04F049F82068416901F48051416138
:102F3000206804F01AFA800415D5206803F00AFE10
:102F4000206804F0D9F9E06000F040FA0146227BE5
:102F5000206804F045FA204600F00CF92068416929
:102F600001F400514161206804F0FFF9000707D522
:102F7000204600F019F92068416901F0080141611B
:102F8000206804F0F2F9C00208D50021204600F0C4
:102F900035F82068416901F480114161206804F02E
:102FA000E4F9800208D50021204600F02BF82068C3
:102FB000416901F400114161206804F0D6F9400034
:102FC00007D52046FFF7D9FC2068416901F0804110
:102FD0004161206804F0C9F940070AD520684568B6
:102FE000680702D52046FFF7DFFC206841682943C7
:102FF0004160BDE8FC9F00000A30544FD0F8040443
:1030000003F0A2BAD0F8040403F0AEBA2DE9F041FF
:103010008AB0040005D094F8BD032668002520B1CD
:1030200008E001200AB0BDE8F08184F8BC532046D6
:1030300000F05EF8032084F8BD03F06BC00500D4F7
:103040002561206803F026FF04F11001282288463C
:103050006846FDF7BBF994E80F0003F089FD0226EE
:10306000C8BB0021206804F092F9002001270EE07F
:10307000C0EBC00104EB810181F83D7001F83C0F09
:10308000C880CD708D60CD60401CC0B24D6161685C
:103090008142EDD8002011E0C0EBC00104EB8101BA
:1030A00081F8FD5181F8FC0181F8FF51C1F804520B
:1030B000C1F80852401CC0B2C1F810526168814288
:1030C000EAD8282241466846FDF780F994E80F00C7
:1030D00003F026FE10B184F8BD63A2E784F83850EF
:1030E00084F8BD73206803F00DFE00209AE700000D
:1030F00010B586B0044614216846FDF78EF92068A5
:10310000B0F1A04F2FD119480021026842F001020E
:103110000260006800F0010005904FF4C05000907C
:103120000220CDE90101032003900A2004906946A2
:103130000F48FEF78FFF0D48001D016841F0800128
:1031400001600A481430016841F480410160006860
:10315000002200F48040059005214320FFF7B4FBD6
:103160004320FFF7A3FB06B010BD0000303802403B
:103170000000024070B50446C068012570B1022805
:1031800001D0FEF7BDF82946D4F8040403F058FA3C
:10319000D4F80404BDE8704003F00BBA0025F2E750
:1031A000D0F8040403F032BAD0F8040403F038BABB
:1031B00010B5044690F8BC0301280BD0012084F818
:1031C000BC0384F83810206804F0F8F8002084F874
:1031D000BC0310BD022010BDD0F8042400F57171AD
:1031E000104603F039BA10B50446006894F8BC13D1
:1031F000012906D0012184F8BC13A16A012902D05B
:1032000008E0022010BDA169012903D0816B41F4BF
:1032100080318163206804F047F8206803F064FD82
:10322000002084F8BC0310BD10B50446D0F8040497
:1032300003F054FA2068D0F8001E41F00101C0F8F4
:10324000001E206A002804D00248016841F00601EF
:10325000016010BD10ED00E02DE9F0470E460500BD
:1032600065D0DFF81481D8F80000F7B200F00F0045
:10327000B04207D288F80070D8F8000000F00F00C4
:10328000B04254D128683D4C810712D5400703D580
:10329000206840F4E05020602878000703D52068BB
:1032A00040F4604020602068A96820F0F0000843E6
:1032B00020602878C0072DD0304968680839012877
:1032C00012D0022813D0032811D0096889070029D9
:1032D0002DDA216821F0030101432160FEF7DCFFB4
:1032E000814641F2883A0EE009688903EFE70968F0
:1032F0008901ECE7FEF7D0FFA0EB0901514502D9A7
:103300000320BDE8F0872068696800F00C00B0EB8E
:10331000810FEFD1D8F80010404601F00F01B14203
:1033200007D90770006800F00F00B04201D00120FB
:10333000E7E72878400705D52068E96820F4E050E1
:10334000084320602878000706D52068296920F402
:10335000604040EAC100206000F05EF82168084A41
:10336000C1F30311515CC840064908600648006873
:10337000FFF746FA0020C4E7003C0240083802404C
:103380005C7D0408940A00108C0A00100F22026071
:103390000C4A136803F003034360136803F0F0035F
:1033A0008360136803F4E053C36012684FF4E05382
:1033B00003EAD20202610448006800F00F000860CE
:1033C0007047000008380240003C02400148006895
:1033D00070470000940A0010044805490068096815
:1033E000044AC1F38221515CC8407047940A00101E
:1033F000083802406C7D04080448054900680968E3
:10340000044AC1F34231515CC8407047940A00102D
:10341000083802406C7D0408154810B5006810F0AB
:103420000C02144813D01449042A0FD0082A0ED1D4
:103430000F4C241F2268236802F03F025B0207D56D
:103440002068C0F38810A0FB010106E0084610BD0B
:103450002168C1F38811A1FB00010023FCF724FFC0
:103460002168C1F30141491C4900B0FBF1F010BDD6
:10347000083802400059000140787D01F0B51F4C2A
:1034800016460D461D4B002102220327283C00282A
:10349000186887B019D040F004001860186800F070
:1034A0000400059010020090CDE90121CDE90371DF
:1034B00069461348FEF7CEFD206845EAC60120F0B4
:1034C00078400843206007B0F0BD40F0010018606C
:1034D000186800F0010005904FF480700090CDE96D
:1034E0000121CDE9037169460648FEF7B3FD206866
:1034F000354320F0EC602843E4E700003038024018
:1035000000080240000002402DE9F84F04006ED090
:103510002078DFF84C93C007A9F104054AD009F1DF
:1035200004000168C1F38101012908D00068C0F3DB
:10353000810002280AD1D9F80000400206D5286887
:10354000800337D560680028E1D033E06068B0F5CB
:10355000803F10D0B0F5A02F286810D020F4803024
:103560002860286820F4802028606068A8B1FEF7F1
:1035700093FE06460DE0286840F48030F4E740F4FE
:1035800080202860F7E700BFFEF786FE801B6428D6
:1035900073D828688003F7D50CE0FEF77DFE064659
:1035A00005E000BFFEF778FE801B6428F0D828688D
:1035B0008003F7D42078DFF8AC8280074FF0000A50
:1035C0003ED5A748001D016811F00C0F08D0006817
:1035D000C0F3810002280BD1D9F80000400207D4C3
:1035E0002868800716D5E068012800D112E033E191
:1035F000E068B8B10120C8F80000FEF74DFE0646AD
:1036000005E000BFFEF748FE801B0228C0D82868EE
:103610008007F7D52868216920F0F80040EAC1004A
:1036200028600DE0C8F800A0FEF736FE064604E06C
:10363000FEF732FE801B02281FD828688007F7D4C7
:103640002078000722D5864F87486169703771B1AD
:1036500001210160FEF720FE064604E0FEF71CFE95
:10366000801B022809D838688007F7D50EE0C0F81B
:1036700000A0FEF711FE064605E082E0FEF70CFE14
:10368000801B02287DD838688007F7D4207840074F
:1036900068D5DFF8CCB100270BF13C0BDBF800005C
:1036A000C0000BD4DBF8001041F08051CBF80010C3
:1036B000DBF80000012700F0805000906B4E30686E
:1036C000C00510D4306840F480703060FEF7E4FD2F
:1036D000009005E0FEF7E0FD0099401A022850D85E
:1036E0003068C005F6D55E4EA0686C3601280FD054
:1036F0000528306810D020F001003060306820F0DC
:1037000004003060A068B8B1FEF7C6FD00900FE07D
:10371000306840F00100F4E740F004003060F7E763
:10372000FEF7BAFD0099411A41F28830814266D80D
:1037300030688007F4D50EE0FEF7AEFD009007E09C
:10374000FEF7AAFD0099411A41F28830814256D80D
:1037500030688007F4D42FB1DBF8001021F08051DD
:10376000CBF80010A069C8B33D49091D0968C1F331
:10377000810102294AD00228504607D0C8F86000CB
:1037800000E03CE0FEF788FD04463BE04746C8F811
:103790006000FEF781FD064605E000BFFEF77CFDF8
:1037A000801B02282BD828688001F7D4D4E90701B0
:1037B0000843A16A2E4A490802EB0141626A41EAC4
:1037C0008211084394F82C1040EA0161C9F80010F6
:1037D00001203866FEF760FD044606E03EE000BFCB
:1037E000FEF75AFD001B022809D828688001F7D58A
:1037F00034E000BFFEF750FD001B022802D9032071
:10380000BDE8F88F28688001F4D427E00128F7D0BC
:10381000D9F80000E26900F4800191421CD1226ACB
:1038200000F03F01914217D147F6C071626A014032
:10383000B1EB821F10D1A26A4FF0FF3300F4403188
:1038400003EB5202B1EB024F06D194F82C1000F0BA
:103850007060B0EB016F01D00120D1E70020CFE70D
:103860000438024000004742800E4742007000408A
:103870000000FFFF70B5040009D0606A002540B168
:1038800025616561A56294F8510040B10CE001200A
:1038900070BD6068B0F5827FF4D0E561F2E784F82E
:1038A0005050204600F04AF8022084F85100206869
:1038B000016821F040010160A088218900F4827034
:1038C00001F404410843A18901F400610843217C0B
:1038D00001F002010843217D01F001010843218B21
:1038E00001F400710843217F01F03801084394F886
:1038F000201001F080010843218D01F4005108439C
:1039000021680860A069042101EA104094F824109D
:1039100001F010010843216848602068C16921F462
:103920000061C1616565012084F85100206801686B
:1039300041F040010160002070BD000010B586B06C
:10394000044614216846FCF768FD14492068884243
:1039500021D113480021026842F40042026000684D
:1039600000F4004005900E481038026842F004024E
:103970000260006800F0040005904FF4E0500090F1
:103980000220CDE90101032003900620049069463E
:103990000448FEF75FFB06B010BD0000003C00408D
:1039A00040380240000802402DE9F84F04464068C4
:1039B0000025984616460F464FF0040BB0F5827F5F
:1039C00001D1A06888B194F85000012818D00120D6
:1039D00084F85000FEF760FC814694F851004FF0E7
:1039E000000A01280ED0022582E084F851B0134667
:1039F0000A462046CDF8008000F036F9BDE8F88F81
:103A00000220FBE7002F72D0002E70D084F851B056
:103A1000C4F854A0A763A687E687C4F830A0A4F82A
:103A200034A0A4F836A0C4F840A0C4F844A0A0680C
:103A3000B0F5004F09D12068016821F04001016014
:103A40002068016821F4804101602068016849060E
:103A500003D4016841F040010160E068D8B139E069
:103A600020688168C90709D0007BA16B0870A06B32
:103A7000401CA063E08F401EE0870CE0FEF70CFCCA
:103A8000A0EB0901414503D3B8F1FF3F03D036E075
:103A9000B8F1000F33D0E08F0028E1D11DE020689D
:103AA0008168C90709D0C068A16B0880A06B801C21
:103AB000A063E08F401EE0870CE0FEF7EDFBA0EB7B
:103AC0000901414503D3B8F1FF3F03D017E0B8F136
:103AD000000F14D0E08F0028E1D14A46414620462D
:103AE00001F0EEF908B120206065606D00B101259C
:103AF000012084F8510084F850A028467EE7032571
:103B0000F6E72DE9F84F044690F8500000271D46CF
:103B10001646894601280DD04FF0010B84F850B0AD
:103B2000FEF7BAFB804694F85100BA46012804D04B
:103B3000022793E00220BDE8F88FB9F1000F73D09F
:103B4000002E71D0032084F85100C4F854A0C4F8AA
:103B50003090A686E686C4F838A0A4F83CA0A4F865
:103B60003EA0C4F844A0C4F840A0A068B0F5004F3F
:103B700009D12068016821F04001016020680168D6
:103B800041F48041016020680168490603D401685E
:103B900041F040010160E068B0F5006F606803D05B
:103BA00030B3012E24D041E008B1012E1CD1206B8E
:103BB00021680088C86006E020688168890709D507
:103BC000216B0988C160206B801C2063E08E401E41
:103BD000E08609E0FEF760FBA0EB0800A84202D3F4
:103BE000681C01D031E07DB3E08E0028E4D120E0F4
:103BF000206B21680078087306E0206881688907D7
:103C000009D5216B09780173206B401C2063E08E7D
:103C1000401EE0860AE0FEF73FFBA0EB0800A8424A
:103C200003D3681C02D010E017E06DB1E08E0028CD
:103C3000E3D142462946204601F070F908B1202020
:103C40006065A06818B106E0FFE7032706E020687A
:103C5000C16880680090606D00B1012784F851B0A0
:103C600084F850A0384666E72DE9F84F044690F8EE
:103C7000500000270A9E1D4692468B464FF00109D0
:103C800001280ED0012084F85000FEF705FB804685
:103C900094F85100616801280CD0B1F5827F07D1FA
:103CA00002E00220BDE8F88FA16809B9042801D01C
:103CB0000227C2E0BBF1000F27D0BAF1000F24D0D9
:103CC0001DB394F85100042802D0052084F8510057
:103CD00000206065C4F838A0E587A587C4F830B037
:103CE000E586A5862064606420680168490603D4DF
:103CF000016841F040010160E068B0F5006F606864
:103D000005D0E8B3012D46D07FE0012795E008B14A
:103D1000012D39D1206B21680088C860206B801C80
:103D20002063E08E401EE0862EE0206881688907CF
:103D30000FD5E18E69B1B9F1010F0AD1216B098864
:103D4000C160206B801C2063E08E401EE0864FF037
:103D5000000920688168C9070CD0E18F51B1C068A3
:103D6000A16B0880A06B801CA063E08F401EE087E1
:103D70004FF00109FEF790FAA0EB0800B04200E016
:103D800009E001D3701C50D1E08E0028CDD1E08F26
:103D90000028CAD13FE0206B216800780873206BAF
:103DA000401C2063E08E401EE0862EE02068816883
:103DB00089070FD5E18E69B1B9F1010F0AD1216BE5
:103DC00009780173206B401C2063E08E401EE08662
:103DD0004FF0000920688168C9070CD0E18F51B10C
:103DE000C068A16B0870A06B401CA063E08F401EF0
:103DF000E0874FF00109FEF74FFAA0EB0800B04250
:103E000002D3701C01D010E07EB1E08E0028CDD12D
:103E1000E08F0028CAD142463146204601F07EF8A4
:103E200028B101272020606507E0032705E0A0688E
:103E300018B92068C16880680090012084F851009A
:103E4000002084F8500038462CE77047704710B5C2
:103E5000040003D094F83D0010B107E0012010BD2C
:103E6000002084F83C00204600F01EF8022084F870
:103E70003D00211D206801F05DFD012084F8460011
:103E800084F83E0084F83F0084F8400084F8410044
:103E900084F8420084F8430084F8440084F8450024
:103EA00084F83D00002010BD7047000090F83D10E0
:103EB000012901D001207047022180F83D100168DE
:103EC000CA6842F00102CA6000681149884214D0F1
:103ED000B0F1804F11D00F4988420ED00E49884270
:103EE0000BD00E49884208D00D49884205D00D49B3
:103EF000884202D00C49884204D1816801F0070150
:103F0000062903D0016841F00101016000207047DB
:103F1000000001400004004000080040000C004088
:103F2000000401400040014000180040704770B597
:103F30000446006801694FF00005C943890715D49C
:103F4000C168C943890711D4E91E016101202077A6
:103F5000206880698007204602D0FFF7E7FF04E071
:103F600000F098F8204600F096F82577206801695F
:103F7000C943490717D4C168C943490713D46FF02F
:103F800004010161022020772068806910F4407FDD
:103F9000204602D0FFF7CAFF04E000F07BF820467D
:103FA00000F079F8257720680169C943090716D41C
:103FB000C168C943090712D46FF0080101610420E8
:103FC00020772068C0698007204602D0FFF7AEFF47
:103FD00004E000F05FF8204600F05DF825772068E7
:103FE0000169C943C90617D4C168C943C90613D4B6
:103FF0006FF010010161082020772068C06910F47B
:10400000407F204602D0FFF791FF04E000F042F825
:10401000204600F040F8257720680169C943C907A8
:1040200008D1C168C943C90704D1891E016120466E
:1040300000F032F820680169C943090609D4C16853
:10404000C943090605D46FF0800101612046FFF7DE
:10405000FCFE20680169C943490609D4C168C94307
:10406000490605D46FF040010161204600F01EF8BA
:1040700020680169C94389060BD4C168C943890610
:1040800007D46FF0200101612046BDE87040FFF7C2
:10409000DDBE70BD7047704700680349884201D19A
:1040A000FEF78CBB7047000000100040704770B5F1
:1040B000040004D094F83D00002510B106E0012072
:1040C00070BD84F83C50204600F022F8242084F88B
:1040D0003D002068C16821F40051C160204601F014
:1040E00099FC2068016921F49041016120684169CF
:1040F00021F02A0141612068C16841F40051C1608A
:104100002564202084F83D0084F83E00002070BD26
:1041100010B586B0044614216846FCF77EF91B49A9
:10412000206888422FD11A480021026842F40032E8
:104130000260006800F400300590154810380268ED
:1041400042F008020260006800F00800059060205C
:1041500000900220CDE90101032003900720049084
:1041600069460C48FDF776FF0B480068C16841F0CE
:104170002001C16009494020C1F8000107495020D1
:10418000223181F8000406B010BD00000044004058
:1041900040380240000C0240B002002004E000E081
:1041A0002DE9F843044690F83D001F4616460D469B
:1041B00020284CD1C5B1BEB194F83C00012846D0AE
:1041C000012084F83C004FF00008C4F84080212012
:1041D00084F83D00FEF760F8A6848146E684A06876
:1041E000B0F5805F03D004E00120BDE8F8832069CA
:1041F00028B12E465FF0000584F83C800EE00026D2
:10420000FAE78021204601F08BFCA0B9AEB116F888
:10421000010B21684860E08C401EE084E08C4B4636
:104220004FF0000200970028EBD14FF040012046EC
:1042300001F076FC30B10320D7E735F8020BC0F36C
:104240000800E6E7202084F83D000020CDE70220AA
:10425000CBE700000648016841F080710160054825
:10426000016841F0010101600021416070470000D8
:10427000FCED00E0001000E0FEE701684A69D2436F
:1042800052050FD46FF480624A61002140F8301F5C
:10429000202242738173026942F0040202610173B9
:1042A00001207047002070472DE9F84F0446C06A8E
:1042B0001E4693460D4621680A6842F480620A60F1
:1042C000082807D0012805D010F5803F02D0206BC8
:1042D000112804D12068016841F4807101604FF019
:1042E00001195B46002249462046009600F0C6F8B8
:1042F0004FF4007840B120680068C00501D5C4F8CB
:1043000040800320BDE8F88F2069DFF884A0B0F575
:10431000804F0FD00620216800EAD51747F0F00043
:10432000086133465A460AF10601204600F0DAF8E1
:1043300058BB03E0E8B240F001001CE02168E8B29D
:10434000086133465A465146204600F0CBF8E0B9A2
:104350002068416981690091016841F480710160C0
:104360005B46002249462046009600F087F8002868
:10437000C1D147F0F1002168086133465A465146E1
:10438000204600F0AFF80028BCD00120BAE70000BA
:1043900002000100F8B50446C06A1E460D461746E5
:1043A000082807D0012805D010F5803F02D0206BE7
:1043B000122804D12068016841F48071016013461D
:1043C00000224FF001112046009600F057F840B14E
:1043D00020680068C00502D54FF4007020640320F7
:1043E000F8BD2069B0F5804F0ED00620216800EAA4
:1043F000D51040F0F000086133463A460B4920469C
:1044000000F070F878B902E005F0FE0000E0E8B2D4
:1044100021680861054933463A46891F204600F065
:1044200061F80028DCD00120F8BD00000800010080
:1044300070B516460D4604460DE02046FFF71DFFF9
:1044400008B1012070BD681C05D0FDF725FF801B59
:10445000A84207D835B120684069C0434007ECD472
:10446000002070BD002044F8300F20216173A0733C
:10447000216941F0200121612073E2E72DE9F04735
:104480001E4690460D460446C1F30747DDF82090CE
:1044900008E0701C06D0FDF7FFFEA0EB0900B0425B
:1044A0000FD876B12068012F18D0806925EA000066
:1044B0000004000C14D000214145EAD00020BDE8E2
:1044C000F087002044F8300F20216173A073216928
:1044D00041F02001216120730120F0E74069E5E708
:1044E0000121E9E72DE9F0479A4691460E46044638
:1044F00000254FF02008C1F3074725E020684069F8
:10450000C043400514D42068016841F40071016083
:1045100021686FF480604861256384F83D8084F8E9
:104520003E50206C40F00400206484F83C501FE0B2
:10453000B9F1FF3F08D0FDF7AFFEA0EB0A014945F6
:104540000CD8B9F1000F09D02068012F13D0806971
:1045500026EA00000004000C0BD0CFE744F8305FDF
:1045600084F80D80A573206940F020002061257338
:104570000120BDE8F0874069EAE72DE9F041002518
:1045800090460E460446202717E04069C043C00607
:104590000CD454F8301B6FF01000486144F81059E7
:1045A0006777A577206A2062257717E0FDF774FE0C
:1045B000A0EB0800B04208D83EB120684169C94369
:1045C0004906E2D40020BDE8F08144F8305F67730B
:1045D000A573206940F02000206125730120F2E7D7
:1045E00070B516460D4604460DE02046FFF745FE21
:1045F00008B1012070BD681C05D0FDF74DFE801B81
:10460000A84207D835B120684069C0430006ECD401
:10461000002070BD002044F8300F20216173A0738A
:10462000216941F0200121612073E2E738B5084C8F
:10463000002500952068002803D0A18811B1491EEB
:10464000A18038BD694621F013FA256038BD00000D
:10465000F8000020F0B500230A24302537261F4635
:1046600011E000BFB4EB107F02D905EB107C01E034
:1046700006EB107C01F813C001EB430C00015B1C3E
:104680008CF80170DBB29342ECD3F0BD10B5044658
:104690000C490BF0D3FA0B4904F11000091D0BF083
:1046A000CDFA084904F1200008310BF0C7FA054B98
:1046B00004F1300008331A1FBDE81040111F10F03C
:1046C00093BA0000280100202DE9F0410025056083
:1046D000456085600446C560984617460E46084604
:1046E000FBF7C2FE024631462046FBF76FFE25610E
:1046F0006561A5613846E561FBF7B6FE024604F147
:10470000100039460646FBF761FE25626562A56228
:104710004046E562FBF7A8FE024604F12000414650
:104720000546FBF753FE0C4920460BF087FA0A4971
:104730003046091D0BF082FA0749284608310BF074
:104740007DFA04F13000BDE8F041034B08331A1F35
:10475000111F10F049BA00002801002010B50446CE
:104760000B490CA00BF06AFA09490EA0091D0BF0C9
:1047700065FA07490FA008310BF060FA044B04F109
:10478000300008331A1FBDE81040111F10F02CBA7A
:10479000280100203139322E3136382E302E323574
:1047A000340000003235352E3235352E3235352E77
:1047B000300000003139322E3136382E302E3100A3
:1047C00010B504490448FCF79DFD0249491E0870D4
:1047D00010BD000001010020240A00101CB54FF498
:1047E000FA6021F067FA00F077F9012021F0A8FAC9
:1047F0000D4C03220021A060012021F0B3FAE060FB
:1048000003220021012021F0ADFA206103F088FB92
:1048100000200090034601904FF4007203A1064867
:1048200021F038FD1CBD00000000002064656661B9
:10483000756C745461736B00E15302082DE9F0410B
:1048400086B014216846FBF7E8FD4A480024016859
:1048500041F080010160016801F08001059101686B
:1048600041F004010160016801F004010591016853
:1048700041F001010160016801F001010591016849
:1048800041F010010160016801F01001059101681B
:1048900041F002010160016801F002010591016827
:1048A00041F0080101600068334F00F008000590F6
:1048B000002241213846FDF7EAFCDFF8C0800122E2
:1048C00011464046FDF7E3FC002202214046FDF779
:1048D000DEFC412000900125CDE9015469463846AF
:1048E0000394FDF7B7FB382002268DE87100694676
:1048F0003846FDF7AFFB4FF478508DE871006946FC
:104900004046FDF7A7FB280300901D48CDE90104B0
:1049100069461C48FDF79EFBA8028DE831006946F8
:104920003846FDF797FB80200090CDE90154694699
:1049300040460394FDF78EFB68020090CDE90164C8
:104940000394694610480494FDF784FB0320CDE9E5
:104950000005CDE9025669464046FDF77BFB002283
:1049600005212820FDF7B0FF2820FDF79FFF06B0A6
:10497000BDE8F0813038024000000240000C0240E7
:104980000000211000100240000802400D4810B540
:104990000B4901600C49416000214FF48042816065
:1049A000C0E9031241618161C1610162FDF77AFCD6
:1049B000002803D0BDE81040FCF7A2BC10BD0000E9
:1049C000005400405C020020801A06003EB50446F8
:1049D0001E490BF033F91D4904F11000091D0BF0BD
:1049E0002DF91A4904F1200008310BF027F9184A73
:1049F000184900208DE80700144B04F130000833FB
:104A00001A1F111F0FF006FF94F8590040F004011F
:104A1000062084F858001048027884F85220427822
:104A200084F85320827884F85420C27884F8552082
:104A3000027984F85620407984F8570040F2DC501F
:104A400024F8500F41F00A0060723EBD280100209A
:104A500075220408A9CE0208200100200F4810B5D5
:104A60000D4901604FF48271416000218160C16095
:104A70004FF400720161C0E90512C1610162416237
:104A800081620A21C162FEF7F5FE002803D0BDE86D
:104A90001040FCF735BC10BD003C00404C1300102A
:104AA0000C4810B50A4901604FF4E1314160002122
:104AB00081600C22C160C0E904128161C161FFF70D
:104AC000F6FA002803D0BDE81040FCF719BC10BD71
:104AD00000440040B002002010B500220F491048E9
:104AE00001F031FC08B1FCF70BFC0E490C4801F059
:104AF0001DFE08B1FCF704FC0B49094801F021FA3E
:104B000008B1FCF7FDFB064801F08AFE002803D03F
:104B1000BDE81040FCF7F4BB10BD0000380A0010DF
:104B2000D82A00101C02002008010020FEE7FEE742
:104B30000148FEF749B80000243400202DE9F04177
:104B400003680D4604461E6C03EB4511D1F8080BB3
:104B5000D4F810E04FF400474FF0200C04F57172C8
:104B6000BEF1010F09D0DFF898E0764539D1020493
:104B700032D500BFC1F8087B3FE0224B5FEA007EE0
:104B800004D59E4239D90004F4D436E05FEA806E41
:104B900002D5C1F808CB30E010F0280F2DD19E428D
:104BA00001D90004E6D4C5EBC50004EB8000D1F8C0
:104BB000101BD0F80432C1F31201591AC0F81412B4
:104BC000D0F808121944C0F8081295B9D4F81002A8
:104BD00078B9012120680AE080060AD5C1F808CB1F
:104BE00007E035B9D4F8100218B90021184602F0D0
:104BF000E3F9E9B22046FDF7CDFE0020BDE8F081E3
:104C00000A31544F0A30544F2DE9F84F0E46C1EB8C
:104C1000C60100EB810481460568D4E914103C34D8
:104C2000884202D90120BDE8F88F081AA1688142A4
:104C300000D20846C01C870805EB46181BE000BFE1
:104C4000A0EB010AA068504500D282460AF1030099
:104C5000870899F8100000901FFA8AF3F2B22846EC
:104C6000E16802F031FCE16801EB0A00E060A16953
:104C700001EB0A00A061D8F8180980B2B84205D348
:104C8000D4E90501814201D20028D9D1D4E9050136
:104C9000884208D806F00F0101208840D5F8341862
:104CA0008143C5F834180020BDE70000026853684E
:104CB000074A126902EBC30292F87431012B01D04A
:104CC000062B04D1D2F878010078086004207047E0
:104CD0000000001002685368074A126902EBC30221
:104CE00092F89C31012B01D0062B04D1D2F8A001FF
:104CF00000780860042070470000001002685368C4
:104D00000F4A126902EBC30292F82430012B14D02F
:104D1000042B09D0032B0CD0062B0ED0052B07D16A
:104D2000906A90F9000001E0906A00880860042011
:104D30007047906AB0F90000F8E7906A0078F5E7EC
:104D40000000001002685368114A126902EBC302A6
:104D500092F89430012B17D0042B0AD0032B0ED0DD
:104D6000062B11D0052B09D1D2F8980090F900003C
:104D700002E0D2F898000088086004207047D2F85A
:104D80009800B0F90000F7E7D2F898000078F3E750
:104D90000000001002685368114A126902EBC30256
:104DA00092F80431012B17D0042B0AD0032B0ED01C
:104DB000062B11D0052B09D1D2F8080190F900007B
:104DC00002E0D2F808010088086004207047D2F899
:104DD0000801B0F90000F7E7D2F808010078F3E71E
:104DE0000000001070B50D460168134C06464A6875
:104DF000216901EBC20313F8043C012B15D0022BEF
:104E000002D0062B11D015E051F83200FBF72CFB35
:104E1000024630682169406851F830102846FBF797
:104E2000D5FA2846FBF720FB04E051F83200007861
:104E30002860042000B270BD000000100348016823
:104E4000C907FCD00148001D0068704704080650DF
:104E5000074808B5016841F040010160006800F0B2
:104E6000400000900348016841F00401016008BD62
:104E7000343802400008065038B50F49D7200F4C8F
:104E80000870002201212046FDF701FA01210A489D
:104E900016F068FA0121684616F05AFA0122114606
:104EA0002046FDF7F4F90020401CC0B20528FBD3D2
:104EB0009DF8000038BD0000EC080010000C024016
:104EC000F8B5044640684FF48273984221D1A06837
:104ED0004FF48065B0F5004F01D0A8420AD1206898
:104EE000066826F0400606606068984211D1A06806
:104EF000A8420ED000920B4600228021204600F0EE
:104F000039F8002804D0606D40F02000606503206F
:104F1000F8BD00920B4600220121EFE738B50446A8
:104F20001248134B0068B0FBF3F04FF47A73584308
:104F300000906068B0F5827F0DD10B460092002290
:104F40008021204600F016F870B1606D40F020001E
:104F50006065032038BD009830B1401E0090206885
:104F60008068C0430006F6D5002038BD940A0010C2
:104F700000366E012DE9F8431E46914688460446E8
:104F8000089DFDF789F9401B351AFDF785F907469D
:104F900025480068C0F3CB30684338E0701C37D038
:104FA000FDF77AF9C01BA84203D215B1009860B38F
:104FB0002CE02068416821F0E00141606068B0F5B4
:104FC000827F0BD1A068B0F5004F02D0B0F5806FA2
:104FD00004D12068016821F040010160A06AB0F5A9
:104FE000005F09D12068016821F400510160206848
:104FF000016841F400510160012084F85100002053
:1050000084F850000320BDE8F8830025401E00907E
:105010002068816838EA010004D000214945BDD1EB
:105020000020F0E70121F9E7940A001001784078A8
:1050300041EA00207047000008B50C4A12230029FD
:10504000137002DD41F0800300E0CB435370017028
:105050004FF4FA6000900223044AD0210448FDF77F
:10506000D5FABDE80840FCF729B900006C00002023
:105070005C0200202DE9F843064680886421A0F5F3
:10508000FA6090FBF1F0394DC7B201202870F07939
:105090000A24B0FBF4F104FB1101B0FBF4F041EA87
:1050A000001000F07F006870307A4FF4FA68B0FBAF
:1050B000F4F104FB1101B0FBF4F041EA001000F040
:1050C0007F00A870707A0423B0FBF4F104FB110197
:1050D000B0FBF4F041EA001067F39F10E8702A4635
:1050E000D0212348CDF80080FDF790FAFCF7E6F8D0
:1050F000002838D005202870B078B0FBF4F104FB0C
:105100001101B0FBF4F041EA001000F03F006870BC
:10511000F078B0FBF4F104FB1101B0FBF4F041EACC
:10512000001000F01F00A870B1886FF0180017FB86
:1051300000F2C8F1000000EB8200084490FBF4F19B
:1051400004FB110190FBF4F041EA0010E870042325
:105150002A46D0210648CDF80080FDF757FABDE871
:10516000F843FCF7ABB8BDE8F88300006C00002002
:105170005C020020F8B50BF0F1FB1F4D4FF4FA6410
:1051800070B9012028700020687002232A46D021BF
:105190001A480094FDF73AFAFCF790F800282AD054
:1051A00008262E700123144AD02114480094FDF7DC
:1051B0002DFAFCF783F800281DD001230E4AD021D8
:1051C0000E480094FDF732F9FCF778F8002812D069
:1051D000287841060ED440F0400068702E700223FB
:1051E000054AD02105480094FDF710FAFCF766F84F
:1051F000002800D00120F8BD6C0000205C020020D7
:1052000070B50546BAB00020544C349035903690B5
:1052100037908DF8E00006466580CC22504901A801
:10522000FBF7D4F804F13C0000904EA3002250A1FB
:10523000099551A021F008FB28B152A00168E16353
:105240008088A4F8400038A8009050A3002248A10C
:1052500049A021F0F9FA18B938A8FBF785F9C6B2C8
:105260003E484DA34C300090002241A142A021F0C5
:10527000EBFA28B143A00168E1648088A4F85000EB
:1052800034A8009048A3002239A13BA021F0DCFA09
:1052900028B149A0016834918088ADF8D40000207D
:1052A00015F0E2FB012015F0E6FB2C483C3014F031
:1052B0002FFF2A49A289891D881F13F07FFC2749E7
:1052C000A2890831C81F13F08DFC2449091D01F182
:1052D000180013F07FFC01A814F0C2FFA5F51C51C3
:1052E00011394FF0080002D0012908D101E036A29F
:1052F00000E038A2D2E90012C4E90D12608117491A
:10530000A2890A3101F12A0013F078FCA5F51C509E
:10531000113804D0A5F51C50123804D008E00F480D
:105320000221243002E00D4802212C3014F0A2FFAB
:105330000A484C3014F040FF012E0BD139A934A893
:105340000AF07CFC39A9002015F092F90121002017
:1053500015F086F913F0FEFB3AB070BD00000010A6
:10536000A86A0408636F6D6D756E6974790000003A
:10537000736E6D7000000000636F6E6669672E7853
:105380006D6C00007075626C69630000747261700E
:105390002D656E61626C6500747261702D636F6D56
:1053A0006D756E6974790000747261702D686F7329
:1053B000746E616D650000003139322E3136382E41
:1053C000302E323534000000555053203132303009
:1053D000000000004D4330342D504C4300000000CD
:1053E0000EB520F07BFCDFF890A20122114650465A
:1053F000FCF74DFFA148002502950068A04C6060B5
:105400009E48001D00689FA12060D1E90001CDE900
:1054100000019E4A2946A4F1240900BF01EB020CB9
:10542000DCF80009C7B2C0F307438DF80570C0F37C
:1054300007268DF803304FEA10688DF804608DF868
:105440000280DCF8040900F0FF0CC0F307208DF89F
:1054500001C08DF80000FF2818D0BCF1FF0F15D057
:10546000B8F1FF0F12D0FF2B10D0FF2E0ED0FF2F60
:105470000CD0009BC9F81C30BDF80430C1F1FF000E
:10548000A9F82030062801D3891DC7E74FF44870DA
:105490000FF0A5FC20680090794E99F803002C3697
:1054A000636856F820204C4679A1012002F002FDE5
:1054B000A6F134000178FF290ED14178FF290BD1E4
:1054C0008178FF2908D1C178FF2905D10179FF2909
:1054D00002D14079FF282ED0694A75A1083A0120EF
:1054E00002F0E8FC03F00AFEC8200FF078FCFFF79A
:1054F000B5FA012202217348FCF7C9FE02A8FBF7A6
:10550000CFFF9DF80A0000909DF809309DF8082013
:105510006DA1012002F0CEFCFFF752F901227A4979
:105520007A4808F02DFA074620F0A6F80D2F07D08C
:10553000002F55D01EE076A1012002F0BBFCD1E780
:1055400078A1012002F0B6FCFFF796FCC00701D15C
:10555000FBF7CAFF4FF400700090764B0022072142
:10556000694807F067FF0746024673A1012002F071
:10557000A1FC7FB33A4676A1012002F09BFC00BF5C
:1055800020F088F8E07856F8201077A002F008FDA7
:105590009DF80A309DF809209DF8081073A002F0CC
:1055A000FFFCDAF810005646C043C0F3C2004208C0
:1055B000042A29D24348103000680021C043C0F3B8
:1055C00044232F4802EB4207083000EB870210F813
:1055D000270017E0FFE701224B494C4808F0D0F9BB
:1055E00072A1012002F066FCCAE700BF02EBC1070E
:1055F0003F799F4204D102EBC100001D606003E0CF
:10560000491CC9B28842F1D8606828B342686CA1CD
:10561000012002F04FFC6068416870A002F0C0FCFD
:10562000FEF718FEFFF714FC009500234FF400620C
:1056300070A17248019520F02DFE1CF095FF00220C
:1056400001213046FCF723FE4FF4FA7420F046FBAC
:1056500020460FF0C4FBF9E769A1012002F02AFC03
:105660006CA002F09DFC41F2883400BF20F036FBB4
:1056700020460FF0B4FBF9E700000240F8FF0F08E6
:1056800024000020FFFFFFFFFFFF00000070FF1F4E
:105690000D0A25730D0A532D706F72743A204669F6
:1056A000726D77617265207625642E25642C20004A
:1056B00053657269616C206E756D6265723A202562
:1056C000730D0A00000C0240466C6173682064652B
:1056D000766963653A204D616E75666163747572B3
:1056E00065722049443A203078253032582C2044C5
:1056F00065766963652049443A2030782530325810
:10570000253032580D0A0000010100209C280010AD
:10571000532D706F727420534E3A206E2F610D0A14
:10572000000000004E4F2046696C65737973746504
:105730006D0D0A00F00E0010665F6D6B66732072CF
:105740006573756C74202D2025640D0A000000001F
:10575000665F6D6F756E7420726573756C74202D45
:105760002025640D0A00000025730A00466C617351
:1057700068206465766963653A204D616E7566617F
:105780006374757265722049443A2030782530324E
:10579000582C204465766963652049443A20307866
:1057A00025303258253032580A00000046696C65B1
:1057B00073797374656D3A204F4B0D0A0000000039
:1057C000532D506F727420534E4D5020646576698E
:1057D00063653A2025730D0A00000000532D506FB9
:1057E000727420534E4D50206465766963653A208B
:1057F00025730A004574685461736B00D13C04083A
:10580000556E636B6E6F776E206465766963650DA8
:105810000A000000556E636B6E6F776E20646576CC
:105820006963650A0000000010B5502080F31188FC
:10583000BFF34F8FBFF36F8F20F078FD18B104498D
:105840004FF080500860002080F3118810BD0000E8
:1058500004ED00E030B593B030216846FAF7DDFD85
:1058600014210CA8FAF7D9FD20480025016841F061
:1058700080510160006800F0805011901C48016860
:1058800041F4404101600068022400F4404011905E
:1058900001200090000401908001CDE9064019200C
:1058A00008904FF4A870CDE9090407200B906846D2
:1058B000FDF72AFE08B172B6FEE70CA90F2081E8B9
:1058C00031004FF4A0500F904FF4805010900521FC
:1058D0000CA8FDF7C1FC08B172B6FEE700224FF03C
:1058E00000410120FDF7CAFD13B030BD4038024031
:1058F000007000400448016841F4700101600249F1
:10590000024880390860704788ED00E00000020816
:105910000148FEF70CBB0000A413001010B5FEF701
:1059200085FE0348016821F00101016010BD0000FF
:1059300010140040F0B50268254C264D264E274F26
:10594000274B4FF0804CA04209D0604507D0A842B9
:1059500005D0B04203D0B84201D0984204D122F021
:10596000700E4A6842EA0E02A0421BD0604519D070
:10597000A84217D0B04215D0B84213D0984211D0E7
:10598000184DA8420ED0184DA8420BD0174DA84272
:1059900008D0174DA84205D0164DA84202D0164D8A
:1059A000A84203D122F44075CA682A434D6922F007
:1059B00080022A4302608A68C2620A688262A04248
:1059C00001D0984201D10969016301214161F0BD13
:1059D000000001400004004000080040000C0040AE
:1059E00000040140004001400044014000480140E3
:1059F00000180040001C00400020004008B50020B6
:105A0000009003486946006920F0B2FA08BD000022
:105A10000000002070B5044600680169E26821F4C6
:105A20004051114301612169A068E269084361693D
:105A3000114308432168CA6849F20C639A43024340
:105A4000CA6020684169A26921F440711143416133
:105A500031492068884202D03049884202D1FDF79E
:105A6000CBFC01E0FDF7B8FCE269002319216425B5
:105A70003226B2F5004F626828D0A0FB0101930FD7
:105A80009200FAF711FC0146B0FBF5F06FF0180236
:105A9000504301EB800006EB0010B0FBF5F000F086
:105AA000F002B1FBF5F002EB0012B1FBF5F06FF084
:105AB0001803584301EB800006EB0010B0FBF5F033
:105AC00000F00F0021681044886070BDA0FB010148
:105AD00092185B41FAF7E8FB0146B0FBF5F00201D2
:105AE000B1FBF5F06FF01803584301EB800006EBB3
:105AF000C000B0FBF5F000F0F80002EB4002B1FB93
:105B0000F5F0584301EB800006EBC000B0FBF5F068
:105B100000F00700D6E7000000100140001401402B
:105B20002DE9F041984617460E460446069D1DE0B5
:105B3000681C1BD02DB1FCF7AFFBA0EB0800A842FE
:105B400014D92068C16821F4D071C160206841690E
:105B500021F001014161202084F83D0084F83E00DD
:105B6000002084F83C000320BDE8F0812068006834
:105B700036EA000004D00020B842D9D00020F3E774
:105B80000120F9E700684268054800EBC20090F880
:105B9000A020012A02D1D0F8A40008600420704798
:105BA0005C00001000684268064800EBC20090F8F4
:105BB000F820012A01D0062A02D1D0F8FC000860A2
:105BC000042070475C00001000684268054800EB44
:105BD000C20090F81021032A02D1D0F81401086005
:105BE000042070475C00001000684268054800EB24
:105BF000C200027C032A01D0012A01D14069086059
:105C0000042070475C00001000684268054800EB03
:105C1000C20090F83821012A02D1D0F83C01086076
:105C2000042070475C00001000684268054800EBE3
:105C3000C20090F84021012A02D1D0F84401086046
:105C4000042070475C00001000684268054800EBC3
:105C5000C20090F84821012A02D1D0F84C01086016
:105C6000042070475C00001000684268054800EBA3
:105C7000C20090F85021012A02D1D0F854010860E6
:105C8000042070475C00001070B50C460168124D8E
:105C90000646496805EBC10111F8082C012A02D01B
:105CA000022A05D015E051F8040C2060042010E011
:105CB00051F8040CFAF7D8FB02463068406805EB4F
:105CC000C00050F8041C2046FAF780FB2046FAF783
:105CD000CBFB00B270BD00005C00001000684268A1
:105CE000054800EBC20090F85020012A01D1406D18
:105CF00008600420704700005C00001000684268E3
:105D0000054800EBC20090F87020012A01D1406FD5
:105D100008600420704700005C000010074800681D
:105D20000168890608D5064909680978102903D150
:105D30004068C0B210F07CBB70470000B002002089
:105D4000040000202DE9F0410C46D0F8C422D0F820
:105D5000BC12F9B104EB840300EB83050026AB69A8
:105D60004BB1C4EBC40702EB8702526CB3FBF2F7F2
:105D700002FB173282B1C1F81462D0F8C002036985
:105D80002BB1D1F80802224601F504719847002092
:105D9000BDE8F0810320FBE700231A462146AE61EF
:105DA00000F0A5FCF3E770B5D0F8BC4205466CB135
:105DB00000F086FBC4F80C02D5F8C012D4F8040237
:105DC000CA6804F503719047002070BD032070BDC0
:105DD00070B50446812100F0D2FA00252587012103
:105DE000204600F0CCFAA4F878518221204600F039
:105DF000C6FAA4F84C50A4F84E50D4F8BC0248B1EE
:105E0000D4F8C00204F52F7440688047206800F081
:105E10005CFE2560002070BD10B5D0F8BC4284B196
:105E2000D0F8C01259B194F80002FF2807D08B684F
:105E300094F8012221469847FF2084F800020020B0
:105E400010BD032010BD00000A21018000487047EA
:105E50008C0B00104321018000487047DC0B0010C0
:105E60004321018000487047980B001043210180B6
:105E700000487047200C00102DE9F04704464FF40D
:105E8000077000F023FE05004FF0000735D0C4F87E
:105E9000BC52207C4FF010084FF40079012680B3EB
:105EA000402302228121204600F06EFB26874023FA
:105EB00002220121204600F067FBA4F87861A4F8D3
:105EC0004E80082303228221204600F05DFBA4F8C7
:105ED0004C60D4F8C00200688047C5F81472C5F859
:105EE0001872207CD5F80422A8B140230121204655
:105EF00000F056FB0020BDE8F0870220C4F8BC7219
:105F0000F9E7FFE74B4602228121204600F03CFBE7
:105F100026874B46CCE74B46E8E710B5D0F8BC12D5
:105F200051B1027C002AD1F8042207D0402301217C
:105F300000F036FB002010BD032010BD4FF40073AD
:105F4000F5E719B1C0F8C012002070470320704770
:105F5000D0F8BC0218B1C0F804120020704703202A
:105F60007047D0F8BC0228B1C0F81022C0F808125F
:105F700000207047032070472DE9FC410646D0F809
:105F8000BC7200200C468DF80000ADF804000546F8
:105F900037B1207810F0600128D0202944D102E0E8
:105FA0000320BDE8FC81E288C2B1000660780AD512
:105FB000D6F8C0128B6839469847E288072A00D97C
:105FC0000722394628E087F80002A07987F8010205
:105FD000E2883946304600F06CF82AE0D6F8C01264
:105FE000607800228B682146984722E0607830B1C3
:105FF00001281ED00A2809D00B2815D110E096F8E8
:106000009C02032810D1022201A905E096F89C0207
:10601000032809D101226946304600F064F808E0FF
:1060200096F89C02032804D02146304600F036F84A
:1060300003252846B5E710B5D0F8BC12012219B1E6
:10604000D1F8143213B10FE0032010BD0122C1F8C2
:106050001422D1F81022C262D1F81032D1F80822ED
:10606000812100F044FB0022104610BD10B5D0F88D
:10607000B8220AB152689047002010BD134610B5EF
:106080000A46002100F08CFA002010BD134610B51E
:106090000A46002100F02BFB002010BD10B504467D
:1060A000802100F009FB2046BDE81040002100F0EF
:1060B00003BB10B50323C0F89432C0F8582113462F
:1060C000C0F85C210A46002100F06AFA002010BDE9
:1060D00010B50521C0F8941200231A46194600F0A5
:1060E0005FFA002010BD10B50223C0F8943282611F
:1060F0001346C2610A46002100F0F9FA002010BDE3
:1061000010B50421C0F8941200231A46194600F075
:10611000EEFA002010BD000010B50A46024903A0A7
:1061200000F0E1F8004810BDA82D001043444320C2
:10613000436F6E6669670000122008800048704750
:10614000580A001010B50A46024903A000F0CBF827
:10615000004810BDA82D001043444320496E7465CB
:106160007266616365000000042008800048704783
:10617000540A001010B50A46024903A000F0B3F813
:10618000004810BDA82D001053544D6963726F650F
:106190006C656374726F6E696373000010B50A46B4
:1061A000024903A000F09FF8004810BDA82D001080
:1061B00053544D3332205669727475616C20436FAD
:1061C0006D506F727400000010B51A2008800A48E4
:1061D0000168001D0468001D0068081809D0082225
:1061E0000649FEF737FA0549042210312046FEF72A
:1061F00031FA0248801E10BD107AFF1F6E0A00108F
:10620000F8B504460020ADF8000048880D46010AA4
:1062100008295FD2DFE801F05E0409175E5E3C45A5
:10622000D4F8B412207C0A6819E0207C02260028E9
:10623000D4F8B80205D0C16A68468847014646705E
:1062400039E0816AF8E7C0B2062843D2DFE800F0FF
:10625000030A1014181CD4F8B402426805E0694619
:1062600090471CE0D4F8B402826892B3207CF6E731
:10627000D4F8B402C268F8E7D4F8B4020269F4E7CB
:10628000D4F8B4024269F0E7D4F8B4028269ECE7CA
:10629000207CF0B9D4F8B802416B684688470146C3
:1062A00009E0207CA8B9D4F8B802016B6846884799
:1062B000014607204870EA888AB1BDF8000040B165
:1062C000824200D90246ADF800202046FFF70BFFBE
:1062D000F8BDFFE729462046FFF7E0FEF8E7204635
:1062E000FFF70EFFF4E770B5002300281ED000254D
:1062F000044602E06D1CEDB2641C2678002EF9D134
:10630000022404EB450414801278CA545B1C032257
:10631000CA5400245B1C06E0CA545B1CDAB28C54DD
:10632000521CD3B2401C0278002AF5D170BD010086
:106330004FF0000004D0012901D0022901D0032030
:1063400070470120704778B10023C0F8B832C0F818
:10635000C032C0F8CC3209B1C0F8B412012180F8C3
:106360009C12027000F0B0B80320704710B5D0F84E
:10637000C402FCF743FBBDE81040FFF7D8BF10B5DF
:10638000D0F8C402FCF714FBBDE81040FFF7CFBF04
:1063900070B51646044621B194F89C02032841D0FA
:1063A00048E0D4F8941204F114000025022932D1F7
:1063B000D0E902318B4206D95A1A82603146204612
:1063C000FFF764FE0FE0994214D14068884211D370
:1063D000D4F8981288420DD2002211462046FFF7C9
:1063E00055FEC4F8985200231A461946204600F07C
:1063F000D7F810E094F89C02032805D1D4F8B8022D
:10640000C16809B1204688478021204600F054F930
:106410002046FFF75DFE94F8A00201280AD184F817
:10642000A05207E0D4F8B80242691AB1204690475A
:10643000002800D1002070BD10B51346044621B1DC
:1064400094F89C02032823D02AE0D4F8941204F58F
:10645000AA70032924D1D0E9021291420AD98A1ADA
:106460008260C068824200D3024619462046FFF788
:1064700005FE15E094F89C02032805D1D4F8B80273
:10648000016909B1204688472046FFF739FE07E039
:10649000D4F8B80282691AB120469047002800D18A
:1064A000002010BD0020704710B5012180F89C121B
:1064B000D0F8B82212B1526801799047002010BD7F
:1064C000D0F8C402FCF7C8BA10B5017839BB154939
:1064D0000222C1F80404C0F8C4124FF0A0400860C2
:1064E000042048600020C1E90320C1E906200862B9
:1064F0004862C86208630846FCF788FD08B1FAF7ED
:10650000FFFE80210748FCF712FA402200210548CF
:10651000FCF711FA802201210248FCF70CFA002056
:1065200010BD0000243400200A0601F07F01D0F8DD
:10653000C402C1EBC10100EB810002D590F83E001E
:10654000704790F8FE01704710B5D0F8B82222B11C
:1065500090F89C32032B02D004E0032010BD126A95
:1065600002B19047002010BD10B5D0F8B82222B17A
:1065700090F89C32032B02D004E0032010BD526A35
:1065800002B19047002010BD10B51C461346D0F84C
:10659000C4022246FCF769FABDE81040FFF7C7BE07
:1065A00010B5D0F8C402FCF790FABDE81040FFF730
:1065B000BEBE70B50125044680F89C520020C4F888
:1065C00094026060C4F8A402D4F8B802E0B1D4F830
:1065D000BC1221B1426812B100212046904700222E
:1065E000402311462046FFF7CFFF4026A4F8645110
:1065F0003346002280212046C4F86061FFF7C4FFC3
:10660000A5840020266270BD032070BD90F89C1206
:10661000042903D190F89D1280F89C120020704745
:1066200010B5D0F8B81221B190F89C22032A02D0FC
:1066300004E0032010BDC96901B18847002010BDE6
:1066400001740020704710B5D0F8C402FCF7B0FD0B
:10665000BDE81040FFF76BBE70B5044600F2AA20FB
:10666000054600F04DF80120C4F89402B4F8B002D9
:10667000C4F8980294F8AA0210F01F010AD0012968
:106680000ED0022912D000F080012046BDE87040F3
:1066900000F012B829462046BDE8704000F0C2B8AC
:1066A00029462046BDE8704000F0E6B9294620465C
:1066B000BDE8704000F040B910B5D0F8C402FCF756
:1066C00028FABDE81040FFF732BE10B5D0F8C4027A
:1066D000FCF789FDBDE81040FFF729BE90F89C1239
:1066E00080F89D12042180F89C120020704710B59C
:1066F000D0F8C402FCF747FABDE81040FFF717BE18
:1067000070B5054611F8010B2870087868704C1CAC
:106710002046FEF78BFC6880A41C2046FEF786FC12
:10672000A880A01CFEF782FCE88070BD38B5044646
:106730000020ADF8000049B1C4F8B812C96A19B117
:1067400068468847C4F8CC02002038BD032038BD15
:1067500002460320D2F8B832002B02D01B68104644
:10676000184770472DE9F0410F462C4E89780025D7
:1067700004463170012906D939462046FFF78EFCC0
:106780000320BDE8F08194F89C0202280CD0032875
:106790001DD039462046FFF781FC31782046FFF7AF
:1067A00065FC03252846ECE799B320466160FFF7B6
:1067B000CFFF050004D039462046FFF76FFCF1E714
:1067C0002046FFF79DFC032084F89C02EAE74FF087
:1067D0000208C1B1606888421BD0C1B22046FFF7F1
:1067E00045FC317820466160FFF7B2FF050010D00C
:1067F00039462046FFF752FC21792046FFF736FC48
:1068000084F89C82CEE784F89C8220466160FFF782
:106810002DFC2046FFF774FCC4E70000180200209E
:10682000FFF753BF2DE9F0410A78002512F060020E
:1068300008D0202A01D0402A71D1D0F8B82292681D
:10684000904731E04B78002201260A2B67D2DFE81F
:1068500003F0415E6658660805662D29FFF7D0FCF7
:106860005FE004468888D8B9C888C8B948888028B5
:1068700016D200F07F0794F89C02032810D084F809
:106880009E7239462046FFF7DEFE2046FFF738FCB1
:106890001FB1022084F89C0243E084F89C6240E02F
:1068A00020463CE0FFF75EFF05463AE0CB88012B2F
:1068B00035D190F89C32012B04D0022B02D0032B4F
:1068C0002DD104E08260012200F1080116E00122CE
:1068D000011D13E090F89C22012A03D0022A01D066
:1068E000032A1CD1CA88022A19D1C660D0F8A41282
:1068F00009B10321C160022200F10C01FFF7F3FB93
:106900000FE0498801290CD1C0F8A46211E090F889
:106910009C32012B08D0022B06D0032B04D0FFF7AA
:10692000BDFB2846BDE8F08149880129F9D1C0F8AE
:10693000A422FFF7E5FBF4E72DE9F0410D460446FC
:1069400028780026097910F060000BD0202801D0AB
:1069500040286DD1D4F8B802294682682046904775
:10696000064686E06878A8B3012822D003287CD1A7
:1069700094F89C02022802D0032876D10BE000296B
:1069800073D0802971D02046FFF796FE80212046E3
:10699000FFF792FE6DE0688838B931B1802904D0E4
:1069A000E88810B92046FFF787FE2046FFF7A8FBCE
:1069B0005FE094F89C020228E1D0032855D1688852
:1069C000A8BB480602D02046FFF7D0FC2046FFF7C0
:1069D00097FBBFE7FFE794F89C020027022802D04C
:1069E000032842D111E009B180293ED1080601F007
:1069F0007F0000EB800004EB800101D5143101E041
:106A000001F5AA7102220F602BE0080601F00F00C9
:106A100000EB800004EB80000BD5808C40B101F0CE
:106A20007F0000EB800004EB800514350CE020E0D3
:106A30001BE0B0F86401C0B101F07F0000EB800002
:106A400004EB800505F5AA7541B1802906D02046E2
:106A5000FFF76AFD10B10120286000E02F600222DC
:106A600029462046FFF73FFB03E029462046FFF773
:106A700015FB3046BDE8F08170B506460878002465
:106A80000D4610F0600003D0202801D0402817D117
:106A900096F89C02012803D0022801D003280FD1C8
:106AA000287901280CD8D6F8B80282683046904779
:106AB0000446E888204306D13046FFF721FB02E078
:106AC0003046FFF7EBFA204670BD7047004870472C
:106AD0000432002070B50A78012302F00F054E78C9
:106AE000AB401B4CD0F81C58012E17D045EA03438D
:106AF000C0F81C3800EB4210D0F8002B12040BD465
:106B0000D0F8002B0B89C978C3F30A031A4344EA6F
:106B100081410A43C0F8002B002070BD9BB21D4389
:106B2000C0F81C5800EB4210D0F800391B04F3D415
:106B3000D0F800390D89C978C5F30A0589042B43BB
:106B400041EA82510B432343C0F80039E4E70000D7
:106B500000800010D0F800196FF30A01C0F8001986
:106B6000D0F8041841F48071C0F804180020704770
:106B700070B5044606990A9E049D0D98012916D009
:106B8000E06840F04000E060204600F02BF8A16B88
:106B90001EB321F48031A163012D07D1A16841F01A
:106BA0000601A160A16841F02001A16070BDA16B48
:106BB00021F48031A163E168094A1140E160E16894
:106BC00021F44011E160012803D1E06840F4801015
:106BD000E060204600F006F8DEE741F48031DAE7B5
:106BE000BFFFBDFF01220C4902E0521C8A420BD8B4
:106BF0000369002BF9DA026942F001020261012205
:106C000004E0521C8A4201D9032070470369DB0764
:106C1000F7D1002070470000400D030030B54C78DC
:106C20000A78012300EB4212012C2CD0D2F8004B41
:106C3000002C0BDAD2F8004B44F00064C2F8004B91
:106C4000D2F8004B44F08044C2F8004BD0F83C58D6
:106C50000C7804F00F0403FA04F425EA0444C0F8A5
:106C60003C48D0F81C48097801F00F018B4024EA19
:106C70000341C0F81C18D2F8000B19490840C2F8AB
:106C8000000B002030BDD2F80049002C0BDAD2F8FE
:106C9000004944F00064C2F80049D2F8004944F0C9
:106CA0008044C2F80049D0F83C480D7805F00F0543
:106CB00003FA05F5ADB2AC43C0F83C48D0F81C4827
:106CC000097801F00F018B4099B28C43C0F81C4841
:106CD000D2F8000903490840C2F80009D1E70000D2
:106CE0000078F3EF007833ECD0F8001E21F00301B8
:106CF000C0F8001ED0F8041821F00201C0F80418F2
:106D000000207047D0F8001E21F00301C0F8001EDB
:106D1000D0F8041841F00201C0F8041800207047B0
:106D20002DE9F04F00250E460446DDF82CC0DDF8B5
:106D300024B0109F2846294604EB8002C2F80411B3
:106D4000401C0F28F8D32046C7B1806B20F40012F6
:106D5000A263A06B40F40022A26308468846C4F8F0
:106D6000000ED4F800182046C4F80018BCF1010F3A
:106D700016D0D0F8001841F0030116E0D0F804084E
:106D800040F00202C4F80428A06B40F40012A26391
:106D9000A06B20F40022A263A06B20F48022DBE72A
:106DA000D0F800180BB141F00101C0F80018102113
:106DB00000F090FA00B10125204600F07BFA00B106
:106DC00001254046C4F81088C4F81488C4F81C880B
:106DD00000214FF000694FF0904A4FF67F3314E0E6
:106DE00004EB4112D2F800C9BCF1000F06DA11B170
:106DF000C2F800A904E0C4F8009901E0C2F8000953
:106E0000C2F81009C2F80839491C8E42E8D800219E
:106E100015E000BF04EB4112D2F800CBBCF1000F2B
:106E200006DA11B1C2F800AB04E0C4F8009B01E03F
:106E3000C2F8000BC2F8100BC2F8083B491C8E4286
:106E4000E8D8D4F8101821F48072C4F81028A06192
:106E50006FF080406061BBF1000F03D1A06940F08A
:106E60001000A061A06909490843A0610C9818B1FD
:106E7000A06940F00800A061012F03D1A069044976
:106E80000843A0612846BDE8F08F000000383C8030
:106E900004000040816821F00101816000207047FA
:106EA00070B50D784E78434CEBB200EB4313012ED6
:106EB0001FD0D3F8100B6FF31200C3F8100BD3F8E8
:106EC000100B2040C3F8100B486908B1886848616E
:106ED000D3F8100B40F40020C3F8100BD3F8100BBC
:106EE0008C68C4F312042043C3F8100B012A55D058
:106EF00058E04E69002ED3F8106932D06FF31206B5
:106F0000C3F81069D3F810692640C3F810694E69B8
:106F10008C68A64200D94C61D3F8104944F400248F
:106F2000C3F81049D3F810494E69C6F3120634432A
:106F3000C3F81049012A22D000EB4512D2F80039DB
:106F400043F00443C2F800394A6932B3D0F8342818
:106F5000097801F00F03012199400A43C0F8342851
:106F600026E02640C3F81069D3F8104944F4002401
:106F7000C3F81049D3F810496FF31204D8E7096930
:106F800019B100EB4512C2F8141900EB4510D0F806
:106F9000001941F00441C0F8001909E0C86808B1BF
:106FA000C3F8140BD3F8000B40F00440C3F8000BF7
:106FB000002070BDFFFF07E010B5036C134CA34227
:106FC00003D9D0F8003B002B1EDB0023C0F8103B98
:106FD000D0F8103B43F40023C0F8103BD0F8103B2E
:106FE00043F01803C0F8103BD0F8103B43F0C04307
:106FF000C0F8103B012907D1C0F8142BD0F8001BB2
:1070000041F08021C0F8001B002010BD0A30544F11
:107010004A780B78012A00EB43100BD0D0F8002BF4
:1070200022F40012C0F8002BC978032914D00229D9
:1070300012D017E0D0F8002922F40012C0F800297D
:10704000C978032901D002290CD1D0F8001941F0E8
:107050008051C0F8001905E0D0F8001B41F08051C4
:10706000C0F8001B002070470A784B78D1B200EBC3
:107070004110012B12D0D0F8001B002906DB2AB1E9
:10708000D0F8001B21F08041C0F8001BD0F8001B95
:1070900041F40011C0F8001B00207047D0F800191F
:1070A000002906DB2AB1D0F8001921F08041C0F890
:1070B0000019D0F8001941F40011C0F80019EBE7ED
:1070C000F8B50C784F78774DE3B26FF0604600EB7F
:1070D0004313012F26D0D3F8104B6FF31204C3F8DB
:1070E000104BD3F8104B2C40C3F8104B4C69002CBC
:1070F00074D08D682C44641EB4FBF5F4D3F8105B97
:10710000A4B206EAC4463543C3F8105BD3F8105B5B
:107110008E686643C6F312042543C3F8105B012A48
:1071200071D0A6E04F691FB3D3F810796FF312073F
:10713000C3F81079D3F810792F40C3F810794F694C
:107140008D682F447F1EB7FBF5F506EAC545D3F8D9
:1071500010693543C3F81059D3F810594E69C6F376
:1071600012063543C3F81059CD78012D10D01BE01D
:10717000D3F810692E40C3F81069D3F8105945F4BC
:107180000025C3F81059D3F810596FF3120509E020
:10719000D3F8105925F0C045C3F81059D3F8105949
:1071A00045F00055C3F81059012A18D000EB4413DC
:1071B000D3F8004944F00444C3F80049CC78012CCA
:1071C0002FD04A6962B3D0F83428097801F00F0350
:1071D000012199400A43C0F8342860E036E00A698A
:1071E0001AB100EB4413C3F81429C97801290FD14F
:1071F000D0F80818C90500EB4411D1F8002903D4D0
:1072000042F0005202E030E042F08052C1F8002922
:1072100000EB4410D0F8001941F00441C0F8001907
:107220003DE0D0F80848E405D3F8004902D444F022
:10723000005401E044F08054C3F8004900928A8A67
:1072400093B20A78C96800F03FF928E0D3F8104BF0
:107250008D68C5F312052C43C3F8104BD3F8104BBF
:1072600044F40024C3F8104B59E7CA680AB1C3F8C4
:10727000142BC97801290CD1D0F80808C005D3F81F
:10728000000B02D440F0005001E040F08050C3F801
:10729000000BD3F8000B40F00440C3F8000B0020B3
:1072A000F8BD0000FFFF07E0816841F00101816047
:1072B00000207047002110220261054A491C9142BA
:1072C00001D9032070470369DB06F7D4002070471B
:1072D000400D03000022202343EA8111016105498A
:1072E000521C8A4201D90320704703699B06F7D4D8
:1072F00000207047400D0300D0F8080810F0060089
:1073000004D0022803D0062801D00F2070470220A5
:107310007047406900F001007047D0F81818D0F8A5
:107320001C08084080B27047D0F81818D0F81C0824
:107330000840000C704710B5D0F81038D0F8342849
:1073400001F00F0400EB4110E24002F00102D0F81E
:10735000080943EAC212104010BD00EB4111D1F8F8
:10736000081BD0F81408084070474169806908403C
:107370007047D21C10B59308002200F5805002E03F
:107380000468521C10C19A42FAD3084610BD10B5C9
:10739000C26822F0C042C260012902D029B1012096
:1073A00010BDC16841F0005102E0C16841F0804168
:1073B000C1603220FAF772FA002010BDD0F8002820
:1073C00022F4FE62C0F80028D0F800284FF4FE63D3
:1073D00003EA01110A43C0F80028002070470000AA
:1073E000022A3ED1264A274B0A449A4201D20F2153
:1073F00038E0254A254B0A449A4201D20E2131E059
:10740000234A244B0A449A4201D20D212AE0224AFF
:10741000224B0A449A4201D20C2123E0204A214BFC
:107420000A449A4201D20B211CE01F4A1F4B0A4416
:107430009A4201D20A2115E01D4A1E4B0A449A4283
:107440000FD31D4A1D4B0A449A4201D2082109E07C
:107450001B4A11441B4A914201D2072102E0062136
:1074600000E00921C26822F47052C260C2684FF481
:10747000705303EA81210A43C26000207047000074
:10748000405327FF00350C00401E1BFF40420F00F9
:1074900000DC0BFF804F1200808CF9FE20D6130019
:1074A00060B6E5FE60E3160000D3CEFE40771B0019
:1074B000C05BB3FEC091210000CA91FE2075380068
:1074C000E05459FEE09C410010B5029C64B9DB1CFD
:1074D0009C0800EB0230002300F5805002E004C954
:1074E00002605B1CA342FAD3002010BD0348017860
:1074F00021F001010170007870470000200A00109F
:1075000010B570B90D480078C00701D0032010BD38
:1075100069B1012907D04FF4007002290AD003296C
:1075200003D0042010BD4FF40050106003E0FAF7C0
:1075300001F800E01080002010BD0000200A0010BB
:107540002DE9F0471E461746884638B936B10F4830
:107550000078C00704D00320BDE8F0870420FBE7D3
:1075600000252C464FF400790BE000BF381908EBDA
:10757000050240024946F9F763FF641CA4B205F511
:107580000075B442F2D30020E6E70000200A0010A4
:1075900008B101207047014800787047200A0010A8
:1075A0002DE9F0471E461746884638B936B11148CE
:1075B0000178C90704D00320BDE8F0870420FBE769
:1075C0000078400701D50220F6E700252C464FF44D
:1075D00000790AE0381908EB050240024946F9F73C
:1075E000B5FE641CA4B205F50075B442F2D30020C8
:1075F000E2E70000200A0010FEE70000ADF5306D64
:10760000FEA000F0CDFC4FF0000BADF874BACDF841
:1076100070BA8DF8E4BA8DF8E8BACDF864BACDF84E
:1076200080BA4FF400745D46CDF878BACDF87CBAD4
:10763000CDF884BA21460DF58160CDF86CBAF8F723
:10764000ECFE21460DF63800F8F7E7FEDFF8C4A39C
:107650000BE000BF5FEA080007D001280DD0022828
:107660001AD0B8F1030FF5D12BE09AF800000128E9
:107670000CD001201EF0D6F9F7E7002211461020A9
:107680000CF0BCFCCDF8EC0A10B3022080460120BF
:107690001EF0C8F94046E0E75022DF49DDF8EC0A69
:1076A0000CF042F9A0B9FF21DDF8EC0A0CF052FC15
:1076B000DAA1102000F0FEFB4FF0030801201EF0BD
:1076C000B1F90DF66821DDF8EC0A0BF0FBFF18B1FB
:1076D00001201EF0A7F9BDE71EF000FBD6A1102087
:1076E00000F0E8FB5E46ADF874BA00248DF8E4BA09
:1076F0008DF8E8BADDF8780AC8212746A0F804B06A
:10770000DDF8780AA0F80CB0DDF8680AADF880BAA8
:10771000C1610DF69C210CF03DFD20B1CAA11020E5
:1077200000F0C8FB55E21EF0D9FA0DF6F82200234E
:10773000111FDDF8680A0CF087FB0DF67422111F8B
:10774000DDF89C0A0BF0D2FEBDF8742ADDF8700A51
:10775000B346C2A186540522F8F7B1FE40B10B2210
:10776000C0A1DDF8700AF8F7AAFE00287BD030E24D
:10777000DDF8700A00222021401D13F042FE06B2FF
:10778000002E2CD047DD06F105000FF041FCCDF8AE
:10779000640A90B3DDF8700A0A22B5A1401DF8F71B
:1077A0008EFE58B3DDF8700A0522B4A1401DF8F72B
:1077B00086FE18B3B3A1DDF8640A00F041FBDDF8E2
:1077C000640ADDF8701A3246001D491DF8F7FEFD07
:1077D000361D36B2DDF8640A00F806B01BE00F2053
:1077E0000FF016FCCDF8640A38B1A8A1F8F75EFED8
:1077F000DDF8641A81F80EB00DE009E0FFE7DDF86E
:10780000701A3246491DDDF8640AF8F7DFFDE1E73A
:1078100001208DF8E80A9DF8E80A38B1DDF89C0AE5
:107820009EA18268102000F045FBEAE14FF0FF3195
:10783000DAF808001EF072FC01282FD101220DF5A4
:10784000C160DDF8641A06F0D9F898B301208DF80C
:10785000E40A00BF9DF8E40A00B393A10DF68C2062
:10786000F8F724FE00E08FE093A10DF63820F8F73A
:107870001DFE0DF638230DF68C22924902A80094C5
:1078800000F0DEFA02A8F8F7EFFD0246002302A995
:10789000CDF800B0DDF8680A0CF0ECFEDDF8640A03
:1078A0001DF002FF00231A461946DAF808001EF000
:1078B000AFFA8EE1FFE784A10DF68C20DDF81446C7
:1078C000F8F7F4FD0DF63821DDF8640AF9F758FEF3
:1078D0000DF638230DF68C227A4902A8009400F0A8
:1078E000AFFA02A8F8F7C0FD5F46CDF800B00CB1C2
:1078F000022300E00023024602A9DDF8680A0CF02A
:10790000B9FEC4B3BB46CDF8A07A002640F2B45706
:107910004FF00309BC4201D9384600E020460FF081
:1079200077FBCDF8600A38B3A01B40F2B457B842D9
:1079300002D829F00209074631460DF5C16005F06D
:1079400063FC0DF52A633A460DF5C160DDF8601A57
:1079500006F064FA4B463A46CDF800B0DDF8601AFE
:10796000DDF8680A0CF086FE3E44A642DCD3DDF862
:10797000600A1DF099FE02E001208DF8E40A0DF581
:10798000C16005F097FB65E751A1DDF8700AF8F7D3
:107990004FFD18B11030F8F7E7FD87B250A1DDF8C0
:1079A000700AF8F745FD38B3083004460A220D2165
:1079B00013F027FD0604360C1ED030460FF028FBCE
:1079C000CDF86C0AC0B132462146F8F7FFFC3021F1
:1079D0000DF52B60F8F721FDDDF86C0ACDF8A00A53
:1079E0000DF52B60CDF8A4BACDF8A80ACDF8ACBA45
:1079F000ADF8A46A103877E07DE000004854545098
:107A0000206461656D6F6E20737461727465640AC1
:107A100000000000000000204C830408576562202D
:107A2000736572766572206C697374656E20706F11
:107A300072742038300D0A00436F6E6E656374698E
:107A40006F6E0D0A0000000052656365697665205F
:107A500074696D656F75740D0A0000004745542008
:107A60002F000000504F5354202F6170692E630087
:107A7000636F6E6669672E786D6C00006D69627366
:107A80002F0000007765622F000000007765622FED
:107A9000696E6465782E68746D6C00004E6F206DA1
:107AA000656D6F72790D0A00343034204E6F74208A
:107AB000466F756E64000000746578742F68746D8D
:107AC0006C000000F0970408323030204F4B00006B
:107AD000436F6E74656E742D4C656E6774683A0002
:107AE000436F6F6B69653A0003F075F80DF52A6016
:107AF000CDF8780A01E0CDF878BAEFB3781C0FF032
:107B000087FA040061D0BDF8740ADDF8701AC01B52
:107B100001443A462046F8F759FC04F807B00DF640
:107B2000F420CDF8840A5E46CDF87C4AADF8807A20
:107B300022463CA1102000F0BDF90DF638034FF4A9
:107B400000720DF581610DF6782009F009F92046E3
:107B50001DF0AAFD0DF5816237A1102000F0AAF9F1
:107B6000AFF29C010DF68C20F8F7A0FC0DF6382141
:107B700037A0F9F705FD00E027E00DF58160F8F783
:107B800073FC0DF63801CDE900010DF638230DF632
:107B90008C22314902A800F053F902A8F8F764FCDE
:107BA0000246032302A90096DDF8680A0CF062FD84
:107BB0000DF58160F8F758FC024601230DF581614F
:107BC0000096DDF8680A0CF055FDDDF86C0A1DF032
:107BD0006BFD4FF4FA7400BFDDF8680A4078C00707
:107BE0000AD01EF07BF828466D1CADB2A04215D11C
:107BF0001AA1102000F05EF900251EA1102000F04F
:107C000059F9DDF8680A0BF0EBFEDDF89C0A0BF081
:107C1000EBFCDDF8680A0BF09DFF1BE501201DF071
:107C200001FFD9E70D0A72657175657374206A7377
:107C30006F6E2025730D0A00726573706F6E736529
:107C4000206A736F6E2025730D0A0D0A0000000074
:107C50002E6A736F6E0000009C9804083530306DFA
:107C60007320726563656976652074696D656F75EB
:107C7000740D0A00436F6E6E656374696F6E2063E6
:107C80006C6F73650D0A00002DE9F04700248946EA
:107C9000824626462CE0184FDFF8608000253888A1
:107CA000002281B24046FAF7F2FA022000F004FA0C
:107CB0003888012281B24046FAF7E9FA0A2000F03A
:107CC000FBF9388881B24046FAF7DCFA44EAC01082
:107CD000C4B2072D00D064083C2000F0EDF96D1C03
:107CE000EDB2082DDBD30AF806400024761CF6B26C
:107CF0004E45D0D3BDE8F087C01F002000080240E9
:107D000070B5124C124D0022208881B22846FAF735
:107D1000BEFA4FF4F07000F0CFF92088012281B252
:107D20002846FAF7B4FA412000F0C6F9208881B25B
:107D30002846FAF7A7FA38B15FF000044FF4CD7087
:107D400000F0BAF9204670BD0124F7E7C01F0020FB
:107D5000000802402DE9F047894682460024184E6B
:107D6000DFF8608027E000BF1AF804700025308833
:107D7000002281B24046FAF78AFA022000F09CF90C
:107D8000F80705D03088012281B24046FAF77FFA21
:107D90003A2000F091F93088012281B24046FAF78A
:107DA00076FA022000F088F96D1C7F08EDB2082DEC
:107DB000DDD3641CE4B24C45D6D3BDE8F0870000A7
:107DC000C01F00200008024009490020086008493F
:107DD0001431086006481038016841F00101016063
:107DE00004494FF40000C1F88002C1F80001704757
:107DF0001014004004E000E00748016821F0010190
:107E0000016006494FF40000C1F88001BFF34F8FB5
:107E1000BFF36F8F704700000014004004E000E0E3
:107E20000FB4054B10B503A9044A029800F0F6FA06
:107E300010BC5DF814FB0000F9E7020854020020B2
:107E40000FB4084B10B504A902AA039800F0E6FA93
:107E5000044602A9002000F064FE204610BC5DF834
:107E600014FB0000238B020837B514460846064B66
:107E70006A46214600F0D2FA04466946002000F026
:107E800050FE20463EBD0000238B02080907090E64
:107E9000002804DB00F1E02080F80014704700F0B7
:107EA0000F0000F1E02080F8141D70470048704773
:107EB0006C0C00100FB470B5174D696811B32968C8
:107EC00001421BD04FF0FF31A8681EF027F906AA27
:107ED00012480599FFF7C8FF1048F8F7C5FA0400E3
:107EE00012D003F045FB18B1A1B20C48F9F7EEF837
:107EF00000231A461946A8681DF08AFF012070BCAD
:107F00005DF814FB0020FAE700231A461946A8681A
:107F10001DF07EFFF6E70000740000206C160010D4
:107F20001CB501201DF00CFF094C01210022A060AE
:107F300008021DF017FFE0600020211DCDE90001BF
:107F400003464FF4007203A106481EF0A3F91CBDBE
:107F50007400002064656275672073747265616DDA
:107F600073000000A53B040830B583B0044600F060
:107F700087F89FED090B05468DED000B0022214689
:107F80006846F8F70AFD284600F090F89DED000BD2
:107F900003B030BD00000000000000000000000041
:107FA0000FB44FF0FF3130B5234C85B020681EF080
:107FB000B5F809AA21480899FFF756FF122220A117
:107FC000214805F01BFD00282CD11F4DE968B1F5B3
:107FD000002F10D3284605F06DF81CA006F0C7F856
:107FE0001AA117A005F0D8FF122215A1284605F006
:107FF00005FDB8B9E968144805F006F916480DF111
:10800000040C0E4D417AC379027A8CE82E008188E7
:108010000091C378827811A10B4805F019FE0A4837
:1080200005F048F800231A46194620681DF0F0FEB6
:1080300005B030BC5DF814FB080000209C20001047
:108040006C6F672E747874006C1E00106F6C645F28
:108050006C6F672E747874001C1600102530326423
:108060002E253032642E253032642F253032643A8A
:10807000253032643A253032642025730000000038
:1080800001480068704700006C0C001002E008C84E
:10809000121F08C1002AFAD170477047002001E082
:1080A00001C1121F002AFBD170470000014908607E
:1080B000704700006C0C001010B504461EF016F955
:1080C0000146054801608480BDE810404FF0FF3153
:1080D00001201BF009BC0000F80000202DE9FF5F23
:1080E00082B00021DDE90430020DDDF840B0034329
:1080F00018D044F61050A2F2FF32424315141198E2
:1081000001281FD0A5EB0B00401C5FEA000A4FF0CE
:1081100000064E4FDFF83891B046504615D5CAF1EB
:10812000000413E0119801244AA3012801D16FEA49
:108130000B010298119AC0E90031C0E9024206B071
:10814000BDE8F09FCBF10000DFE704460021404A84
:10815000491842EB0450CDE9001012E0E00707D0C7
:1081600032463B4640464946F8F7B2FA80468946D1
:1081700032463B4610461946F8F7AAFA06460F461D
:108180006410002CEAD1DDE90401DDE90023BAF135
:10819000000F06DAF8F79CFA42464B46F8F798FAD1
:1081A00005E0F8F7C1FC42464B46F8F7BDFC044633
:1081B0000E460022284BF8F71BFB03D84FF0FF3088
:1081C000014607E00022254B20463146F8F7D9F951
:1081D000F8F719FD102409E0002C0ADB0A2200231D
:1081E000F8F762F8039B30321A55641E50EA010218
:1081F000F2D1641C039AC4F111031444119A012AA8
:1082000003D0012208430DD10AE0084304D0002026
:108210004FF0110B119072E7A3EB0B056D1E0DE0F3
:108220005B4504DD4FF0000205F1010504E003DACF
:108230004FF00002A5F10105002AECD00298119937
:10824000C0E90231C0E9004579E7000000001440B0
:108250000000F03F300000000000F0430000E03F6D
:1082600030380A2801D201207047002070470000F2
:1082700010B50F4CE06A012817D1206B401C206319
:10828000D4F8340104EBC00090F83410022902D075
:108290000920E06207E0816B4A1C8263002902DD4D
:1082A0002C2009F06DF809F037F8E06A10BD0000E5
:1082B000841E002030B5154C0546E06A012823D104
:1082C000206B401C2063D4F8340104EBC00090F80C
:1082D0003410012902D00A20E06207E0816B4A1CB9
:1082E0008263002902DD2C2009F04AF809F014F815
:1082F000284609F061F83A2009F042F8D4F838012C
:1083000010B1202009F03CF8E06A30BD841E002046
:1083100030B5821C7D2901D07E2906D103887D25B8
:108320005C1C04809D5401F0DF0103885C1C048008
:10833000995430BD2DE9F04104460E4608880AF0F4
:1083400085FA051E15D00020A4F804066070207080
:1083500031882A46B01C03F029FE060005D00146EC
:1083600028460EF053F8FF2805D0284606F04EFAAE
:108370000020BDE8F08129784FF0010708060BD4F2
:1083800005EB510011F0010F407800D0000900F01A
:108390003F000E2800D167702878A070B01EA4F8A6
:1083A0000406721E691CE01CF8F710F827702846B6
:1083B00006F02CFA0120DCE72DE9F0430646B0F880
:1083C00002060C46401C81B230460EF01FF8002118
:1083D000A71C0122C0434FF07E08228000F0FF0955
:1083E00001F8078031782046FFF792FF002506E06C
:1083F000701941782046FFF78BFF6D1CADB2B6F8BF
:108400000206A842F4D849462046FFF781FF20889B
:10841000411C218000F80780BDE8F0832DE9FF4F63
:1084200095B09A46884606460025EEE1252877D184
:1084300000242746F94A0121039400E0044316F87A
:10844000013F203B01FA03F01042F7D130782A288F
:1084500011D06FF02F033078A0F13002092A16D81E
:10846000039A44F0020402EB820203EB420210443E
:10847000761C0390EFE758F8042B0392002A03DAE6
:10848000504244F40054039044F00204761C3078C7
:108490002E2816D116F8010F44F004042A280DD016
:1084A0006FF02F023078A0F13003092B09D807EBC9
:1084B000870302EB4303C718761CF3E758F8047BE5
:1084C000761C30786C280FD006DC4C2817D0682832
:1084D0000DD06A2814D104E0742810D07A280FD166
:1084E0000DE044F400140AE044F4801401E044F484
:1084F00040147278824202D104F58014761C761CF6
:10850000307866280BD013DC582877D009DC002897
:1085100075D04528F6D04628F4D047281AD193E1E3
:1085200018E0632835D0642879D0652812D18BE112
:10853000702873D008DC6728F1D069286FD06E28C6
:108540000DD06F2806D1ACE073282CD0752874D0DC
:10855000782853D05246179990476D1C54E1C4F3C4
:108560000250022809D003280DD0D8F800100428A2
:108570000DD00D6008F1040846E1D8F80010EA17A4
:10858000C1E90052F6E7D8F800100D80F2E70D704F
:10859000F0E718F8041B8DF8001000208DF801009A
:1085A000EB46012003E058F804BB4FF0FF306107B1
:1085B0004FF0000102D40DE009F101018946B942F2
:1085C0000FDA8145F8DB1BF809100029F4D108E027
:1085D00009F1010189468142FADB1BF809100029E3
:1085E000F6D103985346A0EB090721463846179A5F
:1085F00000F080FA284400EB090507E044E008E1B8
:108600000DE01BF8010B524617999047B9F101098B
:10861000F7D2534621463846179AF2E039E00A214C
:10862000C4F302524FF0000B0091022A06D058F812
:10863000040BC117032A09D00AE023E008F1070060
:1086400020F00702F2E80201904605E000B2C117EF
:10865000042A01D140B2C117002906DA0A460021D6
:10866000404261EB02012D2202E0220504D52B22BB
:108670008DF80420012203E0E20701D02022F7E771
:10868000914657E00A2100E010214FF0000B0091C5
:108690000BE010214FF0000B44F004040827009178
:1086A00003E008204FF0000B0090C4F30252022AAE
:1086B00005D058F8040B0021032A08D008E008F17F
:1086C000070020F00702F2E80201904603E080B2C2
:1086D000042A00D1C0B24FF0000922072AD532780F
:1086E000702A07D0DDF800C08CF0100C5CEA0B0C8F
:1086F00005D00EE040228DF80420012208E050EA67
:10870000010306D030238DF804308DF805200222B5
:108710009146009B83F0080353EA0B030AD150EA09
:10872000010201D1620705D530228DF804204FF0F7
:1087300001097F1E3278582A04D039A20C920CAA63
:1087400002920BE03BA2F9E75B46009AF7F7ACFD1B
:108750000C9B9B5C029A521E0292137050EA01021B
:10876000F2D1029804A9081A00F1200B600702D583
:1087700024F4803400E001275F4502DDA7EB0B0005
:1087800000E0002000EB0B01009003984944401AE0
:108790000390E00306D453462146179A039800F04D
:1087A000A9F90544002706E001A85246C05D1799C3
:1087B00090476D1C7F1C4F45F6DBE0030CD55346FC
:1087C0002146179A039800F095F9054404E03020FB
:1087D0005246179990476D1C0099481E0090002939
:1087E000F5DC08E00298029952460078491C029193
:1087F000179990476D1CBBF10001ABF1010BF1DC47
:108800005BE100F065F90544761C307800287FF4C0
:108810000DAE19B02846BDE8F08F00000928010010
:1088200030313233343536373839616263646566E6
:1088300000000000303132333435363738394142A8
:108840004344454600000000600700D4062708F1B5
:10885000070020F00700F0E80223804603F0004CF8
:108860005FEA0C0001D097A009E0200501D596A091
:1088700005E0E00701D095A001E0AFF24C001390B5
:10888000307823F0004365280CD006DC452809D059
:1088900046281DD047287FD13BE0662818D067289E
:1088A0007AD136E00021112F01DB112000E0781C85
:1088B000CDE9000104A90CA8FFF710FCDDE90D01CA
:1088C0000C9A4FF0000B07F10109109200914EE055
:1088D0004FF000400097CDE9011004A90CA8FFF764
:1088E000FDFBDDE90D020C9B0F994FF0000B91464B
:1088F0001093009211B9791C00EB0109B7EB090044
:1089000003D4C0F1FF3B07F10109A9EB0700019077
:1089100042E0012F00DA01270021112F01DD112093
:1089200000E03846CDE9000104A90CA8FFF7D6FB0A
:10893000DDE90D010C9A00914FF0000BB946109241
:1089400021070FD4009A4A4503DA914601E0A9F1C4
:108950000109B9F1010F05DD109AA9F10101515C7E
:108960003029F4D0B84202DA10F1040F03DA012101
:10897000CDE9011010E0002803DC8344A9EB0001DD
:1089800002E0411C494500DD8946A0EB0B00401C7C
:1089900001904FF000400290200705D4019848450F
:1089A00002DB4FF0FF30019000208DF84B00029861
:1089B0000DF14B07B0F1004F25D002200C902B2079
:1089C0000D90029800280CDA404202902D200D9064
:1089D00007E00A210298F7F73FFF3031029007F8CD
:1089E000011D0C99481E0C900029F2DC0298002809
:1089F000EFD1791E0D980870307800F0200040F01B
:108A0000450007F8020D11A8C01BC01D0290139865
:108A1000007800B1012000EB0901019801EBE07141
:108A2000029801440398401A401E0390E00306D4C4
:108A300053462146179A039800F05CF805441398B2
:108A4000007818B15246179990476D1CE00323D562
:108A500053462146179A039800F04CF805441BE052
:108A6000BBF1000F07DB0098584504DD10981799FB
:108A700010F80B0001E017993020524690470198FA
:108A80000BF1010B401E05F10105019004D12E20D0
:108A90005246179990476D1CB9F10001A9F10109DF
:108AA000DEDC05E017F8010B5246179990476D1C64
:108AB0000299481E02900029F4DC53462146179A79
:108AC00003989EE62D0000002B000000200000000F
:108AD0002DE9F041044600251E461746880404D4BB
:108AE00005E039462020B0476D1C641EF9D52846A4
:108AF000BDE8F0812DE9F041044600251E46904670
:108B0000C80301D5302700E02027880404D505E0FC
:108B100041463846B0476D1C641EF9D52846BDE86D
:108B2000F0810A68531C0B60107070472DE9F04704
:108B30000024984691460D4606462746F7F794FCD2
:108B400010F0FF0005D008E0641CE4B2A04202D19E
:108B50000020BDE8F0877F1CFFB2E919725C4A452E
:108B6000F2D1002005E04119725C08F80020401C99
:108B7000C0B2A042F7D3002108F804102046E8E76D
:108B80002DE9F04790460E4604006FF0050555D0DC
:108B900004F11400814612F0BBFD00284ED0EF1FF7
:108BA000002E3DD0B8F1000F06D032A340F22A22A9
:108BB0003DA147A0FFF734F92078A16A0AF024FE0E
:108BC00005004FF0FF383DD06E600EF069FF29467A
:108BD000484612F08BFDA0B36C680021204613F0CC
:108BE00001FC0021204617F057FA0021204617F01B
:108BF000A5FF00221146204616F080FA00212046EB
:108C000014F0A2F90020686005F11000044612F08B
:108C10002FFD204612F066FD28460BF05FF81FE09E
:108C2000384609F0E5FC0146484612F05FFD28B9D8
:108C3000A36A1BB100221146204698472846BDE88A
:108C4000F0870FE0384609F0D3FC0146484612F0A1
:108C50004DFD28B9A36A1BB1002211462046984752
:108C60004046ECE7A36A1BB1002211462046984714
:108C70000020E4E72E2E2F4D6964646C65776172E5
:108C800065732F54686972645F50617274792F4CF8
:108C90007749502F7372632F6170692F6170695F1C
:108CA0006D73672E63000000657870656374206ED5
:108CB0006577706362203D3D204E554C4C206F72AD
:108CC00020657272203D3D204552525F4F4B00009F
:108CD000417373657274696F6E202225732220665A
:108CE00061696C6564206174206C696E652025641F
:108CF00020696E2025730A0070B50446C0680D46D1
:108D00004069001D12F009FDE06821464069826853
:108D100028469047E0680021406912F059FCE0685D
:108D20004069BDE87040001D12F01EBDF0B5ADF207
:108D3000EC4D054600200F46CDF8E4041646802190
:108D40000DF26440F7F769FB344C4FF0FF312068B7
:108D50001DF0E4F9122232A101A804F04FFE28B957
:108D6000012232A18DA804F049FE48B100231A4621
:108D7000194620681DF04CF800200DF2EC4DF0BDB6
:108D80008DAA80210DF2644004F01AFA00282CD03C
:108D90003C210DF26440F7F75DFB0028F0D026A1DE
:108DA000F7F746FBD8B126A1F7F742FBB8B122216D
:108DB000F7F750FB98B10DF2E44322220121FFF7AF
:108DC000B5FE0DF2E440F7F7CFFBA84207D13B46D2
:108DD0002A461CA101A8009604F03AFFD0E70DF244
:108DE000644101A804F034FFCAE79099939888423F
:108DF000C6D18DA804F05EF901A804F05BF90BA0C0
:108E000005F0B5F909A106A005F0C6F800231A4639
:108E1000194620681CF0FCFF0120AEE70800002086
:108E2000546C6F67696E2E786D6C00006C6F6769AB
:108E30006E2E786D6C000000757365720000000086
:108E400069640000093C757365722069643D2225E0
:108E50006422206E616D653D22257322207061734E
:108E6000733D22257322207065726D697373696F7B
:108E70006E733D2232313437343833363437222F53
:108E80003E0A00002DE9F043B3B089460446242190
:108E900012A8F7F7C2FA14211BA8F7F7BEFA0021AF
:108EA00030912E912F912B912C912D91242120A83E
:108EB000F7F7B3FA00273E46002C67D01BAA3AA169
:108EC000204601F042FE2EAA39A1204601F03DFEC7
:108ED0002BAA39A1204601F038FE20AA38A120464D
:108EE00001F033FEDFF8E480002400BFC4EBC401CE
:108EF00008EBC1000546427C1BA9F7F7CAFA002817
:108F000048D0687C002845D0641C14F0FF04EDD0E4
:108F10002BA8F7F729FB04462D4819F0E9FCA042DD
:108F200034D32C49001B884230D848216846F7F7D3
:108F300074FA6D460DEB07001BAA27A1FEF780FF10
:108F4000C6EBC60108EBC1023844C7B21232144660
:108F5000E81921A1FEF774FF3844C6B2A8192BAA5C
:108F60001DA1FEF76DFF3044C6B2A8192EAA1AA1A2
:108F7000FEF766FF3044C1B212AA684605F058FDFC
:108F8000202212A920A8F7F784FA28B1002033B0D4
:108F9000BDE8F0832646BBE721464A461BA80EF0F3
:108FA000FBFC0120F3E700006C6F67696E000000B6
:108FB0006E6F6E636500000074696D6500000000EF
:108FC00070617373776F72640000000028160010E0
:108FD0001C160010805101002573000010B50446D6
:108FE0000020E070401EA06320460AF0F0F908B1AE
:108FF000042010BD04F23A2008F00BFAA0F52A4133
:10900000553901D0032010BD94F83C00E92805D063
:10901000EB2814D194F83E00902810D104F172008E
:1090200008F0ECF90749B1EB002F06D004F18E00EF
:1090300008F0E4F90449884201D1002010BD022063
:1090400010BD0000004641544641543300E0401C2E
:1090500002780AB18A42FAD1D0B27047F0B5002244
:10906000144D134605EB021426685EB10768BE4234
:1090700009D166688768BE4205D1A4684669B442D2
:1090800004D000E00123521C022AEBD3022A01D0B3
:1090900069B904E04BB9022907D01220F0BD05EBF5
:1090A00002108089B0F5807F01D00020F0BD102033
:1090B000F0BD0000A82F001030B50021054B0C4674
:1090C00003EB01121568854200D11460491C022986
:1090D000F6D330BDA82F00100268490AC06A528931
:1090E000B1FBF2F1001D04C81AB1914203D3891AF1
:1090F000F8E7002070470068084470471CB500205E
:109100000090034601904FF4806202A104481DF0D4
:10911000C1F81CBD436C6F636B5461736B0000003E
:10912000613A040870B50A4C0025A5822561A06843
:1091300010B10CF0DFFCA5600021064812F076FCAF
:109140006068002803D0216849688847656070BD61
:1091500014BE022065270408026A891E921E8A42F4
:1091600001D800207047426B408901FB0020704706
:109170002DE9F0419AB08046142113A8F7F74DF974
:10918000242101A8F7F749F924210AA8F7F745F99E
:1091900000248DF860402646052313AA33A14046DB
:1091A000009407F0D3FC012857D1324F002500BFAF
:1091B000C5EBC50007EBC000427C42B113A9F7F72D
:1091C00068F960B901208DF860002E460BE02AA1F5
:1091D0002BA008F061F82CA127A008F05DF86D1C09
:1091E00015F0FF05E4D09DF86000002838D0052375
:1091F0000AAA2AA14046009407F0A8FC01280BD136
:1092000001E01DA027E0052301AA25A14046009406
:1092100007F09CFC012805D017A119A008F03CF824
:1092200019A1EEE7C6EBC60007EBC00505F1120475
:10923000212201A92046F7F72CF988B920462122DE
:109240000AA9F7F7C3F8224629463046FFF76EFD14
:1092500030B115A10AA008F01FF81AB0BDE8F081DE
:1092600005A107A008F018F810A1CAE77573657288
:1092700000000000281600106572726F7200000076
:109280007374617475730000696E76616C69642033
:10929000706172616D657472000000006E65770028
:1092A00063757272656E74006F6B0000706173732A
:1092B000776F7264206368616E6765206572726F94
:1092C0007200000010B58AB0142104A8F7F7A5F8C1
:1092D000174890F8541090F8574090F8563090F88E
:1092E00055208DE81E0090F8533090F8522011A1BF
:1092F00004A8FEF7A5FD17A117A007F0CDFF18A041
:1093000007F0B0FF04A917A007F0C6FF084916A090
:1093100007F0C2FF064915A0103107F0BDFF044950
:1093200014A0203107F0B8FF07F054FF0AB010BDB9
:10933000700C0010253032583A253032583A25301A
:1093400032583A253032583A253032583A253032A0
:10935000580000006F6B0000737461747573000037
:109360006E6574004D414300697000006D61736B60
:10937000000000006777000010B51BA11BA007F0DC
:109380008BFF1C4819F0B4FA01461BA007F05AFFE6
:109390001848807A010704D5C0F3C00118A007F06F
:1093A00043FF002011F072FD06F00EFD014615A0EE
:1093B00007F072FF002011F073FD014612A007F0C4
:1093C00041FF002011F052FD4FF47A71B0FBF1F132
:1093D0000FA007F037FF002011F050FD0146BDE857
:1093E00010400DA007F02EBF6F6B00007374617406
:1093F000757300001C16001074696D650000000094
:10940000626C0000697000007374726174756D00A5
:10941000706F6C6C00000000726561636800000092
:1094200010B506A106A007F037FF074890F9001015
:10943000BDE8104005A007F005BF00006F6B0000FD
:1094400073746174757300001C160010636F727280
:109450000000000010B5FF2411F00AFB08B1002441
:1094600003E011F00CFB00B1012414A114A007F0DB
:1094700013FF214614A007F0E5FE0FF02BF801467C
:1094800013A007F009FF15A007F0ECFE00200FF075
:10949000F7FA014613A007F0C7FE0FF021F80146C6
:1094A0000BA007F0F9FE00200FF026F801460FA0F0
:1094B00007F0F2FEBDE8104007F08CBE6F6B0000B5
:1094C000737461747573000076657273696F6E00F2
:1094D000636F6D6D756E69747900000074726170F0
:1094E00000000000656E61626C650000697000003C
:1094F0001FB500200190029003900DA10DA007F070
:10950000CBFE0E48017881B1C17800918378407814
:1095100008B12D2200E0202209A101A8FEF790FC4D
:1095200001A90AA007F0B8FE1FBD0AA1F9E70000D3
:109530006F6B00007374617475730000F00000209D
:10954000256325642E2564204300000074656D703A
:10955000000000006D697373696E670010B507A1A4
:1095600007A007F099FE084C08A0616807F06AFEA2
:109570002168BDE8104006A007F064BE6F6B0000D4
:1095800073746174757300002400002076657200A6
:10959000737562566572000010B508A108A007F047
:1095A0007BFE094C2068017808A007F04BFE20687C
:1095B0004168BDE8104007A007F06EBE6F6B000069
:1095C0007374617475730000040000207479706511
:1095D000000000006E616D65000000002DE9F0479D
:1095E000ADF5267D8246142196A8F6F716FF2421B4
:1095F0008DA8F6F712FF24219BA8F6F70EFF002690
:10960000A596A496052396AA63A15046009607F056
:109610009DFA01287DD196A8F6F726FF002878D07C
:109620008DAF5FA3A4AA5CA15FA000971DF04AF8CC
:109630000546022824D15F4CC11E20681CF06EFD37
:10964000122259A101A804F0D9F9002812D15AA177
:1096500001A804F0FDFA62A101A804F0F9FA63A1DF
:1096600001A804F0F5FA71A101A804F0F1FA01A82B
:1096700003F020FD00231A46194620681CF0C8FBA1
:10968000DFF8B491002422466CA1A4A8FEF7D8FB11
:10969000002D5CD042A3A4AA3FA143A000971DF0D7
:1096A00011F8002853D18DA8F6F7DEFEC4EBC402F2
:1096B00009EBC20810F0FF0088F8110047D08DA810
:1096C000F6F7D2FE024640468DA9F6F77FFE4046E9
:1096D00098F8112096A9F6F7DCFEC0BB05239BAADB
:1096E00058A15046009607F031FA01282FD158A30F
:1096F000A4AA29A12CA000971CF0E4FF38BB8DA8D8
:10970000F6F7B2FE5449C0B20978491E014207D1AA
:1097100000E020E008F112002121F6F77EFE06E0CD
:1097200028B108F1120021228DA9F6F74FFE08F1A9
:10973000120021229BA9F6F7ACFEC0B1DAF81000A6
:1097400006F042FB024696A94448FEF729FC641C39
:1097500014F0FF0497D042A143A007F09DFD44A15F
:109760003FA007F099FD0DF5267DBDE8F08746483E
:109770009BA9026896A80EF00FF944A13AA007F041
:109780008BFDDAF8100006F01FFB024696A940A0F8
:10979000FEF706FCE7E70000757365720000000045
:1097A0006E616D65000000006C6F67696E2E786DEC
:1097B0006C000000080000203C3F786D6C2076654E
:1097C0007273696F6E3D22312E302220656E636F99
:1097D00064696E673D225554462D38223F3E0A008B
:1097E0003C75736572733E0A00000000093C757396
:1097F00065722069643D223022206E616D653D22D4
:1098000061646D696E2220706173733D2222207045
:1098100065726D697373696F6E733D2232313437CF
:10982000343833363437222F3E0A00003C2F75730C
:109830006572733E0A0000002816001069643D221C
:109840002564220070617373776F726400000000FA
:10985000706173730000000002000020549A040835
:109860006572726F7200000073746174757300002A
:10987000696E636F7272656374206C6F67696E20C6
:10988000617474656D707400680000206F6B000077
:10989000417574656E74696669636174696F6E2081
:1098A0007375636365737366756C6C7920666F722C
:1098B00020222573222E2052656D6F7574652069F4
:1098C000703A25733B0A000070B50EA10EA007F098
:1098D000E3FC0FA007F09AFC00240F4E0F4D09E0A7
:1098E00004EB440006EB801090F84C0007F02EFCCF
:1098F000641CE4B26878A042F2D8BDE8704007F07A
:1099000069BC00006F6B00007374617475730000B4
:10991000616C61726D730000F4020020640000202D
:109920007CB50021ADF804100091032301AAB7A172
:1099300007F00CF901287CD1BDF80400032878D881
:10994000B4A1B5A007F0A8FCBDF80410AFA007F0C3
:1099500079FCBDF80400B24C00EB400004EB801031
:1099600090F84D10AFA007F06DFCB0A007F04EFCD2
:10997000BDF8040000EB400004EB801090F85E009E
:1099800007F0E4FBBDF8040000EB400004EB80109E
:1099900090F8600007F0DAFB07F01CFCBDF804004B
:1099A00000EB400004EB801090F85F0000EB8000BB
:1099B0008100A0A007F046FCA0A007F027FC00262D
:1099C00007F0A8FBBDF8040006EB860100EB4000A1
:1099D00004EB801001EBC60500EB450090F8620037
:1099E00007F0A6FBBDF8040000EB400004EB80107C
:1099F00000EB450090F8630007F0A8FBBDF80400F9
:109A000000EB400004EB801000EB450090F8640090
:109A100007F09CFBBDF8040000EB400004EB801055
:109A200000EB4500B0F8660007F090FBBDF80400BD
:109A300000E0E2E000EB400004EB801000EB4500AA
:109A4000B0F8680007F082FBBDF8040000EB4000AE
:109A500004EB801000EB4500B0F96A0007F076FBDC
:109A6000BDF8040000EB400004EB801000EB450063
:109A7000B0F96C0007F06AFBBDF8040000EB400091
:109A800004EB801000EB4500B0F86E0007F05EFBC1
:109A9000BDF8040000EB400004EB801000EB450033
:109AA000B0F8700007F052FBBDF8040000EB400076
:109AB00004EB801000EB4500B0F8720007F046FBA5
:109AC000BDF8040000EB400004EB801000EB450003
:109AD000B0F8740007F03AFBBDF8040000EB40005A
:109AE00004EB801000EB4500B0F87A0007F02EFB85
:109AF000BDF8040000EB400004EB801000EB4500D3
:109B000090F8760007F022FBBDF8040000EB40005F
:109B100004EB801000EB450090F9770007F016FB8E
:109B2000BDF8040000EB400004EB801000EB4500A2
:109B300090F8780007F00AFB07F04CFB761CF6B2B1
:109B4000032EFFF43DAF07F045FB3DA007F05EFBA1
:109B50005FF0000507F0DEFABDF8040000EB4000FE
:109B600004EB801000EBC50090F8B00007F0E0FABD
:109B7000BDF8040000EB400004EB801000EBC500D2
:109B800090F8B10007F0E2FABDF8040000EB4000E5
:109B900004EB801000EBC50090F8B20007F0D6FA95
:109BA000BDF8040000EB400004EB801000EBC500A2
:109BB00090F8B30007F0CAFABDF8040000EB4000CB
:109BC00004EB801000EBC50090F8B40007F0BEFA7B
:109BD000BDF8040000EB400004EB801000EBC50072
:109BE000B0F8B60007F0B2FA07F0F4FA6D1CEDB267
:109BF000022DAFD307F0EEFA7CBD13A106A007F04B
:109C00004BFB13A110A007F047FB7CBD756E697478
:109C1000000000006F6B00007374617475730000C6
:109C2000F4020020766572730000000066696C74AF
:109C300065720000706F7765720000004846000092
:109C4000707772416D7000006572726F7200000073
:109C5000696E76616C696420706172616D657472A1
:109C6000000000007CB5054600248DF804400BA1DF
:109C70000BA007F011FB022301AA0BA128460094B8
:109C800006F064FF0A49012804D0097806A007F00D
:109C9000CBFA7CBD9DF8040008707CBD6F6B0000A2
:109CA0007374617475730000656E61626C650000A9
:109CB000640000202DE9F04115A116A007F0ECFA90
:109CC00016A007F0A3FA174D687807F03FFA0024B2
:109CD000154E164F14E000BF07F01CFA04EB4400C9
:109CE00006EB801007F04AFA04EB840000EB441006
:109CF00007EB800007F042FA07F06CFA641CE4B24C
:109D00006878A042E8D8BDE8F04107F063BA0000E7
:109D10006F6B000073746174757300006C69737409
:109D20000000000064000020F4020020700C00100D
:109D30007CB50021ADF804100091032301AA48A1CD
:109D400006F004FF01287DD1BDF8040003287DD86A
:109D500045A146A007F0A0FABDF80400454D00EB70
:109D6000400005EB801090F8411043A007F05CFA2A
:109D7000BDF8040000EB400005EB801140A007F0A7
:109D80008BFABDF8040000EB400005EB801090F862
:109D900042103DA007F056FABDF804003D4C00EB20
:109DA000800101EB401004EB80013BA007F074FA46
:109DB000BDF8040000EB800101EB401004EB8001D2
:109DC00036A0103107F068FABDF8040000EB8001FE
:109DD00001EB401004EB800131A0203107F05CFA68
:109DE00030A007F013FABDF8040000EB400005EBCB
:109DF000801090F85E0007F0A9F9BDF8040000EBB0
:109E0000400005EB801090F8600007F09FF907F024
:109E1000E1F9BDF80400002817D024A007F0F6F9F6
:109E20005FF00004BDF8040000EB400005EB80107B
:109E3000204490F8430007F089F9641CE4B2092C2F
:109E4000F0D300E002E007F0C5F97CBD19A107A03E
:109E500007F022FA19A117A007F01EFA7CBD000036
:109E6000756E6974000000006F6B0000737461749C
:109E700075730000F4020020656E61626C6500007D
:109E80006E616D650000000074696D65506F6C6CEB
:109E900000000000700C0010697000006E6D000082
:109EA0006777000066696C7465720000726F757484
:109EB000650000006572726F72000000696E766165
:109EC0006C696420706172616D65747200000000DD
:109ED0002DE9FC470026ADF80460032301AA3DA14B
:109EE000009606F033FE012814D1BDF804000328C3
:109EF00010D878B1394CDFF8E8A0DFF8E890617845
:109F0000A070091A491E11F0FF074FF0010846D052
:109F1000002541E034A136A007F0BEF936A132A0F9
:109F200054E000BFBDF80400C02200EB40010AEB82
:109F3000811000F1C001F6F749FABDF8040000EB0A
:109F4000800101EB401109EB810000F1940100F167
:109F5000100E91E80E1080E80E1000F1A40191E8B7
:109F60000E108EE80E1000F1B40100F1200E91E801
:109F70000E108EE80E10FAF789FBBDF8040000EB16
:109F800040020AEB8211401C81F8016181F80C81CA
:109F90006D1CADF80400EDB2BD42C3D307E000EB89
:109FA00040010AEB811080F8416080F84C806078B5
:109FB000401EC0B200EB8001607001EB401109EB64
:109FC000810030300AF046FE10A109A007F064F9C4
:109FD000BDE8FC87756E6974000000006400002015
:109FE000F4020020700C00106572726F72000000A5
:109FF0007374617475730000696E76616C696420B6
:10A00000706172616D657472000000006F6B00001A
:10A010002DE9F04186B000248046ADF808408DF867
:10A020000440032302AA71A1009406F08FFD0128C9
:10A030007ED1BDF8080003287AD86EA16EA007F083
:10A040002BF9BDF808006E4D00EB400005EB8010C9
:10A05000012680F84160032301AA6AA140460094CA
:10A0600006F074FDBDF80800052300EB400005EB89
:10A07000801267A182F84C609DF8040082F84200CB
:10A080004046009406F062FDBDF80800002867D045
:10A090000623002260A14046009406F057FD0027E9
:10A0A00003233A4601A94046009606F0CFFCBDF8CE
:10A0B000080000EB400005EB8012D1199DF8040068
:10A0C00091F84330834203D081F8430082F8406026
:10A0D0007F1CFFB2092FE3D3BDF80800504F00EBFF
:10A0E000800101EB401007EB8002009405234DA195
:10A0F000404606F02BFDBDF80800009400EB8001FF
:10A1000001EB401007EB8002052347A140461032C7
:10A1100006F01CFDBDF80800052300EB800101EBF3
:10A12000401007EB8002009440A14046203200E03E
:10A1300053E006F00BFDBDF8080000EB800101EBD9
:10A14000401007EB8000FAF7A1FABDF8080000EB19
:10A15000800101EB401007EB800030300AF0DCFD9D
:10A160000623002232A14046009406F0EFFC0323B0
:10A17000002201A94046009606F068FCBDF80810D0
:10A180009DF8040001EB410105EB8111032381F8E7
:10A190005E00012201A94046009606F057FCBDF87A
:10A1A00008109DF8040001EB410105EB811181F8D5
:10A1B0006000214901204E7000EB400205EB821245
:10A1C00092F8412012B14A78521C4A70401CC0B229
:10A1D0000428F1D306B0BDE8F08118A106A007F06D
:10A1E0005BF818A115A007F057F8F3E7756E6974CE
:10A1F000000000006F6B00007374617475730000E1
:10A20000F402002074696D65506F6C6C00000000F2
:10A210006E616D6500000000726F7574650000006E
:10A22000700C0010697000006E6D00006777000010
:10A2300066696C7465720000640000206572726F5C
:10A2400072000000696E76616C69642070617261F1
:10A250006D657472000000001BF00EFA4FF4FA7086
:10A26000F7F71CFBBFF34F8F05480168054A01F45F
:10A27000E06111430160BFF34F8F00BFFDE70000B5
:10A280000CED00E00400FA052DE9F041754FADF545
:10A29000147D4FF0FF3138681BF040FF122272A18D
:10A2A00007A803F0ABFB30B172A174A006F0F4FF75
:10A2B00074A170A0C3E076A107A803F0C9FC7EA139
:10A2C00007A803F0C5FC7FA107A803F0C1FC7F4AE3
:10A2D0007FA107A803F0BCFC7C4A81A1103207A82B
:10A2E00003F0B6FC794A85A1203207A803F0B0FC40
:10A2F000002010F0CBFD006848B1002010F0C6FD32
:10A3000005F062FD024684A107A803F0A1FC87A125
:10A3100007A803F09DFC88A107A803F099FC0EF0A4
:10A32000D9F802468AA107A803F092FC00200EF09B
:10A33000A7FB02468EA107A803F08AFC00200EF0BE
:10A34000DBF8024693A107A803F082FC0EF0C8F8E0
:10A3500002469AA107A803F07BFCA2A107A803F07C
:10A3600077FCA34EA3A107A8727803F071FC002527
:10A37000DFF8948253E000BF05EB450108EB811440
:10A3800023462A46A1A107A803F062FC14F8422F35
:10A39000A6A107A803F05CFCA37F227FA8A107A8C1
:10A3A000423C03F055FC002D33D094F848000DF1E9
:10A3B0000C0C94F84B3094F84A2094F849108CE82F
:10A3C0000F0094F8450094F8472094F846108DE863
:10A3D000070094F8443094F84320A0A107A803F0A4
:10A3E00037FC05EB850000EB4511384800EB810494
:10A3F0002246A6A107A803F02BFC04F11002A7A196
:10A4000007A803F025FC04F12002ABA107A803F084
:10A410001FFCB0A107A803F01BFC6D1CEDB2707807
:10A42000A842A9D8AEA107A803F012FCAFA107A8C3
:10A4300003F00EFC07A802F03DFEAFA10FA006F04E
:10A440002BFFAEA003F093FEACA107A003F0A4FD88
:10A4500000231A46194638681BF0DAFC0DF5147D06
:10A46000BDE8F0810800002054636F6E6669672EB6
:10A47000786D6C006572726F7200000073746174A5
:10A480007573000073617665206661696C656400B0
:10A490003C3F786D6C2076657273696F6E3D22313A
:10A4A0002E302220656E636F64696E673D225554BD
:10A4B000462D38223F3E0A003C636F6E6669673E58
:10A4C0000A000000093C6E65743E0A00700C001022
:10A4D00009093C69703E25733C2F69703E0A0000F3
:10A4E00009093C6E65746D61736B3E25733C2F6E7C
:10A4F00065746D61736B3E0A0000000009093C67DA
:10A500006174657761793E25733C2F676174657767
:10A5100061793E0A0000000009093C6E74703E2516
:10A52000733C2F6E74703E0A00000000093C2F6ED1
:10A5300065743E0A00000000093C736E6D70207661
:10A54000657273696F6E3D223263223E0A0000001D
:10A5500009093C636F6D6D756E6974793E25733CB6
:10A560002F636F6D6D756E6974793E0A000000008F
:10A5700009093C747261702D656E61626C653E25DF
:10A58000643C2F747261702D656E61626C653E0A69
:10A59000000000000909093C747261702D686F7336
:10A5A000746E616D653E25733C2F747261702D6809
:10A5B0006F73746E616D653E0A00000009093C749A
:10A5C0007261702D636F6D6D756E6974793E257360
:10A5D0003C2F747261702D636F6D6D756E69747947
:10A5E0003E0A0000093C2F736E6D703E0A000000A9
:10A5F00064000020093C626C6F636B73206E756DA4
:10A600003D222564223E0A00F402002009093C6232
:10A610006C6F636B2069643D22256422206E616D3E
:10A62000653D222573223E0A000000000909093C0D
:10A63000706F6C6C3E25643C2F706F6C6C3E0A0032
:10A640000909093C66696C7465723E25642C2564B1
:10A650003C2F66696C7465723E0A00000909093C6A
:10A66000726F7574653E25642C25642C25642C2539
:10A67000642C25642C25642C25642C25642C2564ED
:10A680003C2F726F7574653E0A0000000909093C91
:10A6900069703E25733C2F69703E0A000909093C28
:10A6A0006E65746D61736B3E25733C2F6E65746DC2
:10A6B00061736B3E0A0000000909093C676174651B
:10A6C0007761793E25733C2F676174657761793EC8
:10A6D0000A00000009093C2F626C6F636B3E0A00A0
:10A6E000093C2F626C6F636B733E0A003C2F636FF3
:10A6F0006E6669673E0A00006F6B0000636F6E66EE
:10A7000069672E786D6C000000B587B0002101915B
:10A710000291039104910091052301AA13A106F06F
:10A7200015FA012806D012A113A006F0B5FD14A158
:10A730000FA016E010F0E8FD01A8F5F795FE50B166
:10A7400005A901A805F07AFA05A9002010F0CAFDB4
:10A7500010F0AEFB03E00021084610F0C3FD0DA190
:10A7600005A006F099FD07B000BD0000697000006B
:10A770006572726F7200000073746174757300000B
:10A78000696E76616C696420706172616D65747266
:10A79000000000006F6B000038B50546002002463F
:10A7A0000090072318A1284606F0D0F9012809D007
:10A7B00016A118A006F070FD18A114A0BDE838403D
:10A7C00006F06ABD01240523194A1AA128460094FF
:10A7D00006F0BCF9164A0523103217A1284600944A
:10A7E00006F0B4F9124A0523203215A12846009438
:10A7F00006F0ACF90E48F9F749FF0D4911A0FDF735
:10A80000CFFB17A103A0D9E76E6574006572726F64
:10A81000720000007374617475730000696E766174
:10A820006C696420706172616D657465720000000E
:10A83000700C0010697000006D61736B0000000007
:10A84000677700006368616E67696E672049502012
:10A850006164647265737320746F20257300000057
:10A860006F6B000000B585B000210091032304AA9E
:10A870000DA106F06BF9012809D00DA10EA006F07C
:10A880000BFD0FA10AA006F007FD05B000BD11A148
:10A8900009A006F001FD01A8049919F059F801A8D2
:10A8A000FAF7E8FBF1E7000074696D65000000004D
:10A8B0006572726F720000007374617475730000CA
:10A8C000696E76616C696420706172616D65747225
:10A8D000000000006F6B00001CB5002100910323F5
:10A8E00001AA0CA106F032F9012808D00BA10DA095
:10A8F00006F0D2FC0DA109A006F0CEFC1CBD10A1F3
:10A9000008A006F0C9FC9DF904100E48FAF794FB64
:10A910001CBD0000636F7272000000006572726FF0
:10A92000720000007374617475730000696E766163
:10A930006C696420706172616D6574720000000062
:10A940006F6B00001C16001070B58AB0002506461B
:10A95000FF2006958DF808002C4603950495059573
:10A960008DF80450284610F07FF8002010F083F88E
:10A97000032302AA3DA13046009406F0E7F801281F
:10A9800069D19DF8080010B1012804D006E001202B
:10A9900010F06AF802E0012010F06DF80523354A46
:10A9A00035A13046009406F0D1F801280ED1314887
:10A9B000F5F75AFD05460DF08DFD2A462D49F5F7B0
:10A9C0007EFD10B12B480FF0A3FB012507230022C9
:10A9D0002CA13046009406F0B9F8012804D0002DCF
:10A9E00039D02AA12AA03CE00124022301AA2AA1ED
:10A9F0003046009406F0AAF8052303AA28A13046A1
:10AA0000009406F0A3F80523264A1BA130460094C3
:10AA100006F09CF82348F5F727FD04460DF060FD8D
:10AA200022462049F5F74BFD10B11E480FF0C4FB3C
:10AA30009DF80400012804D0002100200FF010FE32
:10AA4000CFE708A903A805F0F9F808A900200FF03E
:10AA50000FFE0121F1E714A10DA006F01DFC14A1C9
:10AA600011A006F019FC0AB070BD00007665727383
:10AA7000696F6E003C000010636F6D6D756E6974D8
:10AA80007900000074726170000000006F6B0000BC
:10AA90007374617475730000656E61626C650000AB
:10AAA000697000004C0000106572726F7200000047
:10AAB000696E76616C696420706172616D65746540
:10AAC000720000002DE9F05F82460C4601F11A0089
:10AAD00006F09FFC78BB2078012700F03F00401E65
:10AAE00000EB8001DFF8589001EBC00500264FF61F
:10AAF000FF7B00BF19F80600204406F08AFC804660
:10AB00006FB1FF2D17D203F0BBFC07463AF81500D2
:10AB10006D1C03F0B5FC87420DD1474601E0D845D6
:10AB200009D1761C0D2EE5D32078400606D52FB12D
:10AB30003AF8150010B10020BDE8F09F0120FBE7B6
:10AB4000F47D0408002000F0C1B82DE9F047164656
:10AB5000894604004FF0000702D0B9F1000F00D180
:10AB6000377000254FF004080FE0A16805EB4500A1
:10AB700008EB40028A5A31F8100021680144484627
:10AB8000F5F787FC28B16D1CADB2A089A842ECD8BE
:10AB90001FE0A26805EB45080A2101EB4805505B60
:10ABA000B8B13046F5F760FC01463046F5F735FCA4
:10ABB000A068062303EB4801425B405A2168014428
:10ABC0003046F5F703FCA0682168405B0F54BDE8F0
:10ABD000F0873770FBE770B5002843D0002211469C
:10ABE000022333E00468645C202C0ED03B2C13D08D
:10ABF0003D2C01D0D1B11EE002EB42064C1E85680F
:10AC000003EB4606521CAC5392B2856802EB420637
:10AC10004C1C25F8164017E002EB42064C1E8568D6
:10AC200003EB4606521CAC5392B20DE0846802EB73
:10AC3000420524F81510866802EB4205042404EB53
:10AC40004504355B6D1C3553491C89B284888C42A0
:10AC5000C8D802EB42058468491E03EB4503E15264
:10AC6000521C828170BD000030B504460D4608A01C
:10AC700000F038F8204600F035F83D2000F026F8C6
:10AC8000284600F02FF8BDE8304005A000F02AB8B3
:10AC90005365742D436F6F6B69653A2000000000A7
:10ACA0003B20706174683D2F3B2053616D65536993
:10ACB00074653D5374726963740D0A00024AC2E9F7
:10ACC00000010020906070476016001004490A6877
:10ACD00010700868401C08608868401C88607047D5
:10ACE0006016001000B5034602E05B1CFFF7EEFFA4
:10ACF00018780028F9D100BD2DE9F04105680F0052
:10AD0000804606D003F0EAFD022809D20120BDE802
:10AD1000F0816E6916B1286AB04207D8012605E0B5
:10AD2000411CF4D0296A8142F1D83E463446286A53
:10AD3000641CA04202D80224022E0AD321464046B7
:10AD400003F0CCFD38B10128E1D0411CDFD0B44282
:10AD5000EDD10020DBE74FF0FF3632462146284692
:10AD60000CF0A8F830B957B12246394628460CF005
:10AD7000A1F820B101280FD001242046C7E76C615B
:10AD8000296AA869891E884201D8401EA8612879CD
:10AD900040F001002871F0E73446EEE72DE9F84F66
:10ADA000804600680E680024C76889462546705DA5
:10ADB0006D1C20281AD32F2813D05C2811D0FF2C0B
:10ADC00057D2012103F01EFB5FEA000A51D0BAF10D
:10ADD000800F12D201467CA0FEF738F990BB0CE040
:10ADE0006D1C715D2F29FBD05C29F9D07219C9F84F
:10ADF0000020202805D2042504E027F814A0641CB4
:10AE0000D5E700250021012C04D0022C24D178881C
:10AE10002E2818D138882E2815D127F81410002094
:10AE2000A04201D22E2200E0202208EB0001401CAB
:10AE300081F824200B28F3D3404445F0200280F809
:10AE40002420BEE015E007EB440030F8020C202877
:10AE500001D02E2802D1641E002CF4D127F8141042
:10AE60003CB10B22202108F1240008F0A3F80026B1
:10AE700003E00620BDE8F88F761C37F8160020287E
:10AE8000FAD02E28F8D01EB145F0030500E0641E6C
:10AE90002CB107EB440030F8020C2E28F7D14FF00C
:10AEA000000A4FF0080BCDF800A000BF37F81600DD
:10AEB00006F101065FEA000924D0B9F1200F04D0A1
:10AEC000B9F12E0F04D1A64202D045F00305EDE7FB
:10AED0000098584501D2A64219D1BBF10B0F0FD0F3
:10AEE000A64201D045F003050CD84FF008000090B1
:10AEF0004FEA8A6026464FF00B0B4FEA106AD5E7FF
:10AF000045F0030598F82400E52838D03AE0484693
:10AF1000B9F1800F10D3002103F074FA5FEA000941
:10AF200005D02C4901EB090010F8800C814645F052
:10AF30000205B9F1000F04D0014627A0FEF786F8FC
:10AF400020B14FF05F0945F003050FE0A9F1410082
:10AF5000192802D84AF0020A08E0A9F1610019286C
:10AF600004D841304AF0010A1FFA80F9009A08EB30
:10AF7000020181F824900098401C009096E705217A
:10AF800088F82410BBF1080F03D14FEA8A604FEA1A
:10AF9000106ACAF38100032803D06FEA0A01890707
:10AFA00001D145F00205A90709D40AF003010129DE
:10AFB00001D145F01005012801D145F0080588F8B8
:10AFC0002F50002056E70000222A3A3C3E3F7C7F6B
:10AFD00000000000747D04082B2C3B3D5B5D0000ED
:10AFE00010B5144888B0817A8A0601D512A200E013
:10AFF00013A2CB0601D510A300E011A30C0701D5C5
:10B000000DA400E00EA4C90701D00BA100E00CA123
:10B01000CDE90414CDE906328188C479037A427AF5
:10B020008DE81E00C378827807490120FCF742FFB3
:10B0300008B010BD1C160010747275650000000089
:10B0400066616C7365000000989A04080EB5154996
:10B05000062805D020B101228240086842400A60DB
:10B060000868810601D510A100E010A1C20601D533
:10B070000DA200E00DA2030701D50BA300E00BA376
:10B080000093CDE90121410701D507A300E007A303
:10B09000800701D504A200E004A205490120FCF7C5
:10B0A00009FF0EBD740000206F6E00006F66660021
:10B0B000149B04080848016841F480710160074945
:10B0C0000A6842F001020A60016821F4807101609F
:10B0D000012000F047B900000070004050280040F7
:10B0E00010B508A30AA20DA10120FCF7E3FE1A4C3B
:10B0F00004E01AA10120FCF7DDFE0C342268002ACE
:10B10000F7D110BD31323A32353A33380000000001
:10B110004A616E2031392032303232005F5F5F5F2A
:10B120005F5F5F5F5F5F5F5F5F5F5F5F5F5F5F5F2F
:10B130005F5F0A0D436F6D70696C65643A2025731B
:10B140002025730A0D5F5F5F636F6D6D616E6473C1
:10B150003A5F5F5F0A0D00008400002025730A0D2E
:10B1600000000000F0B5ADF5017D4FF4007101A8BD
:10B17000F5F753F9284B01AC20461F46A3F1100206
:10B1800026A1FCF75DFE244D0646103D95F85900BA
:10B19000C00701D02BA200E02BA2A0192CA1FCF724
:10B1A0004FFE064495F85700009095F8563095F8F4
:10B1B0005520A0192FA15035FCF742FE164A06442F
:10B1C000A0193B46103A3AA1FCF73AFE0644687AC9
:10B1D0002B88C00701D042A200E042A2A01943A1DF
:10B1E000FCF72EFE85194F4ED6F8C421D6F89431BF
:10B1F00060194DA106F5B476FCF722FE32682844AA
:10B20000204451A1FCF71CFE01AA54A10120FCF727
:10B2100051FE0DF5017DF0BD800C00100D0A2320BC
:10B220006966636F6E666967206574683020696E51
:10B230006574202573206E65746D61736B202573B2
:10B240000D0A000075700000646F776E000000004A
:10B2500023206966636F6E666967206574683020B5
:10B2600025730D0A23206966636F6E6669670D0A90
:10B270000000000065746830094C696E6B20656ED3
:10B280006361703A45746865726E65742020485732
:10B29000616464722030323A41443A43383A25308E
:10B2A00032583A253032583A25303258200D0A00AB
:10B2B00009696E657420616464723A2573202042C6
:10B2C000636173743A3139322E3136382E302E3272
:10B2D000353520204D61736B3A2573200D0A00002F
:10B2E00055500000444F574E0000000009257320C0
:10B2F00042524F4144434153542052554E4E494EC1
:10B3000047204D554C54494341535420204D5455EA
:10B310003A256420204D65747269633A31200D0A24
:10B320000000000000800240095258207061636BE9
:10B330006574733A2564206572726F72732043528C
:10B34000433A25640D0A0000095458207061636B6C
:10B350006574733A25640D0A230D0A0025730000F5
:10B360007047000010B5012807D002281AD0BDE8A8
:10B37000104019A10120FCF79DBD26A10120FCF77A
:10B3800099FD4FF4FA701AF04DFBBFF34F8F25482B
:10B390000168254A01F4E06111430160BFF34F8F5A
:10B3A00000BFFDE721A10120FCF784FD234C002212
:10B3B00040212046F6F76BFF322009F010FD0122F4
:10B3C00040212046F6F763FFBDE810404FF4A0622D
:10B3D0001B211B48F6F7E8BD434D443A5265626FA6
:10B3E0006F740D0A090909090931202D205265627F
:10B3F0006F6F7420532D506F72740D0A090909097B
:10B400000932202D205265626F6F74205048590D0B
:10B410000A0000005265626F6F7420532D506F72E6
:10B42000740D0A000CED00E00400FA055265626F2D
:10B430006F74205048590D0A0000000000000240BF
:10B44000CC6800207CB5002001906A4601A917A0B5
:10B4500001F048FE16A10120019AFCF72BFD00988F
:10B4600018A1026A0120FCF725FD00981AA1428963
:10B470000120FCF71FFD00981CA1046A4089A41E4E
:10B48000444322460120FCF715FD00981CA1458984
:10B49000019845432A460120FCF70CFD63086A0821
:10B4A0001CA10120FCF706FD7CBD00002F00000060
:10B4B0006672655F636C7573743A20256C75200D38
:10B4C0000A0000006E5F666174656E743A20256C38
:10B4D00075200D0A0000000066735F6373697A656A
:10B4E0003A20256C75200D0A00000000746F745F0F
:10B4F000736563743A20256C75200D0A0000000006
:10B500006672655F736563743A20256C75200D0A59
:10B5100000000000256C75204B4220746F74616C34
:10B520002064726976652073706163652E200D0A50
:10B53000256C75204B4220617661696C61626C6597
:10B540002E0D0A00F8B5064600200D460446074FAA
:10B55000009006E0311900236A46F8681AF0D4FC1E
:10B56000641C2868A042F5D8F8BD000074000020D3
:10B5700070B50A480025D0F8BC4264B140F2F51617
:10B58000D4F8140200284FF0010005D009F027FC80
:10B590006D1CB542F4D1002070BD0000D82A001007
:10B5A000401E022812D20A4901EB00118889B0F529
:10B5B000807F05D008B1401E80B2888110B103E0C1
:10B5C0000020FAE700200860002070470220704742
:10B5D000A82F00102DE9F04704460021D0F8009074
:10B5E00000F04FFA00285BD1FF25471EA8462763CD
:10B5F0004846E16907F0EBFE060050D1216A087861
:10B6000050B1CA7AE52802F03F02A2713FD0130779
:10B6100004D50F2A3BD105E0042640E00F2A01D0D3
:10B62000E5B120E094F82F20520632D4420606D528
:10B6300091F80D8000F0BF00626905462263A842C0
:10B6400009D14A7B424506D1D9F80C00FFF73AFAF6
:10B6500008B16D1E00E0FF25EDB21AE008460FF0BC
:10B66000FEFE40451BD094F82F00C0070FD1D4F840
:10B67000201004F124000B2211F8013B10F8015BAB
:10B680005B1B521E02D0002BF6D000E03BB1FF2521
:10B6900027630021204600F005F80600A8D03046B8
:10B6A000BDE8F0872DE9F047054647690468C069A1
:10B6B0008946203710B1B7F5001F02D30420BDE83A
:10B6C000F087F90560D1401CE861A9694FF00008D6
:10B6D00029B16089401E10EA572F05D054E0208917
:10B6E000B0EB571F1DD94FE0284603F0F7F8064688
:10B6F00001281BD9701C33D0206AB0423ED8B9F162
:10B70000000F0ED02846A969FFF7F6FA06000BD005
:10B71000012E0BD0701C23D020460FF0F1FEF8B99B
:10B7200006E0C5F81C80C9E70720C8E70220C6E785
:10B730004FF40072002104F13C0007F03BFC4FF095
:10B74000000831462046FDF707FD4FF00109A063D0
:10B750000DE000BF84F8039020460FF0D1FE08B141
:10B760000120ACE7A06B08F10108401CA0636189CF
:10B770004145EFD8A16BA1EB0800A06331462046FC
:10B78000AE61FDF7E9FCE861C7F3080020443C30F6
:10B790006F612862002092E72DE9F0470426FF241C
:10B7A000894605462746D0F8008047E0404607F026
:10B7B0000EFE060046D1296A087880B1CA7AE528CB
:10B7C00002F03F02AA7108D02E2806D022F02003F2
:10B7D000082B06D0B446CC4506D0FF241EE0042634
:10B7E00030E04FF0010CF6E70F2A01D014BB1CE04B
:10B7F000420605D54F7B00F0BF006A6904462A6304
:10B80000A04209D1487BB84206D1D8F80C000AF012
:10B81000C3FD08B1641E00E0FF24E4B20021284605
:10B82000FFF740FF060009D00CE008460FF017FEB6
:10B83000B84209D04FF0FF30286305E0E9690029DC
:10B84000B4D10EB10020E8613046BDE8F0870000B9
:10B850002DE9F04F0446D0F8009090F82F0089B001
:10B8600010F0A00F03D0062009B0BDE8F08F00252E
:10B87000D9F80C0000E06D1C30F815100029FAD141
:10B8800004F124010C226846039107F0DFF89DF8CB
:10B890000B00C00719D0402084F82F000126334642
:10B8A0006946D9F80C20039802F0D8FF2046FFF72C
:10B8B00091FE10B9761C642EF1D3642E0FD00428AB
:10B8C000D2D19DF80B0084F82F009DF80B00800763
:10B8D00007D50D200C35B5FBF0F56D1C02E00720F7
:10B8E000C2E7012500212046276800F0CAF888B980
:10B8F00000263846E16907F06AFD58B9206A0078E9
:10B90000E5280AD048B1002601212046FFF7CAFEEB
:10B910000028EED0042812D012E0761C2846AE4251
:10B92000F2D1451E059567D06169684201EB40116F
:10B93000204600F0A6F85FEA000803D076E0072072
:10B94000804673E003980FF08AFD4FF6FF7B079067
:10B950004846E16907F03BFD5FEA000866D1D9F887
:10B960000C0006900598D4F82080C0B20490079986
:10B9700088F80D100F2188F80B10002188F80C10A2
:10B9800008F11A000FF014FD0498DFF8A4A0401E7F
:10B9900000EB800101EBC006002701E05D4503D00C
:10B9A000069830F81650761C1AF8071001EB0800BC
:10B9B00029460FF0FDFC05B95D467F1C0D2FEDD328
:10B9C0005D4505D0069830F8160008B1049803E0EC
:10B9D000049840F04000049088F80000012189F8A4
:10B9E000031000212046FFF75DFE5FEA00081DD12D
:10B9F0000598401E0590ABD14846E16907F0E7FC89
:10BA00005FEA000812D120220021206A07F0D2FA52
:10BA10000B22206A039907F019F894F82F00216A85
:10BA200000F018000873012089F8030040461BE766
:10BA3000F47D04082DE9F041016B04464669056870
:10BA4000481C04D0204600F01CF8002817D1E52738
:10BA50004FF001082846E16907F0B9FC60B9216A96
:10BA60000F7085F803806169B14208D20021204639
:10BA7000FFF718FE0028EDD0042800D10220BDE811
:10BA8000F0812DE9F04107680E460546B1F5001F2B
:10BA900036D2F00634D16E61AC6824B93878032808
:10BAA00005D33C6B1CB178894FEA402812E03889F5
:10BAB000B0EB561F24D9386B12E0284602F00EFF77
:10BAC0000446401C1AD0022C1AD3386AA04217D957
:10BAD000A6EB080646452146EFD23846FDF73CFB6B
:10BAE000C5E9064060B100EB5620E861C6F30800E6
:10BAF00038443C3028620020BDE8F0810120FBE79B
:10BB00000220F9E7084910B50B5C002253B9012265
:10BB10000A540A1801EB8000127A40680168104646
:10BB200088470246104610BD1469002030B4054C09
:10BB3000231804EB80001B7A406804691846A44669
:10BB400030BC60471469002030B4054D2C1805EB5B
:10BB50008000247A406885682046AC4630BC604747
:10BB600014690020044A111802EB8000097A406829
:10BB700042680846104700001469002030B4054DA3
:10BB80002C1805EB8000247A4068C5682046AC4636
:10BB900030BC60471469002070B505460C46880724
:10BBA00006D00BA34FF4B67215A11DA0FCF738F90F
:10BBB0000FF002FD2A689188491E9180E9680968A2
:10BBC0002160E9680C60BDE870400FF01DBD000009
:10BBD0002E2E2F4D6964646C6577617265732F54E6
:10BBE000686972645F50617274792F4C7749502F85
:10BBF0007372632F636F72652F6D656D702E6300B6
:10BC00006D656D705F667265653A206D656D20705B
:10BC1000726F7065726C7920616C69676E65640023
:10BC2000417373657274696F6E20222573222066DA
:10BC300061696C6564206174206C696E652025649F
:10BC400020696E2025730A0070B505460FF0B4FC1C
:10BC50000646E8680468002C19D021680160A00736
:10BC600006D00FA34FF48C7219A122A0FCF7D8F8CC
:10BC700028688188491C89B281802868C2889142DD
:10BC800000D9C18030460FF0BFFC204670BD296846
:10BC90000888401C088030460FF0B6FC002070BDBC
:10BCA0002E2E2F4D6964646C6577617265732F5415
:10BCB000686972645F50617274792F4C7749502FB4
:10BCC0007372632F636F72652F6D656D702E6300E5
:10BCD0006D656D705F6D616C6C6F633A206D656D45
:10BCE000702070726F7065726C7920616C69676E1C
:10BCF00065640000417373657274696F6E2022255C
:10BD00007322206661696C6564206174206C696EC1
:10BD10006520256420696E2025730A002DE9F0470F
:10BD200016680F468046D6E90414706849681034D6
:10BD300099461546884202D0F120BDE8F087F821E7
:10BD400004F11000F4F769FBC5F8E8402A7905F121
:10BD5000080104F114000DF02BF93069C4F80480D7
:10BD6000C4E9036027727069806830B14946204693
:10BD7000FCF7C2FF207818B125E0F120207022E006
:10BD800094F8E10085F8D10094F8E00085F8D0003F
:10BD90000E48C5F8E000D4F8E40000B10C48C5F83E
:10BDA000D400D4F8EC0000B10A48C5F8DC00D4F89F
:10BDB000E80000B10848C5F8D800227D04F1180158
:10BDC000281D0DF0F5F82078B7E7000039280408A1
:10BDD000F5270408AD280408692804082DE9F04770
:10BDE0000F46040006D141A34FF4DC724CA150A0D1
:10BDF000FCF716F80FF0E0FB00266660277294F857
:10BE0000201041F0010184F82010657866700FF071
:10BE1000FBFBA36A7BB10022042120469847A36A5A
:10BE20004BB10022114620469847A36A1BB100225D
:10BE3000022120469847384606F0DAFB804604F196
:10BE4000100081460FF064FC18B1414648460FF0DF
:10BE50004DFC04F1140081460FF05AFC18B1414624
:10BE600048460FF043FC012D0FD0042D0DD0032DBB
:10BE70000BD0606A002836D0BDE8F0471BA340F223
:10BE8000F71235A12AA0FBF7CBBF94F82010C1F31D
:10BE9000800001F0FB0184F82010002823D1606AA3
:10BEA00030B912A34FF4F37232A121A0FBF7B8FF0F
:10BEB000606A042D08D00771606A05680C35284651
:10BEC0000FF090FC10B108E00671F5E707A340F20F
:10BED000EF122FA116A0FBF7A3FF28466662BDE86C
:10BEE000F0470FF07CBCBDE8F08700002E2E2F4DF0
:10BEF0006964646C6577617265732F5468697264F4
:10BF00005F50617274792F4C7749502F7372632F91
:10BF10006170692F6170695F6D73672E6300000047
:10BF2000636F6E6E20213D204E554C4C000000008A
:10BF3000417373657274696F6E20222573222066C7
:10BF400061696C6564206174206C696E652025648C
:10BF500020696E2025730A00636F6E6E2D3E637537
:10BF60007272656E745F6D7367203D3D204E554C57
:10BF70004C000000636F6E6E2D3E63757272656ECD
:10BF8000745F6D736720213D204E554C4C000000BE
:10BF9000696E61766C6964206F705F636F6D706C41
:10BFA000657465645F73656D0000000070B5002402
:10BFB00005462046234618E034B1EC5C5E2C0CD0DC
:10BFC0005D2C0AD0002070BDEE5C7D2E03D016548F
:10BFD000401C80B207E0012405E044F02004145422
:10BFE000401C80B200245B1C9BB28B42E4D370BD2A
:10BFF00070B5094D0646002404EB440005EBC00073
:10C00000017D29B18068B04202D1204600F036F9A6
:10C01000641C0A2CF0DB70BD04BD02202DE9F74F33
:10C0200084B04FF00A0B00240646DA465F46D94634
:10C0300002940194CDF80040514904EB440001EB17
:10C04000C008039098F814500A2F1DD0002D2AD054
:10C05000012D08D0022D06D24AA340F2231257A187
:10C0600066A0FBF7DDFE9EB13168D8F8040081427E
:10C070000ED1069820B1D8F808100698814207D151
:10C08000204607B0BDE8F08F002DE1D127460AE039
:10C09000012D16D0022D06D3B8F81200009988425F
:10C0A00001D3A2460090641C24B20A2CC4DB05987C
:10C0B00081074FF0FF30E4D40A2F16D018DA3C463F
:10C0C0003EE02F49039851F830000028B8F81200DC
:10C0D00005D002998842E6D3A1460290E3E7019990
:10C0E0008842E0D3A3460190DDE70599C907C8D08F
:10C0F0005146BAF10A0F0EDA0C46214801EB440111
:10C1000050F8310080B11FA340F26D1245A13BA051
:10C11000FBF786FE08E05946BBF10A0F03DB4946F0
:10C12000B9F10A0FADDA0C460A2C06DB15A340F272
:10C130007F1242A131A0FBF773FE204600F09EF86B
:10C140000A2C06DB0FA340F283123CA12BA0FBF7C5
:10C1500067FE0B4804EB440100EBC105287D30B1BC
:10C1600008A34FF4C2723AA124A0FBF759FE0EB106
:10C1700030686860002068820698A86080E7000048
:10C1800004BD02202E2E2F4D6964646C65776172A8
:10C1900065732F54686972645F50617274792F4CB3
:10C1A0007749502F7372632F636F72652F697076B2
:10C1B000342F6574686172702E630000737461744B
:10C1C00065203D3D204554484152505F53544154F1
:10C1D000455F50454E44494E47207C7C2073746136
:10C1E0007465203E3D204554484152505F535441B0
:10C1F00054455F535441424C450000004173736500
:10C200007274696F6E2022257322206661696C65E5
:10C2100064206174206C696E6520256420696E203D
:10C2200025730A006172705F7461626C655B695DA1
:10C230002E71203D3D204E554C4C000069203C2085
:10C240004152505F5441424C455F53495A450000AA
:10C250006172705F7461626C655B695D2E7374619D
:10C260007465203D3D204554484152505F53544130
:10C2700054455F454D5054590000000070B5074CBF
:10C2800000EB4005002654F8350018B109F032FCE7
:10C2900044F8356004EBC500067570BD04BD02208E
:10C2A0002DE9F0411C4615460E00074606D116A39F
:10C2B00040F2662222A126A0FBF7B2FD35B912A3F7
:10C2C00040F267222CA122A0FBF7AAFD34B90EA3ED
:10C2D0004FF41A722CA11EA0FBF7A2FD0A2F10D258
:10C2E0002D4807EB470100EBC100017D022908D36F
:10C2F000011D316081680C30296020600120BDE89B
:10C30000F0810020FBE700002E2E2F4D6964646C45
:10C310006577617265732F54686972645F506172EA
:10C3200074792F4C7749502F7372632F636F726546
:10C330002F697076342F6574686172702E63000007
:10C3400069706164647220213D204E554C4C0000A0
:10C35000417373657274696F6E20222573222066A3
:10C3600061696C6564206174206C696E6520256468
:10C3700020696E2025730A006E6574696620213D70
:10C38000204E554C4C0000006574685F7265742047
:10C39000213D204E554C4C0004BD02202DE9F047B4
:10C3A00086B00D0006460AD074684FF480792B4899
:10C3B0002188494513D12179062910D109E028A304
:10C3C00040F28A2234A138A0FBF72AFD06B0BDE86E
:10C3D000F0876179042902D16188082906D0018D8E
:10C3E000491C0185C18B491CC18322E0418B8046D9
:10C3F000491C4183D4F80E000490A169686820B1FB
:10C40000814202D101273B4601E00027022304F1CB
:10C410000802924604A9284600F0C6FBE088484579
:10C420000BD0B0F5007F04D0B8F82C10491CA8F848
:10C430002C10304609F05EFBC8E7002FF9D002222D
:10C4400004ABCDE90232291DCDE9001A05F1220322
:10C4500019465246284600F0A1FAEAE748BB0220F6
:10C460002E2E2F4D6964646C6577617265732F544D
:10C47000686972645F50617274792F4C7749502FEC
:10C480007372632F636F72652F697076342F6574D2
:10C49000686172702E6300006E6574696620213DCC
:10C4A000204E554C4C000000417373657274696FE7
:10C4B0006E2022257322206661696C656420617498
:10C4C000206C696E6520256420696E2025730A0042
:10C4D000FEB515460E46040006D145A340F21E32B5
:10C4E00051A155A0FBF79CFC36B941A340F21F3285
:10C4F0005BA151A0FBF794FC35B93DA34FF4487202
:10C500005AA14DA0FBF78CFC2146286802F080FE62
:10C5100008B15A4B3FE02868C0F303110E2925D01B
:10C52000A168636800EA01020B409A4208D080B219
:10C53000A0F57E41A93903D0E068B0B304F10C0541
:10C540004F4B50481A7802EB420100EBC1010F7DBE
:10C55000022F2ED38F68A7422BD12F6849688F42B4
:10C5600027D14949C88D401CC88532E001208DF88B
:10C57000040000208DF805005E208DF80600687824
:10C5800001AB00F07F008DF80700A8788DF8080057
:10C59000E8788DF809004FF40060009004F1220261
:10C5A0003146204600F0FEFBFEBDFFE76FF00300C2
:10C5B000FAE7002202EB420100EBC1010F7D022FDE
:10C5C0000CD38F68A74209D12F6849688F4205D1E3
:10C5D0001A703146204600F059F8E5E7521CD2B2F5
:10C5E0000A2AE7D332462946204600F0D7F8DBE78F
:10C5F0002E2E2F4D6964646C6577617265732F54BC
:10C60000686972645F50617274792F4C7749502F5A
:10C610007372632F636F72652F697076342F657440
:10C62000686172702E6300006E6574696620213D3A
:10C63000204E554C4C000000417373657274696F55
:10C640006E2022257322206661696C656420617406
:10C65000206C696E6520256420696E2025730A00B0
:10C660007120213D204E554C4C00000069706164E2
:10C67000647220213D204E554C4C0000CC810408B2
:10C680000C0B001004BD022048BB02202DE9F8432A
:10C690000646154688461C4802EB450100EBC104DE
:10C6A000207D022806D219A340F2EE2225A131A056
:10C6B000FBF7B6FB144A05EB4501207D02EBC105F3
:10C6C0000C35022813D1608A0327B0F58E7F04D978
:10C6D000211D304600F022FA07E0B0F5877F06D32F
:10C6E0002A46211D304600F01FFA00B927754FF485
:10C6F000006000902B4606F122024146304600F0D1
:10C7000051FBBDE8F883000004BD02202E2E2F4D02
:10C710006964646C6577617265732F5468697264CB
:10C720005F50617274792F4C7749502F7372632F69
:10C73000636F72652F697076342F657468617270EB
:10C740002E6300006172705F7461626C655B617280
:10C75000705F6964785D2E7374617465203E3D205E
:10C760004554484152505F53544154455F535441DE
:10C77000424C4500417373657274696F6E202225C7
:10C780007322206661696C6564206174206C696E37
:10C790006520256420696E2025730A002DE9FC5F61
:10C7A0008246223001900E46086814464FF0FF374B
:10C7B0004FF0000B514602F02BFDA8B93068C0F3D2
:10C7C00003110E2910D07EB170B1524601213046BE
:10C7D000FFF724FC05000AD51CB14048818C491C98
:10C7E000818468B2BDE8FC9F6FF00F00FAE77F2DEF
:10C7F00006D33BA340F2C13247A14BA0FBF710FB8D
:10C8000005F0FF09524909EB490801EBC805287DED
:10C8100000280ED0012808D0022806D230A340F20A
:10C82000CD324CA140A0FBF7FBFABBF1000F06D1C3
:10C8300004E001202875C5F808A000E034B93146AD
:10C84000504600F06BF90746002CCBD0287D404EB7
:10C8500002280ED349494FF4006005F10C0381F81A
:10C860000090009021465046019A00F09BFA07463E
:10C8700031E001282FD1254640F2F1376889298916
:10C88000884207D1286828B115A33A463CA126A0C2
:10C89000FBF7C6FA287B400607D522464FF42071E5
:10C8A0000E2008F05DFF044605E02D68002DE5D15F
:10C8B000204609F0F5FA44B156F8380008B109F0FD
:10C8C00019F946F83840002705E004484FF0FF37D3
:10C8D000818C491C8184384684E7000048BB0220D3
:10C8E0002E2E2F4D6964646C6577617265732F54C9
:10C8F000686972645F50617274792F4C7749502F68
:10C900007372632F636F72652F697076342F65744D
:10C91000686172702E63000074797065206F7665AF
:10C9200072666C6F77000000417373657274696F93
:10C930006E2022257322206661696C656420617413
:10C94000206C696E6520256420696E2025730A00BD
:10C9500004BD02206172705F7461626C655B695D29
:10C960002E7374617465203D3D2050454E44494E00
:10C9700047206F7220535441424C45000C0B00106D
:10C980006E6F207061636B6574207175657565737A
:10C9900020616C6C6F776564210000002DE9FF4F0A
:10C9A00081B09846DDE90FAB07004FF0000906D1D2
:10C9B0002FA340F257423CA13FA0FBF731FA4FF4BE
:10C9C00020721C210E2008F07BFC454E050049D04A
:10C9D00068891C2806D226A340F2624241A136A0F3
:10C9E000FBF71EFA6C68119804F0FEFDE08097F8E2
:10C9F0002800062806D01EA340F2694246492EA010
:10CA0000FBF70EFAD8F80010A160B8F80400A08176
:10CA1000DAF80010C4F81210BAF80400E0820E9898
:10CA200029460068C4F80E00DBF80000A0614FF44E
:10CA300080702080082060800620207104206071B2
:10CA400040F60600DDE902230090384600F0AAF91E
:10CA5000308B401C3083284609F04CF8484605B01E
:10CA6000BDE8F08FB08C401CB0844FF0FF30F6E78B
:10CA70002E2E2F4D6964646C6577617265732F5437
:10CA8000686972645F50617274792F4C7749502FD6
:10CA90007372632F636F72652F697076342F6574BC
:10CAA000686172702E6300006E6574696620213DB6
:10CAB000204E554C4C000000417373657274696FD1
:10CAC0006E2022257322206661696C656420617482
:10CAD000206C696E6520256420696E2025730A002C
:10CAE00048BB0220636865636B20746861742066CC
:10CAF0006972737420706275662063616E20686F5E
:10CB00006C642073747275637420657468617270EC
:10CB10005F68647200000000949C0408014A00F001
:10CB200003B80000CC8104087FB5064D031D012425
:10CB3000CDE90035CDE902141E331946FFF72EFF6B
:10CB400004B070BDD281040870B5164D002400BF3A
:10CB500004EB440005EBC002117DF1B1508A401C8A
:10CB600080B25082B0F5967F0AD2012906D00329FF
:10CB70000AD004290AD001290BD00EE0052808D3D9
:10CB80002046FFF77BFB08E0042000E00220107540
:10CB900003E0111D9068FFF7C1FF641C0A2CD7DB6E
:10CBA00070BD000004BD0220F8B5044690F82800CE
:10CBB0001F4616460D46062806D020A340F2A912AD
:10CBC0002CA135A0FBF72CF99DB1286888B121462E
:10CBD00002F01EFB68B92878C0F303100E2808D0B5
:10CBE000224639462846FFF719FA002804DA40B2EF
:10CBF000F8BD6FF00F00F8BD00EB40013048022394
:10CC000000EBC102137594603368D360B38813825C
:10CC10000023538250F8315075B140F831304FF451
:10CC200000600090334604F122022946204600F0BD
:10CC3000B9F8284608F05EFF0020F8BD2E2E2F4DD3
:10CC40006964646C6577617265732F546869726496
:10CC50005F50617274792F4C7749502F7372632F34
:10CC6000636F72652F697076342F657468617270B6
:10CC70002E6300006E657469662D3E68776164649A
:10CC8000725F6C656E203D3D204554485F485741BA
:10CC90004444525F4C454E00417373657274696F32
:10CCA0006E2022257322206661696C6564206174A0
:10CCB000206C696E6520256420696E2025730A004A
:10CCC00004BD02202DE9F04105464089334C0E4653
:10CCD0004FF00E080E2809D8208D401C2085E08BCF
:10CCE000401CE083B06C401C88644BE0E87B18B9C2
:10CCF00096F82C00401CE873686801788789CA0799
:10CD000014D0012905D006222549F3F7C2FB48B10A
:10CD10000CE0417851B980785E2807D1687B40F0FB
:10CD2000100002E0687B40F008006873082F0CD008
:10CD3000B7F5C16F17D0208D401C2085E08B401CBB
:10CD4000E083F06C401CF0641CE096F829000007BA
:10CD500018D54146284609F0F1F898B931462846D9
:10CD600002F0B0FB16E096F8290000070AD541460C
:10CD7000284609F0E3F848B1608C401C6084E08BE1
:10CD8000401CE083284608F0B5FE03E03146284603
:10CD9000FFF704FB0020BDE8F081000048BB022043
:10CDA000CC8104082DE9F04104461F4690460E460A
:10CDB000069804F019FC05460E21304608F01CFACE
:10CDC00038B113484189491C41816FF00100BDE829
:10CDD000F0817068858139680160B9888180D8F8F0
:10CDE0000020C0F80620B8F80410418194F828000B
:10CDF000062806D007A34FF4997214A120A0FBF7D0
:10CE00000FF831462046A269BDE8F0411047000006
:10CE100048BB02202E2E2F4D6964646C65776172C9
:10CE200065732F54686972645F50617274792F4C16
:10CE30007749502F7372632F6E657469662F65741E
:10CE40006865726E65742E63000000006E6574691B
:10CE5000662D3E6877616464725F6C656E206D75E7
:10CE60007374206265203620666F72206574686571
:10CE7000726E65745F6F75747075742100000000C8
:10CE8000417373657274696F6E2022257322206668
:10CE900061696C6564206174206C696E652025642D
:10CEA00020696E2025730A0010B5040006D10AA37C
:10CEB00040F2D2220FA113A0FAF7B2FF732084F838
:10CEC0002A00742084F82B00184844F8140F1848DE
:10CED0006060002010BD00002E2E2F4C5749502FAF
:10CEE0005461726765742F65746865726E657469E4
:10CEF000662E63006E6574696620213D204E554C98
:10CF00004C000000417373657274696F6E202225B6
:10CF10007322206661696C6564206174206C696E9F
:10CF20006520256420696E2025730A00D1C402089B
:10CF300001150308DFF89C80274E4FF0FF39494662
:10CF4000D8F8000008F0A2F80028F8D1002004F07A
:10CF50006FFA0500F3D000246FF00D016F6808F040
:10CF60009EFEB88904F040FBB0F5006F04D0A0F538
:10CF7000006006381DD10EE06868346808E0016979
:10CF80006268914203D194F82910C90711D124682D
:10CF9000002CF4D10DE068683468806907E06168AE
:10CFA000884203D194F82910C90702D12468002CC3
:10CFB000F5D10E21284608F072FE24B122692146DF
:10CFC0002846904718B1284608F094FDB7E7002D91
:10CFD000BCD1B4E71C010020040B0010F0B589B0EF
:10CFE0000D4606461C461746202101A8F3F715FA00
:10CFF000D5E900010023012204F05AF90020009035
:10D00000052301AA1CA1304603F0A0FD012825D16B
:10D0100001A919A004F040F9052218A101A8F3F70D
:10D0200038FA20B121463846FBF72CFF08B1154CE1
:10D0300011E015A116A004F02FF917A112A004F019
:10D040002BF915E0F3F710FA024601A82168F3F76F
:10D0500020FA48B10C3420680028F3D10AA10CA0B2
:10D0600004F01AF910A1E9E76268294630469047B2
:10D0700004F090F809B0F0BD636D64006C6F6769EF
:10D080006E000000000900106572726F72000000EF
:10D0900073746174757300006E6F74206C6F6767D2
:10D0A000656420696E000000756E6B6E6F776E2090
:10D0B000636D640038B5054601F008F804000FD12F
:10D0C0006946284618F0D2FD040009D12869FEF708
:10D0D00067FA040000D128600021009816F096FC41
:10D0E000204638BD2DE9F74787B014468A4600220E
:10D0F000694607A801F004FA5FEA000958D10098D0
:10D1000020600098076A8169BA1E914202D8CAF865
:10D1100000104DE001784FF00008012901D0C66AE7
:10D1200019E002240190214601A801F0D7FB411C1F
:10D1300003D0012803D028B106E0012000E002203E
:10D1400081462CE008F101080098641C006A8442C2
:10D15000E9D324E05DB93146761C009806F037F932
:10D160005FEA00091BD1009C4FF400753C34009825
:10D1700000780228204604D004F040F9000108D0CD
:10D1800009E004F046F908B908F10108A41CAD1E35
:10D1900003E008F10108241D2D1F7F1EDAD1CAF813
:10D1A00000800098C0F81880017941F001010171F8
:10D1B0004946009816F02AFC0AB04846BDE8F087B8
:10D1C0002DE9FC4100259046074604464E1E11E01D
:10D1D00001AB01226946404600F020FE019801287B
:10D1E0000AD19DF800000D2804D06D1C04F8010B35
:10D1F0000A2801D0B542EBDB0020207015B138467B
:10D20000BDE8FC810020FBE72DE9FE4F0D460446FA
:10D21000694618F02BFD070064D1677D002FFBD114
:10D22000E06A4FF0020A4FF0010804F1300B0028C9
:10D230006AD0691C29D0E068A84200D20546A561E1
:10D24000002D4FD02046691EFBF746FF0146E061E6
:10D250000098FBF781FF002875D000996D1E4A8960
:10D26000521E02EA55221518208BC005E9D0226A09
:10D27000AA42E6D0207D00063BD5487801235946D6
:10D28000FEF77CFC00286ED12FE002C80191A16856
:10D2900083460225F1B10026AD1C02918946204645
:10D2A000761C01F01BFB014601284CD9481C5AD0C2
:10D2B00009F101008142F1D00198854206D8CBF8EE
:10D2C00000600BF10400029A04C083460098006AD3
:10D2D0008842E0D8E06A05600198854203D80021C1
:10D2E000CBF800109FE011279DE0207D00F07F002B
:10D2F0002075009801232A4640785946FEF724FC01
:10D30000002830D125628EE0E068A84203D2217D5A
:10D31000890700D405464FF00009A069C4F81890A9
:10D3200005B3009949894E0270B1691EB1FBF6F24E
:10D33000401EB0FBF6F18A4206D3711E8843A061FD
:10D340002D1AE1690DE04FE0A16849B9002120469E
:10D35000FDF7D2FC0146012846D0481C59D0A160F7
:10D36000E161D9B927E054E0A069AD1B3044A06168
:10D37000207D8007204605D5FDF7BEFC010004D1C5
:10D3800000250DE001F0AAFA0146481C41D0012910
:10D390002AD90098006A884226D9E161B542E3D8CB
:10D3A000A0692844A061E80505D00098FBF7D4FEE9
:10D3B000D0B100EB5529E168A069884204D9E0604A
:10D3C000217D41F040012175C0052CD0226A4A45DB
:10D3D00029D0207D000614D50098012359464078B5
:10D3E000FEF7CCFBA8B908E084F815A0022100984C
:10D3F00016F00CFB0220BDE8FE8F207D00F07F00C0
:10D400002075009801234A4640785946FEF79CFB58
:10D4100038B184F815800121009816F0F7FA012040
:10D42000E9E7C4F820903946009816F0EFFA38463C
:10D43000E1E700002DE9FF4F91B01D4614464FF47F
:10D44000007611A8DDF8788001F0B9FA002803DA37
:10D450000B2015B0BDE8F08FF54951F8201009B147
:10D4600000220A70C0B20490FEF74CFBC10701D045
:10D470000320EEE7400701D50A20EAE70EAA0321C0
:10D480000498FEF753FB38B90E9828B1B0F5004F59
:10D4900002D8411E084201D001200E90B24624B1AC
:10D4A00054453AD3B4F1807F37D8601E044234D15A
:10D4B000B8FBFAFBB4FBFAF75FEA4B202C4610905E
:10D4C0007ED00CAA01210498FEF730FB002878D109
:10D4D000129800076FEAA0104FEA90690C9848452F
:10D4E0006ED3A0EB090086460C90802868D3802F6D
:10D4F00013D812984FF6F5728007129840F6F5731C
:10D5000007D500F0070002287ED01298C0077BD014
:10D5100001E0C00701D0022696E0132099E73D0004
:10D520000DD100204FEA5E480125DFF808C301E075
:10D530006D00401C3CF8101009B14145F8D9BEFB04
:10D54000F5F00AEB8001C91DB1FBFAF82021039127
:10D5500000210791904233D9B749884230D828E05A
:10D56000B449002001254FEA1E3C0E3901E06D0050
:10D57000401C31F81080B8F1000F01D0E045F6D919
:10D58000BEFBF5F0984203D9042101EB400006E010
:10D59000012600EB40000321401C01EB50005044E9
:10D5A000401EB0FBFAF8012081030390B1FBFAF0B2
:10D5B0000790039909EB010000EB0801059001E0D9
:10D5C00055E034E1079808440E9900EB010C491E20
:10D5D000ACF1010C2CEA010CACEB0001032E1AD0CB
:10D5E00008EB010800EB0511A1EB090171453ED8DC
:10D5F00003990798AEEB0101A1EB0801081AB0FBF3
:10D60000F5F00190032E00E024E00ED0022E13D09E
:10D61000012E2AD02DE0DDF80CC08C44CDF80CC0D2
:10D62000DDF814C061440591DCE7904221D8F7B9D8
:10D630006F087FF474AF1AE0904211D93FB94020CF
:10D64000B0EB450F03D36F003D0099D188E71298E6
:10D65000800707D5032662E76F00802FF4D906E024
:10D66000984206D8002FF7D001E0984201D90E2049
:10D67000EFE652460021204605F09CFC0B226FA1EC
:10D68000204605F0E3F9514604F10B000DF090FE41
:10D690006573039881B204F10E000DF089FE01203C
:10D6A0002074032E0ED0514604F111000DF080FEBF
:10D6B0000C99B1F5803F07D289B204F113000DF047
:10D6C00077FE05E00021EFE704F120000DF068FE91
:10D6D000F82060753F2104F118000DF069FEFF216C
:10D6E00004F11A000DF064FE494604F11C000DF02F
:10D6F00057FE8027032E27D001F04FF9014604F191
:10D7000027000DF04DFE1FFA88F104F116000DF010
:10D710004FFE84F82470292084F8260013224AA1A1
:10D7200004F12B0005F092F904F5FF704AF655213B
:10D7300008900DF03DFE01234A4621460498FEF76D
:10D740001DFA002873D124E001F027F9014604F105
:10D7500043000DF025FE414604F124000DF020FEAB
:10D76000022104F12C000DF01BFE012104F1300018
:10D770000DF01EFE062104F132000DF019FE2920E5
:10D7800084F8407084F84200132234A104F1470069
:10D79000C8E7032E32D1012309F10602214604987D
:10D7A000FEF7ECF952460021204605F003FC304913
:10D7B00020460DF0F5FD2F4904F5F2700DF0F0FD57
:10D7C000019904F5F470491E0DF0EAFD022104F5FB
:10D7D000F6700DF0E5FD4AF6552108980DF0E8FDCC
:10D7E000012309F1070221460498FEF7C7F9012336
:10D7F00009F1010221460498FEF7C0F900212046F4
:10D80000109A05F0D7FB6FF00701032E02D0012E0E
:10D8100032D032E020460DF0C3FD4FF0FF31201D25
:10D820000DF0BEFD6FF0704104F1080026E073E0DA
:10D830009C0A0010107E0408F5FFFF0FEBFE904DD0
:10D8400053444F53352E30004E4F204E414D45200E
:10D850002020204641542020202020004E4F204EE2
:10D86000414D4520202020464154333220202000C5
:10D870005252614172724161404920460DF090FD63
:10D88000474658465F4500D8384680460346DDE99E
:10D8900004022146FEF772F9F0BB524600212046F1
:10D8A00005F088FB0598B7EB080740440590E8D1E0
:10D8B000032E00D0079D58465D4501D9074600E07C
:10D8C0002F46DDE904023B462146FEF757F918BB17
:10D8D0000598ED1B38440590EDD1032E05D00C982A
:10D8E000B0F5803F03D3062604E00C2602E0022EAA
:10D8F00038D001261298000736D45246002120461F
:10D9000005F058FB4AF6552108980DF051FD04F535
:10D91000DF750020287000E02EE001216970A970F9
:10D92000E8702E710C9909EB010043F6C161B0FB60
:10D93000F1F0FE2169713F2141EA9001A971E8717E
:10D94000494605F108000DF02BFD05F10C000C997E
:10D950000DF026FD0123002221460498FEF70EF962
:10D9600050B901E00426C5E7002211460498FEF7ED
:10D97000DDF800283FF47DAD01206AE5F8FFFF00E7
:10D980002DE9F74181B0904602980090684601F079
:10D9900016F8040003D50B2004B0BDE8F081164E44
:10D9A000002756F824503DB12846FBF785FB28692F
:10D9B00000F051FD88B12F70019929B101F8107B59
:10D9C000E0B200F03BFD40B1019846F8240010B1F0
:10D9D000B8F1010F03D00020DEE70220DCE70022CF
:10D9E00001A902A800F08CFD04460146019816F03A
:10D9F0000DF82046D0E700009C0A00102DE9F74FF3
:10DA00008EB005000BD002F03F06324669460FA8E3
:10DA100000F076FD04004FF0000904D006E1092073
:10DA200011B0BDE8F08F00984FF4007B019058468C
:10DA300000F016FD5FEA000809D0009901A8C1F8BE
:10DA40000C800F9900F08EFE040006D014E0112126
:10DA5000009815F0DBFF1120E2E79DF83300000687
:10DA600001D5062408E0700801D0012100E0002162
:10DA700001A8FBF7F3FA044616F01C0F5FD04FF035
:10DA8000010AC4B1042C10D10020704902E0401CEE
:10DA9000022804D201EB00121268002AF7D10228F2
:10DAA00007D001A8FDF7D4FE044646F008066CB185
:10DAB000A3E01224A1E09DF80A0010F0110F01D09C
:10DAC00007249AE0700701D50824ACE0300745D55B
:10DAD00000F063FF0746099839460E300DF060FCF0
:10DAE0000998394616300DF05BFC09992020C87260
:10DAF0000999009803F06FFC0746002209990098E5
:10DB00000DF03AFC099800211C300DF049FC0099F9
:10DB100081F803A007B3D1F838A00022394601A844
:10DB200009F0D6FD040068D15146009805F04FFC7D
:10DB300004000098A7F1010747610BD05DE0ECBB42
:10DB40009DF80A00C10601D5042456E0B10701D5AD
:10DB5000C007B5D1300701D546F040060098806B6C
:10DB600068620998A862700801D0012100E00021D4
:10DB700001A801F039FA286150B30999009803F01F
:10DB80002AFCA86009981C3003F038FCC5F82C90DA
:10DB9000E86000992960009905F130005A46C9886B
:10DBA000A9802E7585F81590C5F820900021824631
:10DBB000C5F8189005F0FEF9B00600E01DE040D56C
:10DBC000EE68DEB3AE610098A9684089470210E0B4
:10DBD000022412E0284600F081FE0146012800D808
:10DBE0000224481C02D0F61B1CB104E00124F61BE1
:10DBF00001E0BE42EED8E96124B1404600F032FCBB
:10DC0000A4B915E0F0051CD00098FBF7A5FAB0B157
:10DC100000EB56222A620098012351464078FDF716
:10DC200093FF58B10124404600F01CFCC5F8009059
:10DC30002146009815F0EAFE2046F1E601E00224B4
:10DC4000F1E7404600F00EFCF2E70000A82F0010BC
:10DC50000FB42DE9F0479CB00DF198090090002019
:10DC600001900DF14C080290259810F8011B2590A9
:10DC7000002976D0252903D0684609F090F9F3E70A
:10DC8000002510F8011B2E462590302902D02D29A1
:10DC900002D010E0012500E0022510F8011B2590BC
:10DCA00009E000BF06EB860001EB40062598303EF8
:10DCB00010F8011B2590A1F130000928F2D96C2938
:10DCC00001D04C2905D1259845F0040510F8011B19
:10DCD0002590002945D0A1F161000A46192801D8F4
:10DCE000203AD2B24F2A42D006DC422A3DD0432A03
:10DCF00038D0442AC0D13CE0532A0DD0552A38D020
:10DD0000582AB9D11023680701D4442A33D059F8CE
:10DD1000040B442A31D035E059F8047B002400E09C
:10DD2000641C385D0028FBD1A80704D50CE0202135
:10DD3000684609F034F92046641CB042F7D303E08A
:10DD400068467F1C09F02BF939780029F8D103E0E7
:10DD50002021684609F023F92046641CB04283D292
:10DD6000F6E753E019F8041B86E70223CBE7082304
:10DD7000C9E70A23C7E759F8040B002802DA404232
:10DD800045F0080500244746B0FBF3F203FB1202FE
:10DD9000B0FBF3F0D2B2092A05D9782914D04FF09C
:10DDA000070C6244D2B230323A55641C08B1202CC0
:10DDB000EAD3280703D52D2008F80400641C274661
:10DDC000E80704D0302003E04FF0270CE9E72020DB
:10DDD000824603E05146684609F0E1F8A80703D4FB
:10DDE00038467F1CB042F5D34546641E6846295D1F
:10DDF00009F0D5F8002CF8D103E05146684609F047
:10DE0000CEF838467F1CB042A9D2F6E7684609F042
:10DE1000E9F81CB0BDE8F0075DF814FB2DE9FE4FF2
:10DE200088460021196099461546044602A917F054
:10DE30001DFF060001D1667D36B13146029815F00E
:10DE4000E5FD3046BDE8FE8F207DC0070BD0A169FF
:10DE5000E0680127401A4FF0020A04F1300B8542B6
:10DE600000D905468FE00721029815F0CFFD072065
:10DE7000E8E7A169C8056ED102984089401E10EA02
:10DE8000512611D129B1E06A28B12046FBF724F9C7
:10DE900005E0A06803E02046E16900F01FFD0228CC
:10DEA0001BD3411C4ED0E061E1690298FBF754F9A5
:10DEB00098B130440190680A009029D00299321834
:10DEC0004889824201D9801B0090DDE90032487800
:10DED0004146FDF739FEA8BB07E084F815A00221F2
:10DEE000029815F093FD0220ACE7207D00060CD5CA
:10DEF000216A0198081A0099884206D208EB40204E
:10DF00004FF40072594604F0A1FD0098460230E03B
:10DF1000226A019882421CD0207D00060AD5029810
:10DF2000012359464078FDF729FE58B9207D00F0BD
:10DF30007F0020750298012359464078019AFDF729
:10DF400003FE30B167750121029815F05FFD0120D5
:10DF500078E701982062208BC0F30800C0F50076B6
:10DF6000AE4200D92E46011932464046303104F007
:10DF70006DFDA069B0443044A061D9F8000081195A
:10DF8000AD1BC9F80010002D7FF473AF002102987B
:10DF900015F03CFD002055E773B5A2B023A800F0B2
:10DFA0000EFD022201A922A800F0AAFA040070D1F5
:10DFB000019802904FF4007000F052FA050008D06A
:10DFC0000198C56002A8229900F0CCFB040007D09C
:10DFD00073E01121019815F019FD112024B070BDD6
:10DFE0009DF8370010F0A00F01D0062465E0022153
:10DFF00002A8FBF733F804005FD10A9915220FA895
:10E000000B3104F023FD342202A915A804F01EFDF3
:10E0100015A8239900F0A6FB040002D0042C0AD016
:10E020004BE004991798884203D107991A988842BF
:10E0300001D0082441E015A8FDF70AFC04003CD1FA
:10E040001D9C13220DF13E0104F10D0004F0FEFCB5
:10E050009DF83C00012640F02000E0720198C67057
:10E06000E17AC90620D5179A049991421CD021461D
:10E0700003F0B1F901460198FBF76EF8010009D0F1
:10E08000019805F0A4F90400019800F15C0103D0A7
:10E0900013E015E0022410E04A782E2A04D1179AE2
:10E0A0000DF06AF90198C67002A8FDF7C3FC0400E0
:10E0B00003D101980DF0E0F90446284600F0D2F9AA
:10E0C0002146019815F0A2FC204687E7F8B50446E2
:10E0D000694617F0CBFD050043D1207D410640D5B0
:10E0E000000612D50098226A0123407804F130011D
:10E0F000FDF744FD28B10121009815F087FC0120AF
:10E10000F8BD207D00F07F00207500F046FC06463B
:10E11000616A009805F05BF9050022D1A56A2946DD
:10E12000E87A40F02000E872A26820680DF024F937
:10E1300005F11C00E1680DF033F9314605F11600D8
:10E140000DF02EF9002105F112000DF031F90098C3
:10E150000121C1700DF090F90546207D00F0BF004F
:10E1600020752946009815F051FC2846F8BD71B578
:10E170009DB002220DA91DA800F0C2F904000D985F
:10E1800000905DD14FF4007000F06AF9060008D0ED
:10E190000D98C66068461D9900F0E4FA040007D0A7
:10E1A0004BE011210D9815F031FC11201EB070BD0F
:10E1B0009DF82F00800609D402216846FAF74EFF29
:10E1C00004003AD19DF82F00000601D5062434E062
:10E1D0009DF80600C0071DD108990D9803F0FBF8C3
:10E1E00005469DF80600C00616D50D98C169A942DE
:10E1F00010D00F90002111950FA8FDF742FC0400EC
:10E200001BD100210FA8FDF7C7FA040002D0042C8F
:10E2100002D012E0072410E06846FDF70BFC040072
:10E220000BD135B100222946684609F051FA0400A5
:10E2300003D10D980DF020F90446304600F012F994
:10E2400021460D9815F0E2FB2046AFE72DE9FE4F81
:10E2500088460021196099461546044602A917F020
:10E2600005FD060001D1667D36B13146029815F0F4
:10E27000CDFB3046BDE8FE8F207D800705D4072109
:10E28000029815F0C3FB0720F4E7A06901274219A3
:10E290004FF0020A04F1300B824200D2C543A3E0E2
:10E2A000A169C8057DD102984089401E10EA512617
:10E2B00018D129B1E06A38B12046FAF70DFF07E01E
:10E2C000A06838B9002100E0E1692046FCF714FDA0
:10E2D00000287DD001282DD0411C58D0E061A168D4
:10E2E00001B9A060207D00060BD50298226A0123A7
:10E2F00040785946FDF742FCC0BB207D00F07F000E
:10E300002075E1690298FAF727FF98B1304401902F
:10E31000680A00902BD03218029841898A4201D9AC
:10E32000891B0091DDE9003240784146FDF726FC6B
:10E33000E0B907E084F815A00221029815F066FB09
:10E34000022097E7216A0198081A009988420AD2A8
:10E3500008EB40214FF40072584604F077FB207D13
:10E3600000F07F002075009846022CE00FE0216A43
:10E370000198814213D0E168A06988420FD20298C7
:10E38000012359464078019AFDF7DEFB38B16775E5
:10E390000121029815F03AFB01206BE701E001989A
:10E3A0002062208BC0F30800C0F50076AE4200D991
:10E3B0002E46204432464146303004F047FB207D53
:10E3C00040F080002075A069B0443044A06100E0B6
:10E3D0000DE0E168884200D80846E060D9F8000006
:10E3E0008119AD1BC9F80010002D7FF459AF207DB5
:10E3F000002140F040002075029815F007FB002036
:10E4000038E70000802804D30B4A51B1FF2801D916
:10E410000020704702EB4000A0F58050B0F8000FDC
:10E42000704732F81130834203D0491C89B28029E9
:10E43000F7D38031C8B270471E7E040838B500207B
:10E440000C4600900121684606F0D6FD20600028A9
:10E4500000D0012038BD10B506F0E4FD012010BD4C
:10E4600008F0D6BD17F020B906F0E8BD10B50024BD
:10E470004FF47A7106F00AFE00B90124204610BD5F
:10E4800030B5B0F5805F01D21B4900E01B4931F87F
:10E49000022B002A15D0904213D331F8024B230AE5
:10E4A000E5B252FA84F4844221D9092B09D2DFE87B
:10E4B00003F005090E11131517191B00801A31F806
:10E4C000100030BD811A01F00101401A00E010383F
:10E4D00080B230BD2038FBE73038F9E71A38F7E76B
:10E4E0000830F5E75038F3E7A0F5E350F0E7002BEC
:10E4F000CDD101EB4501CAE71E7F04081081040855
:10E500002DE9FF41002790460E460F6000F057FAB4
:10E51000050003D50B2004B0BDE8F0818E4850F80B
:10E520002540BCB1204602F079FFA8B134602078C4
:10E5300008F0FE0620B16078FDF714FBC1070DD08E
:10E540002770E8B2B8466070FDF7DCFAC1070AD060
:10E550000320E0E70C20DEE70F20DCE70EB14007E8
:10E5600004D40020D7E71EB1400701D50A20D2E726
:10E57000002631462046FAF731FD022822D1002537
:10E580004FEA0D0704EB051090F8FE1100F5FD7041
:10E5900019B1083002F032FF00E0002047F82500F2
:10E5A0006D1C042DEED3002557F8256036B1314699
:10E5B0002046FAF713FD022801D203E003206D1C68
:10E5C000042DF1D3042809D002286DD204F14700AC
:10E5D00002F01FFFB0F5007F66D101E001209AE74D
:10E5E00004F1520002F015FF18B904F1600002F0C6
:10E5F00005FF606294F84C50A570012D01D0022DEA
:10E6000052D1454394F849006081E8B3411E084265
:10E610004AD104F14D0002F0FCFE2081000743D1F5
:10E6200004F14F0002F0F5FE070004D104F15C0094
:10E6300002F0E4FE074604F14A0002F0EAFE01009F
:10E6400032D02389481900EB131297422CD3B81A01
:10E650006789B0FBF7F0B8B103274FF6F57C60454A
:10E6600000D8022740F6F57C604500D80127801CC1
:10E670003244626331442062C4E90A61032F15D039
:10E6800013B12944216300E00EE0022F1FD000F0F7
:10E69000010100EB400001EB500000BF616A00F295
:10E6A000FF10B1EB502F14D20D2034E704F16600B7
:10E6B00002F0AFFE0028F7D120890028F4D104F140
:10E6C000680002F09BFE2063206A8000E6E74000BD
:10E6D000E4E74FF0FF30A061606180202071032FDC
:10E6E0002CD104F16C0002F094FE012826D1711C9B
:10E6F000204604F06CFE08BB84F8048004F23A2043
:10E7000002F087FEA0F52A41553917D104F13C00EB
:10E7100002F074FE1149884210D104F5087002F02D
:10E720006DFE0F49884209D104F5097002F066FEBA
:10E73000A06104F50A7002F061FE6061064927706D
:10E74000091F0888401C0880E0802046C4F81C800F
:10E75000FAF7B2FC05E700009C0A00105252614132
:10E760007272416173B504460568019800782F28DC
:10E7700003D05C2801D0E96908E00198401C0190B1
:10E7800000782F28F9D05C28F7D00021A1600198EB
:10E7900080260078202806D284F82F6000212046A9
:10E7A000FDF76FF97CBD01A92046FCF7F7FA0028B8
:10E7B000F8D12046FCF70EFF94F82F1068B104281A
:10E7C000F0D18A0605D54807EDD584F82F600020E2
:10E7D0007CBD4907FCD405207CBD4907FCD4A07949
:10E7E000C006F8D5A08AC0F30800411928463C317C
:10E7F00002F0F1FDA060D6E738B504468DF80000C0
:10E8000069460320ABBE204638BD000010B5002885
:10E8100021D0114B0022001F196803E0814203D868
:10E820000A4649680029F9D152B11368841A9C42FA
:10E8300004D1006818441060104602E0506000E007
:10E84000186039B102680B1A934203D10B681A445D
:10E8500002604968416010BD680C00107CB5164626
:10E860001C4605460B2204F0F1F8052C11D91A4A72
:10E870000CE00021B61C2346044663F35F04400805
:10E88000E30300D55440491C1029F4D330880028F4
:10E89000EFD107214FEA0D0204F00F003030392884
:10E8A00000D9C01D5054491E2409F5D17E20505472
:10E8B000002000E0401C884202D22B5C202BF9D1C2
:10E8C000082902D2535C491C00E020232B54401C31
:10E8D0000828F5D37CBD0000211001002DE9F0418E
:10E8E00004680D4602290BD3206AA84208D9207873
:10E8F0004FF0FF36012807D002282BD0032839D04B
:10E9000001263046BDE8F081E06A05EB550700EBD3
:10E910005721204604F05BFD0028F2D1C7F3080020
:10E9200020447F1C90F83C80E06A00EB5721204691
:10E9300004F04DFD0028E4D1C7F30800204490F80E
:10E940003C1048EA0120E90701D00609D9E7C0F3E5
:10E950000B06D6E7E06A00EB1521204604F037FDF0
:10E960000028CED1E8B204EB40003C3002F051FD6B
:10E970000646C6E7E06A00EBD511204604F027FD05
:10E980000028BED140F2FF1000EA850020443C3050
:10E9900002F034FD20F07046B3E70020704710B558
:10E9A00002690446017A9368406804F110029847AE
:10E9B0002070E0684069BDE810400CF010BF10B551
:10E9C00004464FF0FF302268002A13D0114600E0C1
:10E9D000491C0B78202B0ED33A2BF9D112F8013BAE
:10E9E000303B0A2B06D28A4204D1002B02D1491CAB
:10E9F0001846216010BD002010BD10B50269044604
:10EA0000017AD368406804F1100298472070E068EA
:10EA10004069BDE810400CF0E2BE000010B50446AD
:10EA2000024813F065FF206010BD00001C160010A6
:10EA30002DE9FF41002716460097019702976A4685
:10EA4000039703F039FF35460024E84606A118F87D
:10EA500004202846F9F7F4F9641C0544102CF5DB72
:10EA600086F82070BDE8FF81253032780000000074
:10EA700070B506460020024613E0B45C5FF0000368
:10EA800084EA000515F0010F4FEA50004FEA5404E4
:10EA900001D080F08C005B1CDBB2082BF0D3521C41
:10EAA000D2B28A42E9D370BD044AD2F8AC315B1CC1
:10EAB000C2F8AC310A46032100F0E8B948BB022095
:10EAC00010B50368002229481B2B4CD2DFE803F065
:10EAD0004B0E1115181B1E2124272A2D30333639D1
:10EAE0003C3F42424245484242424200D0F8700117
:10EAF00001E0D0F8740108602DE0D0F87801FAE761
:10EB0000D0F87C01F7E7D0F88001F4E7D0F8840171
:10EB1000F1E7D0F88801EEE7D0F88C01EBE7D0F808
:10EB20009001E8E7D0F89401E5E7D0F89801E2E732
:10EB3000D0F89C01DFE7D0F8A001DCE7D0F8A40111
:10EB4000D9E7D0F8A801D6E7D0F8AC01D3E7D0F8E0
:10EB5000B001D0E70A60042010BDD0F8B401CAE7C4
:10EB6000D0F8B801C7E7002010BD000048BB022064
:10EB70002DE9FE4F904C05468B46B4F862008F4954
:10EB8000401CA4F86200D4F87001401CC4F8700165
:10EB9000D1F8089099F800000007860E142E6FD364
:10EBA00068890428FBD368680078A0B1082818D0C9
:10EBB00003286ED00B286DD00C286CD004286BD0A5
:10EBC00005286AD00D2869D00E2868D0112867D092
:10EBD000122866D0D5E0D4F89001401CC4F890010A
:10EBE000D7E0D4F88C01DFF8D481401CC4F88C0144
:10EBF000486908F11408C0F303120E2A56D08A4659
:10EC0000096800F005FB002850D128890828C6D3E0
:10EC100006F10E010F46284606F0EEFA002830D025
:10EC20002889811989B2884240D84FF420720E2079
:10EC300006F046FB070039D0798906F108008142C9
:10EC400015D3324649467868F1F7C0FB314638465D
:10EC500007F074F930B15AA3B62267A174A0F9F78E
:10EC6000DFF804E02946384606F0C8FD18B13846FA
:10EC700006F040FF1AE0284606F03CFF3D4623E040
:10EC80008CE03946284607F059F9E8B14CA3C72271
:10EC900008E041E046E04BE050E055E05AE05FE03C
:10ECA00064E069E06CA162A0F9F7BAF8284606F0C2
:10ECB00021FF34F8740F401C2080D4F80001401C60
:10ECC000C4F80001BDE8FE8F314628466F6806F0A3
:10ECD00093FA00BB6868D8F80010FF22C160DAF828
:10ECE000101001610021397079800272418134F87D
:10ECF000600F0122401C24F8DC0BFF23A06E401C97
:10ED0000A066E06F401CE0678DE8060800224146DF
:10ED1000284600F011FD3CE0D4F87801401CC4F80E
:10ED200078012EE0D4F87C01401CC4F87C0128E076
:10ED3000D4F88001401CC4F8800122E0D4F884019A
:10ED4000401CC4F884011CE0D4F88801401CC4F8BD
:10ED5000880116E0D4F89401401CC4F8940110E036
:10ED6000D4F89801401CC4F898010AE0D4F89C013A
:10ED7000401CC4F89C0104E0D4F8A001401CC4F875
:10ED8000A00134F8700F401C24F80A092088401CA8
:10ED900020802846BDE8FE4F06F0ACBE284606F0AF
:10EDA000A9FE34F86A0F401C2080D4F80A01401CE8
:10EDB000C4F80A0186E7000048BB022050B30220D5
:10EDC0002E2E2F4D6964646C6577617265732F54C4
:10EDD000686972645F50617274792F4C7749502F63
:10EDE0007372632F636F72652F697076342F696356
:10EDF0006D702E630000000069636D705F696E7056
:10EE000075743A206D6F76696E6720722D3E706161
:10EE1000796C6F616420746F2069636D7020686520
:10EE200061646572206661696C65640A00000000B7
:10EE3000417373657274696F6E2022257322206698
:10EE400061696C6564206174206C696E652025645D
:10EE500020696E2025730A0069636D705F696E70AA
:10EE600075743A20726573746F72696E67206F7281
:10EE70006967696E616C20702D3E7061796C6F619D
:10EE800064206661696C65640A0000002DE9FF4733
:10EE9000284C07469246D4F8A4018946401CC4F881
:10EEA000A4014FF420722421222006F009FA060062
:10EEB00039D07089242806D21FA34FF4B4722CA134
:10EEC00036A0F8F7ADFF7568D7F804801C2285F8E6
:10EED000009085F801A04FF00009A5F80490A5F86E
:10EEE0000690706879680830F1F770FAD8F80C006D
:10EEF000039003A800F068FE80B1A5F8029034F8F2
:10EF0000602FFF23521C22800122CDF80090CDE912
:10EF1000012003AA0021304600F00EFC304606F026
:10EF2000E9FDBDE8FF87D4F8A801401CC4F8A8019A
:10EF3000F7E7000048BB02202E2E2F4D6964646C59
:10EF40006577617265732F54686972645F5061728E
:10EF500074792F4C7749502F7372632F636F7265EA
:10EF60002F697076342F69636D702E630000000086
:10EF7000636865636B20746861742066697273747A
:10EF800020706275662063616E20686F6C64206912
:10EF9000636D70206D6573736167650041737365A0
:10EFA0007274696F6E2022257322206661696C6518
:10EFB00064206174206C696E6520256420696E2070
:10EFC00025730A00044AD2F8B0315B1CC2F8B03194
:10EFD0000A460B21FFF75ABF48BB0220EFF305801A
:10EFE000002800D001207047F0B502461D4BD2F832
:10EFF0000050002003EB00142668AE4207D166687B
:10F000009768BE4203D1A4685669B44202D0401C3E
:10F010000228EFD3022814D1002002E0401C02286D
:10F0200004D203EB00142468002CF7D102280ED080
:10F0300003EB00142560956865605269A2600022A8
:10F04000A281002903EB0011898902D019B10020A7
:10F05000F0BD491C01E04FF4807103EB0012401C2D
:10F060009181F0BDA82F001070B510460C461D46CA
:10F07000014601230B4A20460AF09EF878B10A485F
:10F080002668046809E0204605F0A4FEB04203D1DA
:10F090000020C5F8E84070BD2468002CF3D1F120B1
:10F0A00070BD000084850408040B001070B588B0A2
:10F0B0000120009016460D4611F8042B06AB01A85E
:10F0C00009F007FF104804680AE0204605F082FEB8
:10F0D000009023460122694601A809F0CBFE24686E
:10F0E000002CF2D19DF8120010B1F12008B070BDD3
:10F0F0009DF810202846039909F05AFF0598C6F894
:10F10000E8000020F2E70000040B001070B50B4689
:10F110000146D0F8E800CC68022101221D46172CD8
:10F120005DD2DFE804F05C0C0F14191C1E272F3B86
:10F130003D3F41434547494B4D4F5153560005F024
:10F1400049FE44E00224224600F12A010DE090F835
:10F150002E0002E004240BE0008C1860FAE7006B3C
:10F1600035E00624224600F122012846F1F72EF967
:10F17000204670BD90F82900C00701D01A60E9E769
:10F180001960E7E790F82900C30705D0400701D5CB
:10F190002A60DFE707201AE02960DBE7406B16E012
:10F1A000806B14E0C06B12E0006C10E0406C0EE06D
:10F1B000806C0CE0C06C0AE0006D08E0406D06E079
:10F1C000806D04E0C06D02E0006E00E00020286069
:10F1D000C0E7044801788C0022464168C5E700205A
:10F1E00070BD00003084040800684068012801D028
:10F1F0000020704705480022006801E00068521CAA
:10F200000028FBD104200A6070470000040B0010A6
:10F21000421C12D088B191F8292092070BD54B6877
:10F22000834208D0896800EA01020B409A4202D169
:10F230000143491C01D000207047012070470000A5
:10F240002DE9F74F88B00446099800251426008C54
:10F25000AF1F1438C11700EB5170C0F3CF000390FB
:10F2600060680690017801F00F01052903D0384647
:10F270000BB0BDE8F08F6189142907D263A34FF466
:10F280003F7271A177A0F8F7CBFDF0E7C08802F0DC
:10F29000ABF9C0F30C0100F40050029107902089F3
:10F2A00014381FFA80F894E003994FF6FF7000EAD3
:10F2B000C1004146404500D9084604904FF42072F1
:10F2C00014210E2005F0FCFF5FEA000A7ED0BAF898
:10F2D0000A00142806D24DA34FF449726BA161A015
:10F2E000F8F79EFD1422DAF804000699F1F76EF89B
:10F2F000DAF804000590049F35E06089811B8DB227
:10F30000B04206D241A340F22D3268A155A0F8F7D1
:10F3100087FDAF4200D23D461DB3052003F0E6FF56
:10F320005FEA000961D060684B463044CDE90005D2
:10F3300041222946002006F04DF95FEA000B60D01B
:10F34000204606F0ADFD5D49C9E904145946504612
:10F3500006F05CF9781B07043F0C06D000262468F1
:10F36000CBE724680026002FC7D1701986B2099810
:10F37000008C143840450298C0F30C0001DB07995B
:10F3800009B140F4005002F02FF90599C8800498A3
:10F39000143080B202F028F90599488005980021C0
:10F3A0004181099851460A9A436998474448018E19
:10F3B000491C0186504606F09DFB0499A8EB01000C
:10F3C0001FFA80F8DDE90201084400E010E080B295
:10F3D0000290B8F1000F7FF467AF3948D0F82411DC
:10F3E000491CC0F82411002042E7504606F082FB79
:10F3F0003348D0F82811491CC0F828114FF0FF30CD
:10F4000036E7484600F004FFEFE700002E2E2F4DB0
:10F410006964646C6577617265732F54686972649E
:10F420005F50617274792F4C7749502F7372632F3C
:10F43000636F72652F697076342F6970345F6672FE
:10F4400061672E63000000006970345F6672616757
:10F4500028293A207062756620746F6F2073686F78
:10F4600072740000417373657274696F6E20222597
:10F470007322206661696C6564206174206C696E1A
:10F480006520256420696E2025730A0074686973FD
:10F49000206E656564732061207062756620696EF8
:10F4A000206F6E652070696563652100702D3E6C6C
:10F4B000656E203E3D20706F66660000C50803083B
:10F4C00048BB02202DE9F047DFF83482074640466A
:10F4D0000E4630F84A1F491C0180D0F8EE10491C36
:10F4E000C8F838117D6804212878B1EB101F11D0BD
:10F4F000384606F0FFFA404630F85C1F491C20F8F9
:10F500000E190188491C0180D0F8AE10491CC8F8BA
:10F51000FC10A6E000074FEA9069688802F064F8E2
:10F5200004463889A04203D92146384606F01EFC1D
:10F530007989494505D33889A04202D3B9F1140F1E
:10F540000ED2384606F0D6FA404630F8521F491C13
:10F5500020F804190188491C0180D0F8BA106BE02A
:10F560002969DFF8A0A1C1F303100E28CAF814100E
:10F57000EA68CAF8102005D0304600F0C7F850B14C
:10F58000344619E096F82900C00702D070680028B8
:10F59000F6D1002410E09AF8140000247F280BD044
:10F5A0005948046806E0B44203D0204600F0AEF8A3
:10F5B00010B92468002CF6D13146DAF81000FFF7B4
:10F5C00027FE60BB9AF81000C0F303100E2826D067
:10F5D000B4B3E88830F0C00005D0384600F08EF9AA
:10F5E00007003ED07D68CAF80850CAE9004629786D
:10F5F00038460907890EAAF80C10494606F09EFC09
:10F60000687A012845D0062839D011282CD05546D3
:10F610002146DAF81400FFF7FBFD78B350E03846D6
:10F6200006F068FA404630F84E1F491C20F83E1B91
:10F63000416F491C4167C16F491CC8F8081110E0AF
:10F64000FFE7404630F84E1F491C20F83E1B416F33
:10F65000491C4167C16F3846491CC8F8081106F0BB
:10F6600049FA0020BDE8F087D8F80C113846491C4B
:10F67000C8F80C11314613F00BFC32E013E0D8F857
:10F680000C113846491CC8F80C1131460DF04CFEDF
:10F6900027E0D8F80C113846491CC8F80C1131463F
:10F6A000FFF766FA1DE0287DC0F303100E2807D08F
:10F6B0004946384606F0F6FA02213846FFF7F4F9D3
:10F6C000404630F8581F491C20F80A190188491C87
:10F6D0000180D0F8B6103846491CC8F8041106F06D
:10F6E00009FA0021CAF80010CAF80410CAF8081074
:10F6F000AAF80C10CAF81010CAF81410B1E70000EC
:10F7000048BB022050B30220040B001010B590F843
:10F710002910C9070CD0416851B1064A52698A4282
:10F7200004D001461046FFF773FD08B1012010BD5B
:10F73000002010BD50B30220FEB5DDE90954089E3B
:10F740001AB109B10F6807B9211D0096CDE901541E
:10F7500000F002F8FEBD00002DE9F84F0646DDE995
:10F760000BB9807B984617468A46012806D03AA3F3
:10F7700040F2923245A148A0F8F752FB504D6FF08D
:10F780000104D5F81001401CC5F81001002F3AD033
:10F790001421304605F030FD002837D17089746897
:10F7A000142806D22CA340F2C63246A13AA0F8F79C
:10F7B00037FB84F8088084F809B038682061452058
:10F7C00020700A986070308901F00EFFDFF8248104
:10F7D00060804FF0000BA4F806B0B8F8000001F00C
:10F7E00003FFA080B8F80000401CA8F80000BAF1A0
:10F7F000000F05D0DAF80000E060A4F80AB014E0C9
:10F800003D480068F8E7708914280AD235F85C0F83
:10F81000401C25F8B80B2868401C28602046BDE82D
:10F82000F88F70686F460069009035F8480F401CEB
:10F830002880B9F8200040B13189814205D93A4683
:10F8400049463046FFF7FCFCE9E7D9F81430484652
:10F850003A4631469847E2E72E2E2F4D6964646C94
:10F860006577617265732F54686972645F50617265
:10F8700074792F4C7749502F7372632F636F7265C1
:10F880002F697076342F6970342E6300702D3E72AC
:10F890006566203D3D203100417373657274696F68
:10F8A0006E2022257322206661696C656420617474
:10F8B000206C696E6520256420696E2025730A001E
:10F8C00048BB0220636865636B20746861742066BE
:10F8D0006972737420706275662063616E20686F50
:10F8E0006C64207374727563742069705F686472ED
:10F8F00000000000F80100204C8304082DE9F14FBE
:10F90000874D688E401C6886D5F83001401CC5F8CC
:10F91000300100984668307800F00F00052805D0C7
:10F92000B5F84400401CA5F84400F1E0F08801F06F
:10F930005BFEC0044FEA1048708801F055FE317834
:10F940000907890E8142F0D8401A1FFA80F9009801
:10F9500005F0FDFE734C0746208838440A2808D974
:10F960003946304600F044FFF0B3208838440A2876
:10F970003BD8A24664684FF0000B18E06069F1685C
:10F98000884213D1A069316988420FD1A089B1881A
:10F9900088420BD1B5F84600401CA5F8460044B19A
:10F9A000F08801F021FEC00423D02DE02468002C53
:10F9B000E4D1042003F09AFC04000AD13946304611
:10F9C00000F016FFB84210DB042003F08FFC0400A7
:10F9D0000BD02021F0F721FD0F20E077DAF804109A
:10F9E0002160CAF8044009E0FFE7A88F401CA887FF
:10F9F0008EE0E08901F0F8FDC00405D01422314604
:10FA000004F10800F0F7E2FCB07940F34016761CF0
:10FA100008D008EB090080B2404568D34FF6EB717F
:10FA2000884264D832462046009900F08BFC411C85
:10FA30005DD0BAF800203A44AAF8002036B108EBAD
:10FA40000901A183A17F41F00101A17701284CD1D7
:10FA5000A08B142214301FFA80F8606804F10801AA
:10FA6000466830463768F0F7B1FC404601F0BCFD0F
:10FA70007080A6F806B0A6F80AB0D4F8048009E0B1
:10FA8000142138467E6806F059FA3946404605F09A
:10FA9000BDFD3768002FF3D1DAF8041056468C42CA
:10FAA00005D1002105E00868A04202D001460029E6
:10FAB000F9D1204600F06AFD404605F048FE318845
:10FAC0000446A14206D218A340F29B2225A12CA0F5
:10FAD000F8F7A6F93088001B3080D5F81C01401CCF
:10FAE000C5F81C014046BDE8F88F0020FBE76068C0
:10FAF00070B9DAF80400844206D00BA340F2AB22BE
:10FB000029A11FA0F8F78CF90021204600F03EFD46
:10FB1000E88E401CE886009805F0ECFFE5E7000061
:10FB200048BB0220100B00102E2E2F4D6964646C10
:10FB30006577617265732F54686972645F50617292
:10FB400074792F4C7749502F7372632F636F7265EE
:10FB50002F697076342F6970345F667261672E6327
:10FB60000000000069705F72656173735F70627599
:10FB700066636F756E74203E3D20636C656E000099
:10FB8000417373657274696F6E202225732220663B
:10FB900061696C6564206174206C696E6520256400
:10FBA00020696E2025730A006E6F74206669727377
:10FBB00074616C74686F756768206A75737420650A
:10FBC0006E7175657565640070B50146184813E07F
:10FBD00090F82920D3070FD053070DD543685BB1A8
:10FBE00085680C682B4004EA05069E421FD09207E8
:10FBF00002D4C26894421AD000680028E8D10D48A7
:10FC0000006850B190F82920D30706D0520704D5D8
:10FC1000426812B109787F2909D1074830F8561F88
:10FC2000491C20F8C21B0168491C0160002070BDFE
:10FC3000040B0010080B001048BB02202DE9FF4107
:10FC4000884606466F460578F0F7A0FB03461A681B
:10FC5000505D202862D100240A20302D06D116F8EC
:10FC6000015F782D08D0582D06D00820515D20293D
:10FC700004D0102806D016E0102011E0303D04FB1F
:10FC800000540DE081EA810C5FEA0C6C0BD509078A
:10FC900001D5612100E04121691A0A3141EA0414C9
:10FCA00016F8015FE2E72E2D10D01DB11868405DF7
:10FCB000C00734D06846381A012101EBA00005289E
:10FCC00039D2DFE800F02B3E0A13200003A8874258
:10FCD00024D210C716F8015FB9E7B4F1807F1DD2B6
:10FCE0000098FF281AD844EA00642AE0B4F5803F5F
:10FCF00014D20098FF2811D80199FF290ED80006C8
:10FD000040EA014015E0FF2C08D80098FF2805D8EC
:10FD10000199FF2902D80299FF2903D9002004B0D4
:10FD2000BDE8F0810199000640EA0140029940EAED
:10FD30000120044305E008A3F92216A118A0F8F752
:10FD40006FF8B8F1000F04D0204601F04BFCC8F862
:10FD500000000120E3E700002E2E2F4D6964646C43
:10FD60006577617265732F54686972645F50617260
:10FD700074792F4C7749502F7372632F636F7265BC
:10FD80002F697076342F6970345F616464722E63FA
:10FD900000000000756E68616E646C6564000000B0
:10FDA000417373657274696F6E2022257322206619
:10FDB00061696C6564206174206C696E65202564DE
:10FDC00020696E2025730A001022014900F002B854
:10FDD000F4BD02202DE9FC430023006889466C46EF
:10FDE0001E464FF00A0C01AD0090002094F80080F0
:10FDF000B8FBFCF70CFB1787B8FBFCF884F8008015
:10FE000030372F54401CC0B2B8F1000FEED106E0DD
:10FE10001F465B1C974209DA2F5C01F8017B401EEC
:10FE2000C0B2F5D218465B1C904202DB0020BDE850
:10FE3000FC832E20761CF6B2641C01F8010B042E04
:10FE4000D3D3002001F8010C4846F0E7F8B59446FA
:10FE50000F461C46054604230E4A61463846069E58
:10FE600009F0AAF998B16946384609F0DDF90A485F
:10FE70000099006809E04268914205D13346224664
:10FE8000294600F00BF8F8BD00680028F3D1F120F6
:10FE9000F8BD0000D0860408040B001010B50968F6
:10FEA0001446062912D2DFE801F01103050A0C0EF0
:10FEB000406801E004F08EFF2060002010BD8068E3
:10FEC000FAE70120F8E741F6FC40F5E7F12010BD24
:10FED0002DE9F0418EB00646042000901F46904662
:10FEE0000D4611F8042B06AB01A808F0F2FF1248EA
:10FEF00004680AE00AA9201D08F042FE23460422F5
:10FF00000AA901A808F0B6FF2468002CF2D19DF8D8
:10FF1000120018B1F1200EB0BDE8F0819DF810205C
:10FF20002846039909F044F83B4642463146059875
:10FF3000FFF7B4FFEFE70000040B00102DE9FF41CD
:10FF400015460C461E4607460523164A29462046F6
:10FF5000DDF8288009F030F910B325786946201DB6
:10FF600009F062F9002403AB02AA01A92046FCF7BC
:10FF700097F990B1029804F02DFFA8420DD1DDE968
:10FF800000010968884208D1434632463946204676
:10FF900000F00AF804B0BDE8F081641C0A2CE2D33A
:10FFA000F120F7E710870408FEB51D4614460E46FB
:10FFB00002AB01AA6946FCF773F93068012807D043
:10FFC000022809D003280CD004280FD0F120FEBD50
:10FFD000019804F0FFFE06E00298206006202860E9
:10FFE00002E00098006820600020FEBD0320FAE7D0
:10FFF0002DE9F04393B007460520009098469146BE
:020000040803EF
:100000000D4611F8042B0CAB05A808F062FF002484
:100010006E4611AB0BAA0AA92046FCF741F968B15C
:100020000B9804F0D7FE0090311D0A9808F0A8FD47
:1000300023460522694605A808F01CFF641C0A2C0B
:10004000E7D39DF8220018B1F12013B0BDE8F0838A
:100050009DF820202846079908F0AAFF43464A4603
:1000600039460998FFF7A0FFEFE700002DE9FC41B2
:1000700094460F461E4605460423144A61463846F8
:10008000089C09F099F8F8B101A9384609F0CCF8B4
:10009000019939B90E48006820B133462A4601213A
:1000A00000940AE00B480CE0D0E901231A408A4290
:1000B00007D133462A460021009400F00DF8BDE830
:1000C000FC8100680028EFD1F120F8E7F0860408F1
:1000D000080B0010040B00102DE9F04117681C46B6
:1000E0000022069E1D4B551E0E2F34D2DFE807F06E
:1000F00033070F12171717191E231525172A09B1D1
:1001000018681DE0D0E901100140216020E004F0F2
:1001100061FE15E009B1012012E0226018E02560BF
:1001200016E009B1C0680BE0406809E009B104209D
:1001300006E0032004E0022002E00029E0D180680C
:10014000206005E00648416821600078800030604A
:100150000020BDE8F081F120FBE700004C8304089B
:10016000308404082DE9F04190B0804604200090CE
:100170001E4617460D4611F8042B0AAB01A808F0DD
:10018000A8FE204C206848B106A91F4808F0F8FCDA
:10019000042206A901A8236808F06CFE1B48046825
:1001A00010E000BFD4E9010108400E9009D006A973
:1001B0000EA808F0E5FC2346042206A901A808F0D1
:1001C00059FE2468002CEDD19DF8120018B1F120E1
:1001D00010B0BDE8F0810EA90AA809F025F89DF835
:1001E00010202846039908F0E3FE0E98009630B1DF
:1001F00000213B4642460598FFF76EFFE8E70121E4
:10020000F7E70000080B00104C830408040B0010F3
:1002100010B5040006D106A34FF4317213A116A045
:10022000F7F7FEFD2146BDE81040052002F0E0BFD3
:100230002E2E2F4D6964646C6577617265732F543F
:10024000686972645F50617274792F4C7749502FDE
:100250007372632F636F72652F697076342F6970C4
:10026000345F667261672E63000000007020213DDC
:10027000204E554C4C000000417373657274696FD9
:100280006E2022257322206661696C65642061748A
:10029000206C696E6520256420696E2025730A0034
:1002A000006842682648182A47D2DFE802F0460C68
:1002B0000E101316191C1F2225282B2E3033363909
:1002C0003C3F46464642022034E0FF2032E0D0F870
:1002D00038012FE0D0F8FC002CE0D0F8000129E034
:1002E000D0F8340126E0D0F8040123E0D0F808016A
:1002F00020E0D0F80C011DE0D0F810011AE0D0F891
:10030000140117E0D0F8180114E00F2012E0D0F823
:1003100030010FE0D0F81C010CE0D0F8200109E01A
:10032000D0F8240106E0D0F8280103E0D0F82C0131
:1003300000E00020086004207047002070470000A3
:1003400048BB02202DE9F05F4C68064693460F46F5
:1003500000254FF00108608801F046F921784FF040
:10036000FF3A0907890E814231D8A0EB0109E088E4
:1003700001F03AF9C0047C68010C0020206001EB18
:10038000090083B2A180E3808B4220D3726829E008
:100390005068B0F804C0614515D222606DB1B5F85F
:1003A00006C0614513D38088834210D82F60A0888F
:1003B000844506D04FF0000803E08088834206D8C9
:1003C00077608AB12EE002D0C288914202D25046B4
:1003D000BDE8F09F25B1EA88624501D04FF00008E2
:1003E00002680546002AD3D195B1E888A1888842E1
:1003F00006D92AA34FF4DB7237A13FA0F7F710FD0F
:100400002F60E888A18888420CD04FF0000809E0EE
:10041000706830B121A34FF4DF7241A136A0F7F725
:10042000FFFC7760BBF1000F02D1B07FC007CFD0D7
:10043000B8F1000F30D07268002A2DD05068808843
:10044000002829D12168204629B14C68C088A1889C
:100450008842F7D020E0B8F1000F1DD032B90FA3C9
:1004600040F2DF123CA124A0F7F7DAFC7068406884
:10047000A04206D109A34FF4F07237A11EA0F7F7EE
:10048000CFFC206830B105A34FF4F17236A11AA059
:10049000F7F7C6FC01209BE7002099E72E2E2F4D91
:1004A0006964646C6577617265732F5468697264FE
:1004B0005F50617274792F4C7749502F7372632F9C
:1004C000636F72652F697076342F6970345F66725E
:1004D00061672E6300000000636865636B206672CD
:1004E00061676D656E747320646F6E2774206F761C
:1004F00065726C6170000000417373657274696F9E
:100500006E2022257322206661696C656420617407
:10051000206C696E6520256420696E2025730A00B1
:100520006E6F2070726576696F7573206672616791
:100530006D656E742C2074686973206D75737420FA
:1005400062652074686520666972737420667261E2
:10055000676D656E7421000073616E697479206344
:100560006865636B0000000076616C6964617465A6
:100570005F646174616772616D3A6E6578745F7013
:10058000627566213D4E554C4C00000070B5044626
:100590000C480D464168A14202D1216841600AE041
:1005A000002D06D108A340F2451216A11CA0F7F7B2
:1005B00037FC206828602146BDE87040042002F026
:1005C00017BE0000100B00102E2E2F4D6964646CB6
:1005D0006577617265732F54686972645F506172E8
:1005E00074792F4C7749502F7372632F636F726544
:1005F0002F697076342F6970345F667261672E637D
:100600000000000073616E69747920636865636B34
:10061000206C696E6B6564206C6973740000000067
:10062000417373657274696F6E2022257322206690
:1006300061696C6564206174206C696E6520256455
:1006400020696E2025730A002DE9F0470546002435
:100650000F46A94205D132A3AB2240A142A0F7F731
:10066000DFFB002F08D03868A84205D02CA3AD22AC
:1006700047A13DA0F7F7D4FB4A484FF48038D0F8A3
:100680002011491CC0F820116E687068818800290B
:100690001AD100686860142205F108017068EFF74C
:1006A00095FE01213046FEF78DFC304605F04FF8EF
:1006B0000446404505D31AA3BC223BA12AA0F7F764
:1006C000AFFB304605F016FA6E6812E07068B1466E
:1006D0000668484605F03BF80444444505D310A39A
:1006E000CC2231A120A0F7F79BFBA4B2484605F02D
:1006F00001FA002EEAD139462846FFF747FF324D6E
:100700002888A04205D206A3D22230A116A0F7F76E
:1007100087FB2888001B28802046BDE8F087000062
:100720002E2E2F4D6964646C6577617265732F544A
:10073000686972645F50617274792F4C7749502FE9
:100740007372632F636F72652F697076342F6970CF
:10075000345F667261672E63000000007072657618
:1007600020213D2069707200417373657274696F56
:100770006E2022257322206661696C656420617495
:10078000206C696E6520256420696E2025730A003F
:10079000707265762D3E6E657874203D3D206970DF
:1007A0007200000048BB022070627566735F66725B
:1007B000656564202B20636C656E203C3D2030789D
:1007C0006666666600000000100B001069705F72BC
:1007D000656173735F70627566636F756E74203EDA
:1007E0003D2070627566735F667265656400000027
:1007F0002DE9F0471D4F8946064600240022134686
:1008000011461546786822E0D0F814C0D6F80C805E
:10081000C4450BD1D0F818C0D6F81080C44505D116
:10082000B0F80CC0B6F80480C44509D06D1C2AB1DC
:1008300090F81FC092F81F80C44501D8024619469F
:10084000D0F800C0BCF1000F00D00346604600287D
:10085000DAD11AB11046FFF7F7FE04444C4501DA2D
:10086000012DCBDC2046BDE8F0870000100B001006
:1008700070B50948002544680BE0E07F20B1401EB8
:10088000E0772546246804E0204624682946FFF7DF
:10089000DBFE002CF1D170BD100B001001460A20C8
:1008A00009684968012905D0022902D11168FF2988
:1008B00003D0704711680229FBD100207047002047
:1008C0007047000010B5040006D108A340F2CE2204
:1008D00015A118A0F7F7A4FA606908B105F00AF9A4
:1008E0002046BDE81040FFF793BC00002E2E2F4D90
:1008F0006964646C6577617265732F5468697264AA
:100900005F50617274792F4C7749502F7372632F47
:10091000636F72652F697076342F6970345F667209
:1009200061672E630000000070637220213D204E3D
:10093000554C4C00417373657274696F6E202225AB
:100940007322206661696C6564206174206C696E35
:100950006520256420696E2025730A0038B5104C87
:1009600001204FF4FA65207003462246D0210D483D
:100970000095F1F74BFEF0F7A1FC00280ED0012303
:100980002246D02107480095F1F750FDF0F796FC7C
:10099000002803D0207840F3C010401C38BD000070
:1009A0006C0000205C02002010B5040004D019B1D6
:1009B00012B16368934201D3002010BD01EB031014
:1009C0005B1C4FF0FF316360816041600021C160BA
:1009D00010BD000070B50C46050004D01CB10A46DD
:1009E000042902D005E0002070BD12A1EFF751FDEF
:1009F00030B128462246042C04D0052A04D007E052
:100A0000012070BD0DA100E00EA1EFF742FD30B155
:100A10002146284600F05AF918B1032070BD022083
:100A200070BD2146284600F020F90028F8D00420A7
:100A300070BD00006E756C6C00000000747275650E
:100A40000000000066616C73650000002DE9F0474E
:100A50000500089891460C466BD0002C69D0002701
:100A600069683E4600B9EE60287BAA6865E000BF71
:100A700001EB001CDCF80880DCF804C0E0455AD02B
:100A800001EB001C9CF810C0BCF1060F51D1801C7A
:100A90004CE0BC467F1CFFB2CC4546D101EB0017B1
:100AA0003878052806D0032817D004281FD002283C
:100AB00028D03EE0052B3CD11CB32046EFF7D4FCF8
:100AC00001462046EFF7A9FCD7E901010A1A296877
:100AD00001442046EFF77AFC21E0032B29D184B1B1
:100AE000286879680844EFF73FFD206017E0042B81
:100AF0001FD134B1286879680844F7F735FA84EDD6
:100B0000000B0CE0022B14D14CB1D7E901010A1AF9
:100B1000296801440BA0EFF7BCFC18B12670012036
:100B2000BDE8F08701202070F9E7401CC0B2824286
:100B3000AFD80220F4E7401CC0B2824298D8072008
:100B4000EEE7000074727565000000002DE9F047C3
:100B5000040008981E461546894676D0B9F1000F64
:100B600073D067684FF00008A8B9C4F80C8012E091
:100B700007EB0010017805290AD18168406881429D
:100B800006D00A1A216801444846EFF782FC48B1B2
:100B9000E068401CE060D4E902108842E8D30720F6
:100BA000BDE8F087E06807EB0011087C06284AD012
:100BB000052808D003281CD0042824D002282DD0D2
:100BC00007283DD041E0052E3FD135B32846EFF749
:100BD0004BFC01462846EFF720FCE06807EB0010CD
:100BE000816940690A1A216801442846EFF7EEFB43
:100BF0002DE0032E29D185B1206849690844EFF71B
:100C0000B3FC286023E0042E1FD135B12068496968
:100C10000844F7F7A9F985ED000B18E0022E14D16E
:100C2000ADB1D1E905022168121A014409A0EFF71C
:100C300030FC10B185F8008009E00120287006E042
:100C4000072E04D001E0062E01D00220A8E70120E3
:100C5000A6E70000747275650000000018B111B1BC
:100C6000C16000F04DBA0220704770B5040024D076
:100C700011B9EFF7F9FB0146207800222D2800D1A9
:100C8000012200231D461DE0A05CA0F130060A2EC3
:100C900017D32E2804D0652805D0452803D00CE0B2
:100CA0005BB901230DE0901C884206D2A018407861
:100CB0002B2801D02D2800D10DB1002070BD0125B9
:100CC000521C521C8A42DFD3012070BD2DE9F04135
:100CD000040001D019B105E00020BDE8F081EFF774
:100CE000C3FB0146227800202D2A00D101200026D6
:100CF000871CB94209D9225C302A06D122185278C1
:100D0000782A01D0582A00D101260125024600F197
:100D1000010C20E0A35CA3F1300EBEF1090F12D943
:100D20004EB1A3F1410EBEF1050F0DD9A3F1610E35
:100D3000BEF1050F08D962450AD1782B01D0582B96
:100D400006D1B94204D92EB1824203D1302B01D051
:100D5000002502E0521C8A42DCD32846BDE7000091
:100D60002DE9F04190B004461B4802901B480390C7
:100D70004FF4807009901E4690460F46000101F026
:100D800065FD050025D002A90CA8FFF767FF09A89B
:100D9000009022892B460CA8616800F0D3F814213A
:100DA00004A8EFF73AFBE06808906068CDE9040515
:100DB00009980690002007900948CDE90A78066056
:100DC00033460AA904A82268FCF708F903992846C3
:100DD000884710B0BDE8F0814D2803080DE80208EF
:100DE000680000202DE9F0410E46069F040005D062
:100DF00026B11AB113B10FB1256815E00220BDE884
:100E0000F081092914D00A2912D00D2910D02029E7
:100E10000ED02C290CD05D290AD07D2908D03A2982
:100E200006D0401C20601AB12068315C0029E8D14E
:100E30003A4619462046FFF7B7FD07000FD0206855
:100E4000411B7019FFF7C6FD38707D602068B860DF
:100E50000020F8602068401E20600120CFE70320BA
:100E60002560CCE72DE9F0410400069F06D029B1AA
:100E700022B11BB117B12568681C57E00220BDE8FC
:100E8000F081222E02D05C2E13D04DE03A46194656
:100E90002046FFF789FD48B1052101706D1C4560B2
:100EA000216881600021C1600120E8E703202560FE
:100EB000E5E7401C904237D220600E5C662E33D0AE
:100EC00008DC222E30D02F2E2ED05C2E2CD0622E7D
:100ED00035D129E06E2E27D0722E25D0742E23D046
:100EE000752E2CD1401C4FF0000C206014E000BF88
:100EF000A0F1300EBEF10A0F07D3A0F1410EBEF1F2
:100F0000060F02D36138062819D2761C0CF1010CA9
:100F10002660BCF1040F05D22668964202D2885D95
:100F20000028E5D1701E20602068401C206090429F
:100F300002D20E5C002EA4D1052025609FE704207C
:100F400025609CE72DE9F84F1D460A9E1746894605
:100F500004000DD0B9F1000F0AD04FB145B13EB138
:100F6000306828B1204600F0CBF8D4F804803BE08C
:100F70000220BDE8F88F82462C2872D00EDC0D28A6
:100F80002FD005DC09282CD0BAF10A0F14D128E0A3
:100F9000202826D0BAF1220F0ED171E05D284AD068
:100FA00005DC3A2840D0BAF15B0F05D125E07B285B
:100FB00023D0BAF17D0F3ED0306800902B463A46E0
:100FC00049462046FFF70EFF0128D2D1A06808F15C
:100FD0000108411C05D000BF05EB0010C168491C89
:100FE000C1602068401C20602268BA4203D219F810
:100FF00002000028BFD160687AE008F101082946A4
:1010000020463268FFF7D0FC88B1A1684A1C04D0A2
:1010100005EB0111CA68521CCA60BAF17B0F08D0F7
:1010200006210170216841606068401E56E003207F
:101030009FE70721F5E7606808E000BF05EB0011B6
:101040004B685B1C02D08B685B1C04D0401EF5D53E
:10105000411C07D011E04FF0FF33521CA3608A609F
:10106000F6E71FE0042084E705EB00114A68521CF4
:1010700002D08968491C31D0401E0028F4DAB0E75C
:10108000306800902B463A4649462046FFF7EAFE74
:101090000128CDD1A06808F10108411CA1D0002D84
:1010A0009AD19EE7A068411C9BD005EB0010007808
:1010B000062896D0072894D060680CE005EB001154
:1010C0000A78062A01D0072A05D14A68521C02D0A4
:1010D0008968491C02D0401EF0D582E7A06080E7F5
:1010E00005EB00114A68521C02D08968491C05D0E2
:1010F000401EF5D50120C6F800803AE7052038E704
:1011000030B1002101604160491E816001207047BB
:101110000220704700B5F7F7ABF8012807D15B2034
:1011200000F02EF902205DF804EB00F011B900BDCB
:1011300008B102A000E003A000F014B87472756555
:101140000000000066616C736500000010B5044982
:101150000C4602F01DF92046BDE8104000F002B830
:10116000901E002010B50446F7F782F8012804D13C
:101170002046BDE8104000F015B910BD10B504467A
:10118000F7F776F8012804D12046BDE8104000F0BA
:1011900013B910BD30B50E4CE06A012804D1D4F863
:1011A000340118B10D20E062E06A30BD94F834508B
:1011B000D4F8380110B10A2000F0E2F8012D04D073
:1011C0005FF05D0000F0DCF8EEE77D20FAE700005C
:1011D000841E002030B50C4CE06A012810D1D4F8F0
:1011E000340104EBC000836B00F084F80546002B4B
:1011F00001DD00F091F8012D04D05D2000F0C0F871
:10120000E06A30BD7D20F9E7841E002000B5F7F7C5
:1012100051F8012807D15B2000F0B2F802205DF8F8
:1012200004EB00F095B800BD09B102A100E003A1F4
:1012300000F026B8747275650000000066616C737A
:101240006500000070B50A46054904460D46104683
:1012500002F09EF829462046BDE8704000F010B824
:10126000901E002000B5F7F725F8012807D17B2054
:1012700000F086F801205DF804EB00F069B800BDCD
:1012800010B50C46F7F716F8012804D12046BDE842
:10129000104000F087B810BD10B50C46F7F70AF8FB
:1012A000012804D12046BDE8104000F085B810BDEB
:1012B0002DE9F0411E4614460F460546EFF7ADF8FE
:1012C0000B480021C0E90057856080F834408163F5
:1012D000C0F834110121C162C0F838610163012CEA
:1012E00004D05B20BDE8F04100F04AB87B20F9E76C
:1012F000841E0020074AD2F8341102EBC10090F896
:10130000340019B1491EC2F8341170470C21D16262
:1013100070470000841E002030B50A4DD5F8380112
:1013200000280DD00A2000F02BF8002403E006A0CE
:1013300000F038F8641CD5F83401401CA042F6DCFB
:1013400030BD0000841E002020202020000000006E
:101350000A49D1F83421521C202A02DB0B20C86232
:101360007047C1F8342101EBC20282F83400D1F891
:101370003421002001EBC20188637047841E0020E5
:10138000074910B50B688A684C68D31AA34202D388
:101390000820C86210BD10708868401C886010BDAD
:1013A000841E002010B5044602E0641CFFF7E8FF2D
:1013B00020780028F9D110BD10B50446222000E0A5
:1013C000641CFFF7DDFF20780028F9D1BDE810404C
:1013D0002220FFF7D5BF70B506460D4601F11A0071
:1013E00000F017F804463078032805D105F1140001
:1013F00000F00FF844EA0044204670BDC1788278BE
:1014000042EA01214278007842EA012140EA0120C3
:1014100070474178007840EA0120704710B528B144
:101420000069FDF723F808B1012010BD002010BDB0
:101430002DE9F84F0020044600902F480AF06DF97E
:101440002E48F0F7B4FA05462B480AF08DF915B18D
:101450000020BDE8F88F2948818FD0F8409009041A
:10146000090C2ED04FF4C172002003F029FF009028
:1014700038B32248009D40F2F45BD0F830806E898A
:1014800000270FE0A4F2F4525242EEF79FFFD8F883
:101490000C008046D0F808903F1BAAF2F4560024B6
:1014A00007F2F457686806EB040ADA4509EB040111
:1014B0003844E7D83246EEF789FF2D683444002DD2
:1014C000DDD10E480022016B05E00B6843F00043BC
:1014D0000B60C968521C836B9342F6D8002181636C
:1014E000006800F580504269120602D580224261F0
:1014F00081600098ADE70000E00A0010CC68002091
:101500002DE9F05F27480D46C66A00208346044651
:10151000D6F808A031E0306800280CDB6F894FF066
:10152000000818E0A4F2F4525242EEF74FFFF668BA
:101530003068002802DA6FF0070025E0D6F808A02E
:10154000A8EB040000F2F458ABEB0400A9F2F45746
:1015500000F2F45B002407EB040940F2F4518945E2
:1015600069680AEB04004144DCD83A46EEF72EFFE6
:101570000BEB07002D683C448346002DCBD1014680
:101580000848F0F789FC00200649096801F58051F8
:101590004A69920603D520224A6100224A60BDE8CA
:1015A000F09F0000CC68002010B5044640688047DA
:1015B0000AF0DDF8094A216852688B181A1AB2F14C
:1015C000004F03D308442246054902E0044922465D
:1015D0001846BDE810400AF085B90000E40100207B
:1015E000A915030800BA704740BA704710B509F052
:1015F000E3FE0AF031F801F02BFB01F047FE03F0A7
:101600008DFA11F039FC0BF083FEBDE810400AF0B2
:10161000E5B910B5026804466FF00501506830B1B5
:10162000127802F0F002102A09D0202A02D00846CF
:10163000207110BDA289A16811F002FAF8E7A28911
:10164000A1680AF0D3FEF3E770B5016804466FF0B5
:101650000A024B684878002B4DD00B780125B5EB7A
:10166000131F48D1237A032B01D0022843D003282B
:1016700041D001283CD0D80702D0084602F0D0FA69
:101680002068406A30B11DA340F2BD7228A12FA08E
:10169000F6F7C6FB216804204870206800214462E8
:1016A000206800F06DF8002824D0206840780428D5
:1016B00006D012A340F2C2722EA124A0F6F7B0FB0E
:1016C0002E480AF051F8206800210C3009F080FF04
:1016D0002A480AF022F82068407800280AD0BDE89D
:1016E000704006A340F2C67222A118A0F6F798BB7C
:1016F000FB20207170BD227170BD00002E2E2F4D79
:101700006964646C6577617265732F54686972648B
:101710005F50617274792F4C7749502F7372632F29
:101720006170692F6170695F6D73672E63000000DF
:10173000616C72656164792077726974696E672083
:101740006F7220636C6F73696E670000417373651D
:101750007274696F6E2022257322206661696C6540
:1017600064206174206C696E6520256420696E2098
:1017700025730A007374617465210000E00A00108B
:101780002DE9F0478A46040006D169A340F2A2324F
:1017900074A178A0F6F744FB20780121B1EB101F6B
:1017A00006D063A340F2A3327CA172A0F6F738FB07
:1017B0006078042806D05EA34FF469727FA16DA003
:1017C000F6F72EFB606830B959A340F2A53284A128
:1017D00068A0F6F725FB606A30B955A340F2A6323F
:1017E00084A164A0F6F71CFB606AD4F80480007A38
:1017F00000F0010900F0020703280FD0B9F1000F33
:1018000007D098F81400052808D0062806D0082824
:1018100004D04FB198F81A00C00605D50126002162
:1018200040460AF0DFFD00E0002698F81400012889
:101830001DD0B9F1000F07D0002140460EF02CFC5E
:10184000002140460AF0C7FC1FB1002140460FF0BE
:1018500075F996B10022114640460DF04FFC00216B
:1018600040460BF071FB40460AF066FE0AE000219C
:1018700040460AF0B0FC002EF5D13A4649464046B3
:101880000FF0AEF905000ED0681C0CD1606A407AEA
:1018900020B198F8140001282FD035E01EB1404641
:1018A0000AF096FC0025606A0168057100206062FC
:1018B00001F10C086070BDB936B16060A36A1BB15C
:1018C0000022042120469847B9F1000F05D0A36AF1
:1018D0001BB100221146204698472FB1A36A1BB1C5
:1018E0000022022120469847BAF1000F02D040465C
:1018F00009F075FF0020BDE8F0870DA340F24142DA
:1019000043A11CA0F6F78CFA1FB14A4940460FF0DC
:1019100015F90122484940460DF0F0FB4749404681
:101920000BF012FB214640460AF05CFD2846E2E738
:101930002E2E2F4D6964646C6577617265732F5428
:10194000686972645F50617274792F4C7749502FC7
:101950007372632F6170692F6170695F6D73672E99
:1019600063000000696E76616C696420636F6E6E5F
:1019700000000000417373657274696F6E20222548
:101980007322206661696C6564206174206C696EE5
:101990006520256420696E2025730A0074686973C8
:1019A00020697320666F7220746370206E657463A3
:1019B0006F6E6E73206F6E6C79000000636F6E6ED9
:1019C000206D75737420626520696E207374617474
:1019D00065204E4554434F4E4E5F434C4F53450098
:1019E00070636220616C726561647920636C6F73EF
:1019F00065640000636F6E6E2D3E63757272656E76
:101A0000745F6D736720213D204E554C4C000000E3
:101A1000436C6F73696E672061206C697374656EC7
:101A200020706362206D6179206E6F742066616939
:101A30006C210000C1780308E5660308DDBD0208DB
:101A400010B5044600684368002B11D0017801F0FE
:101A5000F001102915D020290DD031A340F27D527C
:101A60003CA142A0F6F7DCF96FF00500207110BD33
:101A70006FF00E00FAE7A2891846A16811F07AF813
:101A8000F4E74178032903D029B16FF00900EDE7AD
:101A90006FF00800EAE706F003F82068A289A16861
:101AA00040683C4B0AF00EFF0028DFD1206803227B
:101AB00090F8201042702068C1F34001002910F80E
:101AC000201F05D041F0040101706FF00400CDE744
:101AD00001F0FB010170206844622068407803280F
:101AE00006D00FA34FF4AE622BA120A0F6F798F911
:101AF0002B4809F039FE206800210C3009F068FD00
:101B0000274809F00AFE206840780328AFD1BDE8D5
:101B1000104003A340F274521FA114A0F6F780B93D
:101B20002E2E2F4D6964646C6577617265732F5436
:101B3000686972645F50617274792F4C7749502FD5
:101B40007372632F6170692F6170695F6D73672EA7
:101B500063000000496E76616C6964206E65746391
:101B60006F6E6E20747970650000000041737365BC
:101B70007274696F6E2022257322206661696C651C
:101B800064206174206C696E6520256420696E2074
:101B900025730A00A51B0308737461746521000096
:101BA000E00A001070B50025164604000CD06078DD
:101BB000032806D025A340F2235231A138A0F6F71E
:101BC0002FF9606A18B10FE06FF0050070BD94F84E
:101BD000200040070CD41DA340F224523AA130A0AB
:101BE000F6F71EF9606A18B10671606A05680C356F
:101BF00020780121B1EB101F03D116B9204605F062
